:020000040801F1
:1000000020C900206D3B010851620508593B0108D9
:10001000593B0108593B0108593B0108593B01086C
:10002000000000000000000000000000C53B0108C7
:10003000593B010800000000113E0108B5A4010869
:10004000CD3E0108CD3E0108CD3E0108CD3E010860
:10005000CD3E0108CD3E0108CD3E0108CD3E010850
:10006000CD3E0108CD3E0108CD3E0108CD3E010840
:10007000CD3E0108CD3E0108CD3E0108CD3E010830
:10008000CD3E0108CD3E0108CD3E0108CD3E010820
:10009000CD3E0108CD3E0108CD3E0108CD3E010810
:1000A000CD3E0108CD3E0108CD3E0108CD3E010800
:1000B000CD3E0108CD3E0108CD3E0108CD3E0108F0
:1000C000CD3E0108CD3E0108CD3E0108CD3E0108E0
:1000D000CD3E0108CD3E0108CD3E0108CD3E0108D0
:1000E000CD3E0108CD3E0108CD3E0108CD3E0108C0
:1000F000CD3E0108CD3E0108CD3E0108CD3E0108B0
:10010000CD3E0108CD3E0108CD3E0108CD3E01089F
:10011000CD3E0108CD3E0108CD3E0108CD3E01088F
:10012000CD3E0108CD3E0108CD3E0108CD3E01087F
:10013000CD3E0108CD3E0108CD3E0108CD3E01086F
:10014000CD3E0108CD3E0108CD3E0108CD3E01085F
:10015000CD3E0108CD3E0108CD3E0108CD3E01084F
:10016000CD3E0108CD3E0108CD3E0108CD3E01083F
:10017000CD3E0108CD3E0108CD3E0108CD3E01082F
:10018000CD3E0108CD3E0108CD3E0108CD3E01081F
:10019000CD3E0108CD3E0108CD3E0108CD3E01080F
:1001A000CD3E0108CD3E0108CD3E0108CD3E0108FF
:1001B000CD3E0108CD3E0108CD3E0108CD3E0108EF
:1001C000CD3E0108CD3E0108CD3E0108CD3E0108DF
:1001D000CD3E0108CD3E0108CD3E0108CD3E0108CF
:1001E000CD3E0108CD3E0108CD3E0108CD3E0108BF
:1001F000CD3E0108CD3E0108CD3E0108CD3E0108AF
:08020000CD3E0108CD3E0108CE
:1002080081F0004102E000BF83F0004330B54FEABF
:1002180041044FEA430594EA050F08BF90EA020F2C
:100228001FBF54EA000C55EA020C7FEA645C7FEABF
:10023800655C00F0E2804FEA5454D4EB5555B8BFE2
:100248006D420CDD2C4480EA020281EA030382EA53
:10025800000083EA010180EA020281EA0303362DE5
:1002680088BF30BD11F0004F4FEA01314FF4801CB8
:100278004CEA113102D0404261EB410113F0004FCA
:100288004FEA03334CEA133302D0524263EB430381
:1002980094EA050F00F0A780A4F10104D5F1200E1F
:1002A8000DDB02FA0EFC22FA05F2801841F100017A
:1002B80003FA0EF2801843FA05F359410EE0A5F14E
:1002C80020050EF1200E012A03FA0EFC28BF4CF07F
:1002D800020C43FA05F3C01851EBE37101F0004535
:1002E80007D54FF0000EDCF1000C7EEB00006EEB42
:1002F8000101B1F5801F1BD3B1F5001F0CD34908CC
:100308005FEA30004FEA3C0C04F101044FEA445222
:1003180012F5800F80F09A80BCF1004F08BF5FEAA9
:10032800500C50F1000041EB045141EA050130BD89
:100338005FEA4C0C404141EB0101013C28BFB1F59B
:10034800801FE9D291F0000F04BF01460020B1FAE6
:1003580081F308BF2033A3F10B03B3F120020CDAB9
:100368000C3208DD02F1140CC2F10C0201FA0CF097
:1003780021FA02F10CE002F11402D8BFC2F1200CFC
:1003880001FA02F120FA0CFCDCBF41EA0C019040B2
:10039800E41AA2BF01EB0451294330BD6FEA0404FB
:1003A8001F3C1CDA0C340EDC04F11404C4F12002E6
:1003B80020FA04F001FA02F340EA030021FA04F3F8
:1003C80045EA030130BDC4F10C04C4F1200220FA4F
:1003D80002F001FA04F340EA0300294630BD21FA8D
:1003E80004F0294630BD94F0000F83F4801306BF53
:1003F80081F480110134013D4EE77FEA645C18BF47
:100408007FEA655C29D094EA050F08BF90EA020FDD
:1004180005D054EA000C04BF1946104630BD91EAD5
:10042800030F1EBF0021002030BD5FEA545C05D1D8
:100438004000494128BF41F0004130BD14F5800417
:100448003CBF01F5801130BD01F0004545F0FE418B
:1004580041F470014FF0000030BD7FEA645C1ABFC0
:10046800194610467FEA655C1CBF0B46024650EAF7
:10047800013406BF52EA033591EA030F41F4002123
:1004880030BD00BF90F0000F04BF0021704730B5A9
:100498004FF4806404F132044FF000054FF000017E
:1004A80050E700BF90F0000F04BF0021704730B53F
:1004B8004FF4806404F1320410F0004548BF404214
:1004C8004FF000013EE700BF42004FEAE2014FEA69
:1004D80031014FEA02701FBF12F07F4393F07F4F44
:1004E80081F06051704732F07F4208BF704793F047
:1004F8007F4F04BF41F40021704730B54FF460745A
:1005080001F0004521F000411CE700BF50EA01025C
:1005180008BF704730B54FF000050AE050EA010205
:1005280008BF704730B511F0004502D5404261EB75
:1005380041014FF4806404F132045FEA915C3FF4B6
:10054800D8AE4FF003025FEADC0C18BF03325FEA53
:10055800DC0C18BF033202EBDC02C2F1200300FA04
:1005680003FC20FA02F001FA03FE40EA0E0021FA29
:1005780002F11444BDE600BF70B54FF0FF0C4CF417
:10058800E06C1CEA11541DBF1CEA135594EA0C0FC9
:1005980095EA0C0F00F0DEF82C4481EA030621EA04
:1005A8004C5123EA4C5350EA013518BF52EA03353F
:1005B80041F4801143F4801338D0A0FB02CE4FF0F1
:1005C8000005E1FB02E506F00042E0FB03E54FF021
:1005D8000006E1FB03569CF0000F18BF4EF0010E19
:1005E800A4F1FF04B6F5007F64F5407404D25FEA15
:1005F8004E0E6D4146EB060642EAC62141EA5551C8
:100608004FEAC52040EA5E504FEACE2EB4F1FD0C09
:1006180088BFBCF5E06F1ED8BEF1004F08BF5FEA87
:10062800500E50F1000041EB045170BD06F0004639
:1006380046EA010140EA020081EA0301B4EB5C04E6
:10064800C2BFD4EB0C0541EA045170BD41F48011DE
:100658004FF0000E013C00F3AB8014F1360FDEBF03
:10066800002001F0004170BDC4F10004203C35DADF
:100678000C341BDC04F11404C4F1200500FA05F362
:1006880020FA04F001FA05F240EA020001F0004203
:1006980021F0004110EBD37021FA04F642EB060179
:1006A8005EEA430E08BF20EAD37070BDC4F10C04A3
:1006B800C4F1200500FA04F320FA05F001FA04F267
:1006C80040EA020001F0004110EBD37041F1000153
:1006D8005EEA430E08BF20EAD37070BDC4F120055E
:1006E80000FA05F24EEA020E20FA04F301FA05F2C6
:1006F80043EA020321FA04F001F0004121FA04F26E
:1007080020EA020000EBD3705EEA430E08BF20EA3D
:10071800D37070BD94F0000F0FD101F00046400077
:1007280041EB010111F4801F08BF013CF7D041EAF9
:10073800060195F0000F18BF704703F000465200FD
:1007480043EB030313F4801F08BF013DF7D043EACE
:100758000603704794EA0C0F0CEA135518BF95EA84
:100768000C0F0CD050EA410618BF52EA4306D1D10B
:1007780081EA030101F000414FF0000070BD50EA2A
:10078800410606BF1046194652EA430619D094EAB4
:100798000C0F02D150EA013613D195EA0C0F05D19E
:1007A80052EA03361CBF104619460AD181EA0301F2
:1007B80001F0004141F0FE4141F470014FF00000AA
:1007C80070BD41F0FE4141F4780170BD70B54FF045
:1007D800FF0C4CF4E06C1CEA11541DBF1CEA1355C5
:1007E80094EA0C0F95EA0C0F00F0A7F8A4EB0504A7
:1007F80081EA030E52EA03354FEA013100F088809E
:100808004FEA03334FF0805545EA131343EA126366
:100818004FEA022245EA111545EA10654FEA00261B
:100828000EF000419D4208BF964244F1FD0404F5D4
:10083800407402D25B084FEA3202B61A65EB030530
:100848005B084FEA32024FF480104FF4002CB6EBED
:10085800020E75EB030E22BFB61A754640EA0C006D
:100868005B084FEA3202B6EB020E75EB030E22BFAD
:10087800B61A754640EA5C005B084FEA3202B6EBEE
:10088800020E75EB030E22BFB61A754640EA9C00AD
:100898005B084FEA3202B6EB020E75EB030E22BF7D
:1008A800B61A754640EADC0055EA060E18D04FEA3B
:1008B800051545EA16754FEA06164FEAC30343EADB
:1008C80052734FEAC2025FEA1C1CC0D111F4801FA8
:1008D8000BD141EA00014FF000004FF0004CB6E7A1
:1008E80011F4801F04BF01430020B4F1FD0C88BF40
:1008F800BCF5E06F3FF6AFAEB5EB030C04BFB6EB4B
:10090800020C5FEA500C50F1000041EB045170BD3D
:100918000EF0004E4EEA113114EB5C04C2BFD4EB6A
:100928000C0541EA045170BD41F480114FF0000EEE
:10093800013C90E645EA060E8DE60CEA135594EA6A
:100948000C0F08BF95EA0C0F3FF43BAF94EA0C0F6D
:100958000AD150EA01347FF434AF95EA0C0F7FF4E2
:1009680025AF104619462CE795EA0C0F06D152EA36
:1009780003353FF4FDAE1046194622E750EA41061A
:1009880018BF52EA43067FF4C5AE50EA41047FF42B
:100998000DAF52EA43057FF4EBAE12E74FF0FF3C90
:1009A80006E000BF4FF0010C02E000BF4FF0010C61
:1009B8004DF804CD4FEA410C7FEA6C5C4FEA430CDA
:1009C80018BF7FEA6C5C1BD001B050EA410C0CBF29
:1009D80052EA430C91EA030F02BF90EA020F00208B
:1009E800704710F1000F91EA030F58BF994208BFF2
:1009F80090422CBFD8176FEAE37040F001007047AF
:100A08004FEA410C7FEA6C5C02D150EA013C07D105
:100A18004FEA430C7FEA6C5CD6D152EA033CD3D050
:100A28005DF8040B704700BF8446104662468C464A
:100A38001946634600E000BF01B5FFF7B7FF00287D
:100A480048BF10F1000F01BD4DF808EDFFF7F4FFA6
:100A58000CBF012000205DF808FB00BF4DF808ED31
:100A6800FFF7EAFF34BF012000205DF808FB00BF54
:100A78004DF808EDFFF7E0FF94BF012000205DF876
:100A880008FB00BF4DF808EDFFF7CEFF94BF01202B
:100A980000205DF808FB00BF4DF808EDFFF7C4FF24
:100AA80034BF012000205DF808FB00BF4FEA410277
:100AB80012F5001215D211D56FF47873B3EB6252A8
:100AC80012D94FEAC12343F0004343EA505311F0CF
:100AD800004F23FA02F018BF404270474FF0000061
:100AE800704750EA013005D111F0004008BF6FF09F
:100AF800004070474FF00000704700BF4FEA4102C6
:100B0800B2F1E04324BFB3F5001CDCF1FE5C0DD963
:100B180001F0004C4FEAC0024CEA5070B2F1004FAD
:100B280040EB830008BF20F00100704711F0804FB0
:100B380021D113F13872BCBF01F00040704741F475
:100B480080114FEA5252C2F11802C2F1200C10FA79
:100B58000CF320FA02F018BF40F001004FEAC1235D
:100B68004FEAD32303FA0CFC40EA0C0023FA02F301
:100B78004FEA4303CCE77FEA625307D150EA0133D7
:100B88001EBF4FF0FE4040F44000704701F00040A7
:100B980040F0FE4040F40000704700BF80F0004085
:100BA80002E000BF81F0004142001FBF5FEA41033D
:100BB80092EA030F7FEA226C7FEA236C6AD04FEA3D
:100BC8001262D2EB1363C1BFD21841404840414082
:100BD800B8BF5B42192B88BF704710F0004F40F434
:100BE800000020F07F4018BF404211F0004F41F450
:100BF800000121F07F4118BF494292EA030F3FD01C
:100C0800A2F1010241FA03FC10EB0C00C3F120032E
:100C180001FA03F100F0004302D5494260EB4000BD
:100C2800B0F5000F13D3B0F1807F06D340084FEA28
:100C3800310102F10102FE2A51D2B1F1004F40EB1D
:100C4800C25008BF20F0010040EA03007047490085
:100C580040EB0000013A28BFB0F5000FEDD2B0FA22
:100C680080FCACF1080CB2EB0C0200FA0CF0AABF45
:100C780000EBC25052421843BCBFD04018437047E3
:100C880092F0000F81F4000106BF80F400000132E9
:100C9800013BB5E74FEA41037FEA226C18BF7FEAC0
:100CA800236C21D092EA030F04D092F0000F08BF02
:100CB8000846704790EA010F1CBF0020704712F0E9
:100CC8007F4F04D1400028BF40F00040704712F128
:100CD80000723CBF00F50000704700F0004343F08D
:100CE800FE4040F4000070477FEA226216BF0846C3
:100CF8007FEA23630146420206BF5FEA412390EA86
:100D0800010F40F4800070474FF0000304E000BF7B
:100D180010F0004348BF40425FEA000C08BF70472C
:100D280043F0964301464FF000001CE050EA0102F0
:100D380008BF70474FF000030AE000BF50EA010205
:100D480008BF704711F0004302D5404261EB4101F2
:100D58005FEA010C02BF84460146002043F0B64317
:100D680008BFA3F18053A3F50003BCFA8CF2083A3C
:100D7800A3EBC25310DB01FA02FC634400FA02FC45
:100D8800C2F12002BCF1004F20FA02F243EB02004C
:100D980008BF20F00100704702F1200201FA02FCAE
:100DA800C2F1200250EA4C0021FA02F243EB0200A1
:100DB80008BF20EADC7070477BB972B90029BEBF52
:100DC80000204FF0004106E008BF00281CBF6FF06C
:100DD80000414FF0FF3000F077B8ADF1080C6DE935
:100DE80004CE002909DB002B1ADB00F0A9F8DDF896
:100DF80004E0DDE9022304B07047404261EB4101A1
:100E0800002B1BDB00F09CF8DDF804E0DDE9022391
:100E180004B0404261EB4101524263EB4303704727
:100E2800524263EB430300F08BF8DDF804E0DDE9A0
:100E3800022304B0404261EB41017047524263EB28
:100E4800430300F07DF8DDF804E0DDE9022304B097
:100E5800524263EB4303704753B94AB9002908BFAC
:100E680000281CBF4FF0FF314FF0FF3000F02CB8C6
:100E7800ADF1080C6DE904CE00F062F8DDF804E08D
:100E8800DDE9022304B07047D0B5FFF71DFB00224F
:100E98000B4B06460F46FFF76FFB00F017F80446AA
:100EA800FFF7F0FA0022074BFFF766FB02460B46F6
:100EB80030463946FFF7A8F900F008F82146D0BDBA
:100EC8000000F03D0000F041704700BF4A0011D219
:100ED80012F5001211D20DD56FF47873B3EB62528C
:100EE8000ED44FEAC12343F0004343EA505323FA98
:100EF80002F070474FF00000704750EA013002D10D
:100F08004FF0FF3070474FF00000704710F8012B8A
:100F180011F8013B012A28BF9A42F7D0D01A70472E
:100F2800034611F8012B03F8012B002AF9D1704769
:100F3800034613F8012B002AFBD1181A0138704711
:100F48002DE9F0478C468E46089E154604461946FC
:100F5800002B40F0D080724547D9B2FA82F74FB1E2
:100F6800C7F120030EFA07FCBD40BC4020FA03F38A
:100F780043EA0C0C4FEA154EA8B2230CBCFBFEF852
:100F88000EFB18CC08FB00F943EA0C43994528D915
:100F9800EB1808F1FF3204D2994502D9A8F10202F0
:100FA8002B44A3EB0903A4B2B3FBFEFC0EFB1C33DA
:100FB8000CFB00F044EA0344A04214D92C190CF1AC
:100FC800FF3304D2A04202D9ACF102032C44241A04
:100FD80043EA02401EB1FC40002334607360BDE860
:100FE800F0874246DDE76346F1E7002A79D0B2FA96
:100FF80082F3002B3FD01946C1F1200302FA01F514
:1010080000FA01F42EFA03F20EFA01FE20FA03F3B5
:10101800AFB243EA0E034FEA154EB2FBFEFC0EFBDD
:101028001C201A0C0CFB07F842EA004290455AD9DA
:10103800AA180CF1FF3004D2904502D9ACF1020095
:101048002A44A2EB08029BB2B2FBFEFC0EFB1C2258
:101058000CFB07F743EA02439F4246D9EB180CF111
:10106800FF3204D29F4202D9ACF102022B44DB1BAF
:1010780042EA004202E0AEEB020301224FEA154EBB
:10108800AFB2200CB3FBFEFC0EFB1C330CFB07F8C5
:1010980040EA034398452AD9EB180CF1FF3004D2F3
:1010A800984502D9ACF102002B44A3EB0803A4B283
:1010B800B3FBFEFC0EFB1C330CFB07F744EA0344AE
:1010C800A74216D92C190CF1FF3304D2A74202D932
:1010D800ACF102032C44E41B43EA00400F461146DE
:1010E80078E71F2188E76046ABE76246BFE76046BE
:1010F800DBE76346EFE7734506D916B900210846D2
:101108006DE7C6E9000EF9E7B3FA83F787B97345C7
:1011180001D3824207D8841A6EEB030301209C4650
:101128001EB900215BE73846FAE7C6E9004CF8E744
:10113800C7F1200CBB4000FA07F422FA0CF520FA9C
:101148000CF1BA401D432EFA0CF30EFA07FE4FEAD3
:10115800154941EA0E011FFA85FEB3FBF9F809FBB0
:1011680018300B0C08FB0EFA43EA00439A4540D9A5
:10117800EB1808F1FF3004D29A4502D9A8F1020011
:101188002B44A3EB0A0389B2B3FBF9F809FB183324
:1011980008FB0EFE41EA03418E452CD9691808F177
:1011A800FF3304D28E4502D9A8F10203294443EA49
:1011B8000040A1EB0E01A0FB02984145CE464346F4
:1011C80002D306D14C4504D20138B9EB020E68EBC4
:1011D8000503002EA5D0B4EB0E0261EB030101FA62
:1011E8000CFC22FA07F3F9404CEA0303C6E9003184
:1011F80097E74046C5E74346D9E7000000000000EE
:101208002DE9F04F984685B000F15803C0E9163330
:10121800129B0026838104239FED257B073222F051
:10122800070A0374119B01EB0A090F4680ED087B3E
:101238004946C0E9066686608373C6730446DDF8CE
:1012480038B002F03BFA109BC51D25F00705C4F81D
:101258008850C4E9207A02930F9BA9EB0505CDE9D4
:1012680000B32A4643463946204602F031FD0F9B1B
:10127800C4E91B8B6367109B6665A367EFF3118254
:10128800102383F31288BFF36F8F0B4B596A5C628C
:10129800E16782F31188BFF36F8F9B680BB1D3F8B6
:1012A8008C302846C4F88C3005B0BDE8F08F00BFFC
:1012B80000000000000000009C3B0020000000002F
:1012C8002DE9F0412DED028B90F8A5300446B0EEE3
:1012D800408A86B01BB9F7EE007A37EEC08AD4F898
:1012E80084202F4B9A4213D118EE100AFFF7ECF81E
:1012F80029A3D3E90023FFF7CFFB011E18BF012163
:1013080004F184000EF07CFB84ED268A012005E0C0
:10131800B4F89C30B3F5807F05D1002006B0BDEC51
:10132800028BBDE8F08104F15008404629F0DAF854
:101338000028F2D0DFED1B7A68EE277AFCEEE77A18
:10134800CDED037A94F8806094F89C209DF80C30D9
:10135800276E206D6EB18DF8153002238DF814209C
:1013680000210122009305ABB847404653F0CDF861
:10137800CAE7012531468DF813208DF814302A4626
:101388000DF113030095B847009532462946276E9C
:10139800206D05ABE8E700BFAE47E17A14AEEF3F3A
:1013A8004CC7070800007F432DE9F04F044685B07D
:1013B80008466160062190461D469DF838709DF8E4
:1013C8003CB01DF06BFEA060067C16F0010602D052
:1013D8007D4812F05DFC9DF8403005FB08F084F86C
:1013E8002A309DF844307D3084F828307E2390FBE5
:1013F800F3F0C0010430C4E90485277360624EF03D
:10140800D7F90DF1080A0622C4E907066F492046F4
:10141800A66159F0BCFA022251462046ADF8088070
:1014280059F0B5FA022251462046ADF8085059F055
:10143800AEFAF623032269462046ADF800308DF84F
:10144800026059F0A4FA7B1EDBB2082B05D840F2E3
:101458005515DD4015F0010501D15D48B9E7052FA7
:1014680009D0072F06D0032F73D1012384F8293020
:10147800002502E02E4684F82960002646F34F1026
:10148800C0EB0020FFF70EF80022524BFEF7BEFE1D
:101498000022514BFFF79AF9FFF708FB5FFA80F833
:1014A800C6F38200C0EB0020FEF7FCFF00224B4B86
:1014B800FEF7ACFE00224A4BFFF788F9FFF7F6FA71
:1014C800C7B206F00300C0EB0020FEF7EBFF0022D6
:1014D800404BFEF79BFE00223F4BFFF777F9FFF7E3
:1014E800E5FAC0B2002D5ED08DF808008DF80980AD
:1014F8008DF80A70032251462046013659F047FA02
:10150800802EBBD1BBF1000F1AD0364D01A92A8815
:10151800AB782046ADF8042003228B7059F037FAD7
:101528000B222046304959F032FAD5F80300EB79FE
:1015380002900522514620468AF8043059F027FACD
:10154800204659F012FAA06959F033FA05B0BDE8FF
:10155800F08F092F84F829608AD10FF25C09D9E944
:101568000089354616A7D7E900672846FEF79AFF8F
:1015780042464B46FEF74AFE32463B46FFF726F9FF
:10158800FFF794FAC0B28DF808008DF809008DF8BD
:101598000A00032251462046FF3559F0F8F9B5F5FF
:1015A800FF4FE2D1AEE78DF808808DF809708DF80D
:1015B8000A009FE7AFF300800000000000C04F4022
:1015C8000000000000C05F40B08608082A680808CC
:1015D800F57D08080000F83F0000084000000C40B6
:1015E80000001C403B3F0708316808080000000065
:1015F80010EE103A33F0004210B52DED028B06D1F3
:101608000120BDEC028BBDE8104042F079BF002BF1
:1016180005DABDEC028BBDE8104042F07FBFB3F1A4
:10162800FF4F06DB30EE008AB0EE480ABDEC028BB5
:1016380010BDB3F5000F6049BBBFDFED607A6FF0F6
:101648001802002260EE277AB8BF17EE903AF7EE3C
:10165800007ADC15C3F316037F3C1944144401F4E3
:10166800000282F07E5204EBD15403F10F011A43B9
:1016780007EE102A524A0A4037EE678AB2BBB5EE27
:10168800408AF1EE10FA0FD1002C00F08C8007EEA2
:10169800904A9FED4C0A9FED4C7AF8EEE77A27EED8
:1016A800808A07EE878ABFE741A1D1E90001FFF7E9
:1016B80025FAB6EE007A07EE900A07EEC87A68EEC9
:1016C800087A27EE277A14B938EE478AACE707EE8E
:1016D800904ADFED3C6AF8EEE77A07EEE67A37EEF5
:1016E800488A9FED397A17EE878A9DE7F0EE007AEF
:1016F8009FED365ADFED364A364A78EE277A1A4495
:10170800C3F5571388EE276A07EE904A03F522734C
:101718001343F8EEE76ADFED307A002B66EE065ADF
:1017280025EEA57A07EE275ADFED2C7A45EE077AE3
:101738009FED2B5A07EE875ADFED2A7A47EE274AA4
:10174800DFED297A44EE877A67EE877A45EE257AC7
:101758001ADDB6EE007A28EE077A27EE087A77EED9
:10176800877A67EE867A14B937EE677AACE79FED29
:10177800156A46EE867A37EE677A37EE488ADFEDE5
:10178800127A16EEA78A4FE778EE677A67EE867ABE
:1017980014B938EE678A47E79FED0A7A46EEC77AAA
:1017A80037EEC88AEBE79FED118A3DE7AFF300807B
:1017B800555555555555D53F20FB4A000000004C5E
:1017C800F0FF7F00D1F717378071313F25333A3E5C
:1017D800298E633E305CCFFF9788173E2549923E9D
:1017E800ABAA2A3F4FD01C3ECDCCCC3E0000000017
:1017F800F8B510EE904A10EE103A34F000472DED8F
:10180800048BB0EE609A0DD183F480035B0013F56E
:10181800000F40F2AA8230EE098AB0EE480ABDEC09
:10182800048BF8BD23F000411846B1F1FF4F02D8F0
:10183800B7F1FF4F08D9B3F17E5FECD184F480048F
:10184800640014F5000FE4E7002B25DAB7F1974F91
:1018580080F09482B7F17E5F39D3FA15C2F196020F
:1018680047FA02F505FA02F2BA4229D105F0010554
:10187800C5F10205B7F17E5F2AD1002C80F27B8288
:10188800B5EE400AF1EE10FA1CD1D80FBDEC048B6E
:10189800BDE8F84042F034BEB7F1FF4F10D1B1F1C6
:1018A8007E5F00F0628205D9002CDFEDD17A29FE37
:1018B800278AB2E7002C80F25B82B1EE498AACE756
:1018C8000025D7E7B7EE007A87EE008AA5E700255E
:1018D800B4F1804F0A4640F05782B1F1BF4F0CD2A5
:1018E800B1F1D05F02D920EE008A96E7B0EEC08A47
:1018F80059BB012D00FE088A8FE723F04046B0EE61
:10190800C08AB6F17E5F17D1002CBCBFB7EE007A53
:1019180087EE088A002B80DAA1F17E51294305D190
:10192800BDEC048BBDE8F84042F0F8BD012D7FF412
:1019380074AFB1EE488A70E739B9002CD9DA002BB8
:10194800A4D06B1E58425841A0E7DE0F013E55EA6D
:101958000600E5D0B7F19A4F71D9A64B994208D83D
:10196800002C0BDA0020BDEC048BBDE8F84042F0F7
:10197800B9BDA14B994208D9002CF3DC0020BDEC7D
:10198800048BBDE8F84042F09FBDB7EE007ADFED6A
:101998009B7ADFED9B9A38EE478A93A1D1E9000143
:1019A80068EE278AFFF7AAF8B5EE007A07EE900AE4
:1019B800DFED946A68EE299A48EE477AB6EE007A27
:1019C80007EEC87A68EE087A27EE277AF0EE687A8A
:1019D80047EE667A39EEA77A17EE103A6FF30B03E3
:1019E80007EE103A77EE699A77EEE97A013DF7EE5D
:1019F800006ABFEE008A6FF30B04354367EE890A6D
:101A080008FE268A06EE904A39EE666A67EE267A5E
:101A180046EE070A30EEA77A17EE101A002921F0D1
:101A2800004340F31381B3F1864F40F2CC80B5EE0A
:101A3800C08AF1EE10FA4CBF0120002093E713F0A2
:101A4800FF4F05BF9FED707A6FF01701002168EE18
:101A5800077A08BF17EE902AD315C2F316027F3B08
:101A680042F07E500B4469498A4206DD68498A4241
:101A780040F3A7800133A0F500000021654A06EE77
:101A8800100AF7EE006A02EB8102D2ED005A75EEF9
:101A9800867A36EE657AC6EEA74A27EE245A15EE00
:101AA800102A6FF30B0206EE902A5B4A02EA6002E4
:101AB80042F0005202F5800202EB415207EE902AF2
:101AC80006EEE77A77EEE57ADFED545A36EE676A86
:101AD80065EE057A06EE667A9FED516A47EE865AFC
:101AE8009FED506A27EE247A66EEA64A05EEA76AAD
:101AF800DFED4D5A46EE275A9FED4C6A05EEA76A70
:101B0800DFED4B5A46EE275A36EE856A67EEA77A1E
:101B180026EE076A05EEA76AF0EE085A74EEA57A73
:101B280077EE867A17EE902A6FF30B0207EE902A6B
:101B380077EEE55A27EE277A66EEA76A75EEE45A3D
:101B480036EE656A06EE057A9FED3A6A76EE877A92
:101B580017EE902A6FF30B0207EE902A364A77EEBB
:101B6800E66A02EB810227EE866A37EE667ADFEDD7
:101B7800336A67EEA67ADFED326A47EE267A92ED8F
:101B8800007A77EE877A07EE103A2E4BF8EEC76A9E
:101B980003EB810336EE277AD3ED005A37EE257A28
:101BA80037EE267A17EE103A6FF30B0307EE103A6A
:101BB80077EE666A76EEE56A76EEC66A77EEE67ADC
:101BC80014E701215AE755D1DFED1F6A37EE677A2E
:101BD80070EEA66AF4EEC76AF1EE10FA3FF727AF87
:101BE80086234BE0AFF30080E13D55555555D53F71
:101BF80000000000F3FF7F3F0700803F70A5EC3630
:101C080000AAB83F3BAAB83F0000804B71C41C0033
:101C1800D6B35D00F0FE070800F0FFDF55326C3EDA
:101C280042F1533E05A38B3EABAAAA3EB76DDB3EFD
:101C38009A99193F0040763FE0FE0708C623F6B898
:101C48004F38763FE8FE07083CAA3833534A934298
:101C580007D9B5EEC08AF1EE10FA4CBF012000207A
:101C68008DE607D137EE677AB4EEE07AF1EE10FA36
:101C7800B6DBEEE7B3F17C5F72D9DB157E3B4FF440
:101C88000000474A002940FA03F00844C0F3C7534C
:101C9800A3F17F0342FA03F2C3F1170302EA000239
:101CA800C0F3160040F4000007EE102A40FA03F0D3
:101CB80077EEC77AB8BF404237EEA07ADFED396ACF
:101CC800DFED395AB7EE000A9FED386A17EE103A81
:101CD8006FF30B0307EE103A77EE677A67EE266A22
:101CE80070EEE70ADFED327A27EE277ADFED317AF8
:101CF80000EEA77A76EE877A77EEE66A37EE667AAE
:101D080067EEA76A07EE877A16EEA56ADFED2A5A0C
:101D180046EE265A9FED296A15EEA66ADFED285A87
:101D280046EE265AB0EE676A05EEE66AF0EE006AFD
:101D380067EE865A36EE666AC5EE866A36EEC77A6A
:101D480077EE677A30EE670A10EE103A03EBC0536D
:101D5800B3F5000F06DA42F03BFA20EE088A5CE59C
:101D68000020A9E700EE103AF7E7B7EE008A54E53D
:101D78009FED148A51E5B0EE408A4EE5B7F1FF4F6A
:101D88003FF48DAD0A460225B4F17C5F7FF4B5AD12
:101D9800002BFFF6B2ADB1EEC08A3EE50000164357
:101DA800000080FF0072313F4CBB31330EEADD3555
:101DB8008CBEBF351872313F55B38A38610B363B3C
:101DC800ABAA2A3E0000000010EE103AB3F1FF4F14
:101DD80010B52DED048BB0EE408A06DB30EE008A9C
:101DE800B0EE480ABDEC048B10BD774A934276DC0E
:101DF80023F00042B2F17E5F13D3FFEE007AB4EE17
:101E0800670AF1EE10FA06D10120BDEC048BBDE89B
:101E1800104042F075BBBDEC048BBDE8104042F0A9
:101E28007DBBB2F1645F0FD2B2F14A5F24BF20EEEE
:101E3800007AF6EE007ABDEC048B28BF07EE670A3D
:101E4800BDE8104042F07EB9604A134493424ED830
:101E5800F7EE007A38EE277A17EE103ADC157F3C59
:101E6800002CD5BF77EE677A37EE488A78EE677A26
:101E780077EEC87A87EE879AC3F31603544A9342DB
:101E8800CCBF43F07C5243F07E52F7EE007AC8BFD5
:101E9800C3F5000307EE102AC4BF01349B1037EEC8
:101EA800678AF6EE008A68EE288A68EE888A002B30
:101EB80044D1B5EE408AF1EE10FA1DD1002C7AD04B
:101EC80007EE904AB0EE498A9FED427AF8EEE77A3B
:101ED80007EE878A9FED407A07EE878A80E7B3F19D
:101EE800B44FB5DBDC159FED3D9A7F3CC4E7012379
:101EF80000249FED3A9AD4E731A1D1E90001FEF719
:101F0800FDFDB7EE007A07EE900A07EEC87A27EED5
:101F1800287A14B938EE478A62E707EE904ADFED6F
:101F28002D6AF8EEE77A07EEA69A37EE497A37EE89
:101F3800488A9FED297A17EE878A51E7F0EE007AF2
:101F48009FED276A9FED277A78EE277AC8EE276AF1
:101F580066EEA67A07EE867A9FED236A07EE276A71
:101F68009FED227A06EE277A9FED216A07EE276A0F
:101F78009FED207A06EE277A9FED1F6A07EE276A03
:101F8800B0EE687A06EE277A27EE267A24B978EE3C
:101F9800C78A38EE688A23E707EE904ADFED0D6AB4
:101FA800F8EEE77A07EEA69A39EE079A78EEC98A2C
:101FB80038EEC88ABDE79FED098A11E7AFF30080C4
:101FC800555555555555E53FD613D43EE0096A4158
:101FD800F6043500D1F717378071313F0000000053
:101FE8009788173E4FD01C3E25333A3E298E633ED4
:101FF8002549923ECDCCCC3EABAA2A3F2DE9F047ED
:102008000546884600AF42F0CAFEA9680646B1F503
:10201800004F36BFA8F10403002303F00703B1F50E
:10202800004F34BF0420082002F0070407341C4482
:102038000444E40804EBD2048C4228BF0C46012275
:102048003146284642F065FE10EA020A16D1E946F2
:1020580088B06A46504BCDE90538032342F8103F53
:102068004FF4C25153464D4800F09EFECD468AF3C8
:102078001188BFF36F8F0423184602DF31462846C4
:1020880042F05DFE06EB000949460022284642F070
:1020980040FEA9EB00094E4518D0E94688B06946CC
:1020A8003F4BCDE90538032341F8103F3B48134621
:1020B8000A464FF4C25100F077FE0023CD4683F361
:1020C8001188BFF36F8F0423184602DF3146284674
:1020D80042F035FE8442804623D028D2344431462B
:1020E8002246284642F0EDFE01223146284642F0BB
:1020F8002CFE214642F023FE2618012231462846AE
:1021080042F007FEC30708D43146284642F089FE4C
:1021180032462146284642F0FBFE2146284642F038
:1021280015FF4FF001094846BD46BDE8F08706EBAC
:10213800000A01225146284642F0EBFD10EA020946
:1021480027D15146284642F0FAFD40448442EAD855
:102158005146284642F065FE5146284642F0EFFDBA
:10216800A4EB0808804509D2344451462846224643
:1021780042F0A7FE2146284642F0E8FE5246314684
:10218800284642F0C5FE01223146284642F0DDFDD0
:10219800C7E74FF00009C6E7EC080808543E0708EF
:1021A800100908082DE9F843884600AF00297DD0BA
:1021B80005680122284642F0F2FD014604462846F9
:1021C80042F0A7FD10EA020616D1E94688B06A4631
:1021D800384BCDE90538032342F8103F4FF4C2517C
:1021E8003346354800F0E0FDCD4686F31188BFF34D
:1021F8006F8F0423184602DF2146284642F09FFDD0
:10220800261831460022284642F083FD361AB44289
:1022180018D06E4688B06946284BCDE905380323A7
:1022280041F8103F244813460A464FF4C25100F0C3
:10223800BBFD0023B54683F31188BFF36F8F0423DA
:10224800184602DF00222146284642F07EFD21463C
:1022580042F075FD261801223146284642F059FD04
:10226800C20708D43146284642F0DBFD32462146F3
:10227800284642F04DFE00222146284642F049FDFC
:10228800261A01223146284642F043FDC30709D4E5
:102298003146284642F0C5FD22463146284642F0DE
:1022A80037FE34462146284642F050FEBD46BDE87A
:1022B800F88300BF39090808543E070810090808C0
:1022C80008B5024843F0DDF9002008BD6609080892
:1022D8000E4A0346904202D30D4A904211D30D4A4A
:1022E80022B1934202D30C4A93420AD30B4A52B109
:1022F8000B48834234BF01200020934238BF00209E
:102308007047012070471046704700BF78380708AB
:10231800309D0808000000000000000000000000D8
:10232800000000002DE9F04F9BB000AF04468B463B
:10233800D7F890A0FA637B6349B903784678807828
:1023480000EB830020445E4522D8A0EB040B0AF082
:10235800010394F80280FB62E378B8F1000F0CBF28
:102368004FF000090AF001093B6313B11AF0020F9C
:1023780017D1B9F1000F14D1FB6B1BB15946204698
:102388007A6B98475D4628466C37BD46BDE8F08FA6
:10239800451C2846FEF7CCFD013028440BF1010B03
:1023A800D1E7CAF3C003FB612378BB629B00BB6122
:1023B80063683B62BB6A04EB8301FB6B002B7DD136
:1023C8005D468844B9F1000F1DD08B469946A94E49
:1023D8001BF8013B54F82300002808BF3046FEF7DD
:1023E800A7FDD7F8943001304BB1D7F898304B455A
:1023F80082BFD7F8943023F8190009F10109C345C1
:102408000544E5D1D8461AF0050F0CBF4FF0020B72
:102418004FF0010B00260AF00203FB633B6B9E4260
:10242800B1D298F8013008F1020854F823A05046B8
:10243800FFF74EFFFA69034602B3B86318F8021CA7
:10244800386A43F0FFF8BB6BC0B1EA468AB06A4607
:10245800894B05933B6ACDE906314FF40073ADF81B
:102468002030864B42F8103F00234FF41251844825
:1024780000F09AFCD546023D0136CFE723B1FB6A4E
:102488002BB9A5EB0B05F7E7FB6B002BF4D07948CC
:10249800BAF1000F18BF5046FEF74AFDD7F894303E
:1024A80053B1D7F8983099453FBFD7F89420431CCB
:1024B80022F8193009F101090544DDE7B9F1000FE7
:1024C8006DD04346102B28BF10230026BB6397F816
:1024D800389007F14800BA6B796260F0F1FE796ACA
:1024E80000227A620AF0020201EB08033A610AF05C
:1024F80004027B61FA6002337A6A396B8A4267D3D5
:102508006378F96A1AF0020F7B624B4418BF002205
:10251800DBB208BF7208002940F0A9801AF0040F46
:1025280014BF314600216370A170E27020467A6BB7
:10253800B969FB6B9847051EFFF625AFBB6A3146A4
:1025480023707B6A7A6B63703B6B84F80280E3705C
:1025580007F15800FB6B9847061EC0F2C5803A6B1E
:10256800BB69386B03EB4203ABEB0301D7E90D23DF
:10257800C91A7B6903EB4000FB6B98470028C0F23F
:10258800B5804FF000082E44351807F1480AC845B1
:1025980078D300217A6B0846FB6B9847F3E6B8F1CD
:1025A800000F0CD01AF0040F0ED04346102B28BF92
:1025B8001023BB6397F8386007F158008BE746464D
:1025C800C146C7F838808BE74E46C7F8388087E79A
:1025D80013F8015C13F8021C54F82500BB60FFF7E0
:1025E80077FE0246F869BB6838B1386AC7E9013234
:1025F80043F028F8D7E90132F0B912B3FA6A72B198
:10260800B9F10F0F18D809F1280107F1400009F1B5
:102618000102014401F8205C5FFA82F90CE0FA68D3
:1026280052B10F2E08D806F1280107F14000721C9C
:102638000E1806F8105CD6B27A6A023301327A6252
:102648005AE73A69002ADBD10F2EF5D806F128009F
:1026580007F1400C6044721C00F8101C07F1680177
:10266800023651FA82F2F6B202F8105CE4E7002171
:1026780059E700BF940908089B09080804000001ED
:10268800AC3D070818F80A3054F823B087F84730EB
:10269800D7F8943033B3D7F89830984522D2D7F882
:1026A800943033F8186001217A6BFB6B07F147000F
:1026B800984700281ADB0E4B0544BBF1000F08BFF2
:1026C8009B4626B95846FEF733FC461CB6B231463F
:1026D80058467A6BFB6B9847002807DB054408F1DE
:1026E800010854E70026DEE735464CE605464AE68B
:1026F80094090808014B1860704700BF800100204A
:10270800044608B5EFF31183102383F31288BFF34F
:102718006F8F46F051FC204601F03EFA024842F025
:10272800B0FF43F0B2FDFCE74F0A0808034A002057
:10273800536823F002035360704700BF004004E071
:1027480008B5094A136943F0005313614168074803
:102758000C3183681B681BB1984700EAE07008BD1C
:102768006FF05700F9E700BF0008024688390708EC
:10277800082810B502D90024204610BD044B53F890
:102788002040204647F0D2F80028F5D1F3E700BFF3
:102798001443070810B5EFF31184102383F312884C
:1027A800BFF36F8F084803683BB9084A916A41F044
:1027B80001019162916AC907FCD50133036084F372
:1027C8001188BFF36F8F10BD7C37002000080246C8
:1027D80010B5EFF31184102383F31288BFF36F8FC2
:1027E80011490B68A3B90122104BD3E8EF1F002948
:1027F80003D1C3E8E02F0028F7D104D102210C4A05
:102808000C4843F08DFB84F31188BFF36F8F10BD24
:10281800012B08BF084803F1FF3302BF826A22F088
:10282800010282620B60EEE77C37002078370020D7
:10283800140B08087C3E07080008024607B505F097
:10284800E9FC0E4B0E4A1A600E4BD3F8942042F066
:102858000402C3F89420D3F8943003F004030193DE
:10286800019B094BDA6A42F00102DA629A6822F0A7
:1028780002029A6003B05DF804FB00BFC80600209E
:1028880000093D00000C0246000802462DE9F04709
:10289800044607464FF00109DFF84C8094FAA4F586
:1028A800B5FA85F509FA05F32E0108EB05156FEA67
:1028B800030A24EA03042B7B63B158F806301B692A
:1028C8006BB94644736802222846196807EA0A0762
:1028D80043F0B6FA002CE1D13846BDE8F087284627
:1028E80098470028F6D1ECE71C3F070810B50022EE
:1028F80088B00E490E4847F072FC002200230024DD
:10290800CDE906230E234FF44072CDE90334CDE917
:102918000144084B08490094084809F0A1FC0849FB
:10292800064847F0BAFA204608B010BD4D290108FC
:1029380068280020592C010800520020802300201C
:102948005C0B0808014809F0D5B900BF54110020F4
:102958002DE9F047804620480F4643F04DFA0646D9
:10296800002832D000252846BDE8F087237B83B1B4
:102978002368DB680BB120469847636883F80690A4
:1029880023681B69CBB9636802222046196843F0A3
:1029980057FA013610345445E8D3B8F1000FE2D0A5
:1029A800002DDFD02846FFF771FF0546002FF7D02E
:1029B8000021642047F073FBF2E72046984700287F
:1029C800E1D009FA06F31D43E3E705464FF0010994
:1029D800024CDFF80CA0DEE7903700201C3F070808
:1029E8002C3F0708014B53F8200070474C43070859
:1029F80008B5034608462BB1044A136000F044FCAE
:102A0800002008BD6FF01500FBE700BF840100201F
:102A180010B5044C237813B9034809F06BF9012366
:102A2800237010BD7E4900205411002010B50446C3
:102A3800094843F0E1F93CB1084BD3E8EF1F0139ED
:102A4800C3E8E21F002AF8D105480AF02BFABDE8CE
:102A58001040044809F04EB9883700208C37002010
:102A680068280020541100200022044BD3E8EF0FFF
:102A7800C3E8E12F0029F9D1704700BF883700204B
:102A880070B5FFF7F1FF0546074C084EB44200D376
:102A980070BD63685B792BB123685B6813B1294605
:102AA800204698471034F1E71C3F07082C3F0708D9
:102AB80010B5044C0449204642F0F1FE034B1C605B
:102AC80010BD00BF6C100020384307088037002075
:102AD80000230D4A10B513700C4A4FF47A71136035
:102AE8000B4A0C481360FFF783FFFFF7E1FF0A4B1F
:102AF8000A4918468B4200D310BD1A1A5C68121195
:102B0800013222711033F5E77F4900208837002011
:102B18008C370020135E05081C3F07082C3F070868
:102B2800014642F210720023014842F0D9BE00BFAC
:102B38006C100020014842F06FBF00BF6C100020ED
:102B4800024B0146186842F0C2BF00BF8037002020
:102B5800014842F0F7BF00BF6C10002070B5254B4C
:102B68001B78002B43D0FFF7E5FF044600283BD134
:102B7800214B224D1B68002B12DD47F0E8FA0A2290
:102B88000023FEF769F9D5E90032C01A40F2E933AB
:102B980061EB0201984271F1000101D3FFF770FF68
:102BA800D5E9003213F57A7342F10002C5E9003223
:102BB800ECB1BDE87040FFF7CBBF6B685B7923B120
:102BC8002B68214628461B6898471035B542F4D330
:102BD8002046FFF7B5FF0A4BD3E8EF1F0139C3E8DA
:102BE800E21F002AC4D0F7E7064D074EEEE70020A3
:102BF80070BD00BF7E490020883700206028002073
:102C08008C3700201C3F07082C3F070870B50D4D76
:102C1800297861B90120FFF79BFE0B4C0B4EB4429B
:102C280006D3FFF79BFF0028FBD101232B7070BD53
:102C380063685B791BB1236820469B68984710340A
:102C4800EDE700BF7F4900201C3F07082C3F07081D
:102C580000212DE9F8430846FFF77AFE044648B3F9
:102C68004FF4FA784FF0000901F03EF91A4B1B4A6D
:102C78001B58136033B11A4B1B68092B02DD194826
:102C880009F038F80025184F44B12046FFF7FEFD3B
:102C9800044618B94FF0FF384FF0FF39FFF75EFFD1
:102CA800064628B9B5B90F4842464B4609F05EF8C2
:102CB8003546E9E74FF0FF384FF0FF39D4E72B6886
:102CC8009B691BB100222846114698471035BD4222
:102CD800F5D3E8E7054DFAE708000000843700203F
:102CE8008C370020541100202C3F07081C3F070890
:102CF80013B5184843F080F8174B1B7873B1EFF3FE
:102D08001184102383F31288BFF36F8FFFF726FF18
:102D180084F31188BFF36F8F02B010BD0F4B1B688F
:102D2800002BF9D050B9002200230D48CDE900232B
:102D380042F2107200230AF08FF8EDE70928EBD170
:102D480007480AF0AFF8074802B0BDE8104008F09D
:102D5800D1BF00BF8C3700207F4900208437002076
:102D6800682800205411002010B5064B04461B6843
:102D780098472146A060044842F02FFEBDE8104065
:102D8800FFF7B6BF840100206C100020044A054BF1
:102D98009B1AB1EBD30F34BF52F8310000207047B3
:102DA8009C3D07081C3F07082DE9F04F8FB0C1F381
:102DB8004A2604AF0D469046B8607B600C0D002E85
:102DC80061D04FF000090A234FF0040B07F1140AF1
:102DD800FE60C7E90799C7F824900093CDF808B0BA
:102DE800CDF804A007F11C034A464046F968FFF7EE
:102DF80099FAB0F5006F03461CD36C468AB0D8F830
:102E0800041004AB24481A46C3E9050140F2FF71D7
:102E1800D9614FF400711984204B42F8103F4FF4E8
:102E280012514B461E48FFF7BFFFA5462C37BD463B
:102E3800BDE8F08FC0F30A0604F11700184420F02B
:102E4800070080083B60FFF76BFE66F353250446D6
:102E580080B13B6800F11001C7E908390A23F9611C
:102E6800CDE901AB009340460E4AF96807F11C030F
:102E7800FFF758FA66F353252A4620467B68B96857
:102E880042F0FEFFD2E704F1170020F007008008A7
:102E9800FFF746FE0446EDE76D0B08080400000145
:102EA8001C3E07085B5E05082DE9F04F87B0054614
:102EB800DDE9106BDDE9127A884614469946BFB100
:102EC80010213B465A460020CDF800A0CDF814A0AA
:102ED80042F0DFF9B0F5006F01460BD340F2FF7303
:102EE8000221184A184807B0BDE8F04F43F021B84E
:102EF8003946384604F0070305F00704E40044EABD
:102F0800831444EA402444EA065406F117000844AE
:102F180020F0070080080391FFF702FE054640B144
:102F28003FB13B465A460399CDF800A0103042F015
:102F3800B0F94B4622464146284607B0BDE8F04F57
:102F480042F09EBFAC0B08081C3E0708406820B141
:102F5800034BC01A40F3CF0070474FF0FF30704763
:102F68009C3D07080EB403B503AB53F8042B014688
:102F78000448019301F0ECF902B05DF804EB03B0EA
:102F8800704700BF9D5F0508CA0605D48B064CBF75
:102F980002490349FFF7E6BF704700BF8D300808B4
:102FA800A22908082DE9F04F8BB099469DF8588062
:102FB800179B044607930D46DDE918A31A9F06924E
:102FC8000593B8F1000F00F0BC80834B07F0020BAB
:102FD80013F80830089307F48073099342F02EFF22
:102FE800024600287AD020467C49FFF7BBFF0646F8
:102FF800BBF1000F08D017F0440F71D12A462046C4
:103008007749FFF7AFFF064407F0010353B1754B4B
:10301800204653F82820744B7449002A08BF1A46E2
:10302800FFF7A0FF07F48073002B07F0080318BF11
:103038004FF00009002B7FD06D4B204653F8282015
:103048006C49FFF78FFF0546069B2BB11A462046B1
:103058006949FFF787FF0544B9F1000F0DD0089BB8
:10306800002B6CD06549664BB8F1040F18BF1946A0
:103078004A462046FFF776FF054462483544079BD9
:103088001BB12246604942F0ACFA059B002B00F0C8
:103098008E80059B3946102B28BF10232046994661
:1030A8000026FFF771FFB54252DC00263346204662
:1030B8001AF803205549FFF755FF0136102E4DD059
:1030C800710703D120465249FFF74CFF4E4533465E
:1030D800EDD320464F49FFF745FFEEE7064687E761
:1030E8004D4B186800288ED04C4B4FF47A7B1B68E8
:1030F8004FF03C0CB5FBF3F5B5FBF0F14FF4616311
:1031080000FB11550BFB05F5B1FBF3F2B5FBF0FE27
:1031180003FB121100FB1E55B1FBFCF30BFB05F57D
:10312800B5FBF0F50CFB131120460091CDE901E544
:103138003B49FFF717FF66E707F0080584E73049C2
:1031480096E7B9F1010F45460CBF2E48354896E77A
:1031580020462F49FFF706FF0136A4E70026204640
:103168003149FFF7FFFE33461AF803202046A2F143
:1031780020035F2B28BF2E222C49FFF7F3FE0136D0
:10318800102E0DD0720703D120462149FFF7EAFE21
:10319800B1453346E8D820461D49FFF7E3FEEEE780
:1031A800059BCA44B3EB090305937FF472AFB8F1EA
:1031B800000F0AD0FB0704D520460B4A0B49FFF73E
:1031C800D1FE39462046FFF7DFFE20460BB0BDE8AA
:1031D800F04F42F0D2BE00BF2C6A0808F20B080874
:1031E800F60B08085C430708E40B0808B530080824
:1031F800704307081C0C0808220C0808E90B08088B
:10320800ED0B08089D5F050859430108260C0808BE
:10321800E4680808E2680808983700209437002016
:10322800000C0808CB5F05082C0C0808CE300808ED
:1032380042F20F7373B58B4228BF0B4605680446EC
:10324800052168460D4A3DF03FFE0646636828465C
:103258000B225B680A4942F082FE6368324669467F
:1032680028465B6842F07BFE63681B2228465B6841
:10327800044942F074FE02B070BD00BF1D2008086A
:10328800206A0808046A080800210123064A9042B7
:1032980006D8064A01B901231360054B1860704728
:1032A800012140085B00F2E740420F0094370020FC
:1032B80098370020F8B50D460446064F4618B44224
:1032C80001D12846F8BD14F8011BBB6801485B68AA
:1032D8009847F4E7643B0708014B036000207047F8
:1032E800B84307082DE9F34205460E4600244FF07F
:1032F8001409084B084F1B680193019BA34202DC89
:1033080002B0BDE8F0823868314609FB0400A847DE
:103318000134F2E7B84307089001002070B5104B5C
:103328000D461C68B4B10F4B196800238B4202DBB1
:103338006FF0010070BD224612F8146B864202D06D
:1033480014460133F2E7E06846F0F0FA28B10020AD
:103358002C60EFE76FF00C00ECE76FF01200E9E784
:1033680090010020B843070810B5436888B002935D
:1033780083680C46CDE9033200230A68C068CDE9AA
:103388000623054901AA059344F09FFF079808B949
:10339800059B236008B010BD5D6105082DE9F84361
:1033A8000646FDF7C5FD0546EFF31188102383F3A4
:1033B8001288BFF36F8F114B1C68D3F804909C429E
:1033C80008BF002434B988F31188BFF36F8F2046F3
:1033D800BDE8F883A7683846FDF7AAFDA84206D1DC
:1033E8002A46394630465FF0B6FF0028EBD04C45F8
:1033F80001D02468E6E70024E5E700BF9401002037
:103408002DE9F0410E461546FFF7C8FF044628B3DC
:10341800C3681BB35F690FB3062E07D0072E20D0F1
:103428002A4631463B46BDE8F0411847838A3BB9F6
:103438002A463146B84750B9A38A0133A38206E029
:103448004FF6FF72934204D00133A3820020BDE8F7
:10345800F0810121114A124842F062FD6FF0150017
:10346800F5E745B12A7832B10022828231462A46F0
:103478005B699847EAE7A38A012B08D12A46072106
:103488002046B8470028E2D1A38A013BD6E70BB112
:10349800013BDAE70221034ADDE700BF800C080898
:1034A800BC3D0708A20C080810B5044608B180689E
:1034B80038B9104A1048012142F032FD6FF015006A
:1034C80010BDFFF76BFF08B10C4AF3E7A082EFF3DA
:1034D8001181102383F31288BFF36F8F084B5A684A
:1034E800C4E9003214605C6081F31188BFF36F8F08
:1034F800E6E700BFC00C0808BC3D0708D90C08085F
:103508009401002080B505460E461746984609F0F6
:10351800C7F9034600F0E8FC0446DFF81890424675
:1035280049F8003039463046A84754F8090000F0F9
:1035380055FC00BF0800000008B50348034A0021F5
:10354800121A42F079FE08BDC0130020FC4D00207D
:10355800074808B5074A0849121A42F06FFEBDE845
:1035680008400648064A0749121A42F067BE00BFDB
:1035780000000020C0130020309D08080000002033
:1035880000000020309D08082DE9F84F80460C46C1
:1035980000AF00296AD0D1E90012E9468AB0A368D1
:1035A8006D464FF0050A6E463948CDE90723CDE947
:1035B800050146F810AF002332464FF42151354833
:1035C800FFF7F2FBD4E90312CD466369AD463248F2
:1035D800C5E90723C5E90501C5F810A0002332464F
:1035E8004FF421512B48FFF7DFFBCD46E36901215A
:1035F8002A4A284842F09DFC0121294A254842F0E0
:103608008FFC264600254FF00A0ADFF8A4B0E946E9
:10361800D6E908C0D6E90A138EB06A46CDF81CC0B0
:1036280005F1010CCDE908C0A81CCDE90A01E91C87
:10363800CDE905B5CDE90C1342F810AF002345F2EA
:10364800400114480435FFF7AFFB102DCD4606F1B5
:103658001006DCD1236E0121124A0E4842F069FCA3
:10366800A3690121104A0B4842F063FCB8F1010F2D
:1036780007D1EFF305830D4A41460648103B42F057
:1036880058FC2146404607F06DFFBD46BDE8F88F5F
:10369800110D08084C3E0708400D08086F0D080872
:1036A8007E0D0808FB0D08080A0E0808380E0808E1
:1036B800B80D080830BFFFF7FDBF00BF2DE9F04186
:1036C80005460B4EDFF83080324606EB0807CC1B68
:1036D800204608495FF0F4FDA01942460021083C45
:1036E8005FF014FEC5F8904007F10800BDE8F081CE
:1036F800000000002C3F07080800000010B5244C0B
:103708002449254842F0A7FDA36A99013ED52248DD
:10371800224942F0A0FD1E20A36ADA0104D51E4802
:103728001F4942F098FD1F20194CA36ADB0204D5FB
:1037380019481C4942F08FFD0220A36A1C0304D5D6
:103748001548194942F087FD2120114CA36A5903F5
:1037580004D51148154942F07EFD2220A36A9A0338
:1037680004D50D48124942F076FD2320084CA36A7F
:10377800DB0304D508480F4942F06DFD2420A36AF5
:103788006FEA03436FEA1343A36210BD1D20C3E72A
:1037980000ED00E04B0E08084C3E0708630E0808D1
:1037A800760E0808900E0808BA0E0808D80E080801
:1037B800FD0E0808170F080870B506460D46294C77
:1037C80029492A4842F047FDA36ADB0647D527481E
:1037D800274942F040FD1120A36A1C0704D523485D
:1037E800244942F038FD12201E4CA36A990712D5CD
:1037F80021491E4842F02FFD636BA26A120609D5C3
:1038080001211E4A194842F094FB1EB1A36A23F015
:103818008003A3621320134CA36ADE0704D5134860
:10382800174942F018FD1420A36A9C0604D50F48D6
:10383800144942F010FD15200A4B9A6AD10658BF68
:103848009A6A9A6A920642BF5A6A22F400525A62E7
:103858009A6A42F0FF029A6200232B7070BD102012
:10386800BAE700BF00ED00E0420F08084C3E070829
:10387800580F08088B0F08089E0F0808B60F08088D
:10388800CC0F0808EB0F080870B506460D46284C03
:103898002849294842F0DFFCA36AD9043CD52648C8
:1038A800264942F0D8FC1720A36A1A0504D52248F5
:1038B800234942F0D0FC18201D4CA36A9B0512D561
:1038C8001D48204942F0C7FCA36BA26A100409D521
:1038D80001211D4A184842F02CFB1EB1A36A23F4AB
:1038E8000043A3621920124CA36A590504D5124853
:1038F800164942F0B0FC1A20A36ADA050ED50E4824
:10390800134942F0A8FC1B20094A936A43F47F43F9
:10391800936200232B7070BD1620C5E7A36A9B0431
:10392800F2D505480B4942F096FC1C20ECE700BF95
:1039380000ED00E01A1008084C3E0708301008088F
:103948008B0F0808411008085A1008086F1008085B
:103958008A100808EB0F0808F0B59DB0664B0546BD
:103968005868002600AFC0F3080386F31188BFF338
:103978006F8F02F07F44B4F17F4F07D102F00C043F
:10398800082C0ED15D495E4842F065FC5D495C48F3
:1039980042F061FC00210846FFF7F6FD7437BD468A
:1039A800F0BD14074CBF0D460126002DEED00022B5
:1039B800FA71DA1E092A7ED8DFE802F005757871F7
:1039C8007D7D7D7D7D7B50494D4842F044FC002340
:1039D800494CFB71E36A9A0705D54C49484842F0BF
:1039E8003AFC00242DE0E36A002B01DA4849F5E7A8
:1039F800E36A5B00F5D54749414842F02CFC63690E
:103A0800AA6943F480736361BFF34F8FBFF36F8F6D
:103A180032F8023C626922F480726261BFF34F8F10
:103A2800BFF36F8F03F47F42B2F55F4F21D1DBB252
:103A3800022B1ED12B680121374A314842F079FA0E
:103A48002C68FB79002BA9D16822294607F10800C8
:103A58005FF036FC7B6A002E4AD0C3F3080222B915
:103A68006FEA53236FEA43237B62204607F108017C
:103A780092E7214B9A6AD2B222B10120F91DFFF7D1
:103A88009BFE0EE09A6A12F47F4F04D00120F91DC4
:103A9800FFF7FAFE05E09B6AB3F5803FA1D3FFF775
:103AA8002DFE0446CDE70020F91DE8E70020F91DAA
:103AB800EEE71A4992E71A4A6C4610F4F87F8AB082
:103AC800184918BF11466A46103B07934FF4007314
:103AD8001548ADF82030154BCDE9050142F8103FE7
:103AE80000234FF411510648FFF75EF9A54678E721
:103AF8006FF30803B8E700BF00ED00E0D010080836
:103B08004C3E0708FB100808371108084E11080832
:103B18006F1108087D1108089C110808B8110808D9
:103B2800B7100808A2100808DC11080804000001F2
:103B3800064B5A6942F010025A615A6942F480628F
:103B48005A615A6922F008025A61704700ED00E094
:103B5800EFF30880EFF3098101B57246FFF7FCFE29
:103B680001BD00BF0A4880F30888102080F311883F
:103B780008484FF40061401880F30988EFF3148077
:103B88000221084380F31488BFF36F8F00F07AF89E
:103B980020C9002000610020BFF34F8F0549064B64
:103BA800CA6802F4E0621343CB60BFF34F8F00BFD3
:103BB800FDE700BF00ED00E00400FA051EF0040F69
:103BC8000CBFEFF30880EFF30980816911F8021C3C
:103BD8000229FFD001B5724642F032FB01BD00BF99
:103BE8000028ACBF00F16040064B4FEA0111C9B292
:103BF800ABBF00F5614000F00F0080F800131954C6
:103C0800704700BF14ED00E040B2002807DB012335
:103C18004109034A00F01F00834042F821307047F1
:103C280000E100E040B200280CDB0122064943090C
:103C380000F01F008240203341F82320BFF34F8F4C
:103C4800BFF36F8F704700BF00E100E0054B4209EA
:103C580053F82220012300F01F0003FA00F010405F
:103C6800704700BF00E100E0044B054A23F07F03E2
:103C78009360BFF34F8FBFF36F8F70470000010849
:103C880000ED00E008B5FFF7EFFF104BD3F88820F0
:103C980022F47002C3F88820D3F8882042F4A002E6
:103CA800C3F888204FF04042C3F83422BFF34F8F47
:103CB800BFF36F8F0023E1EE103AFFF73DFCFFF7EB
:103CC80047FC00F0F3F807F079FD00BF00ED00E0D5
:103CD8008189203A41F0020181814FF47D41C0F889
:103CE800DC101360009B08495360019B21F001011F
:103CF8009360029B9161D3604FF08073D36100237E
:103D08000265C0F8943070470D350108104B9B6868
:103D180083421AD1EFF30580B8B9EFF3118110226D
:103D280082F31288BFF36F8F9A8922F002029A8178
:103D3800EFF3148323F0040383F31488BFF36F8F26
:103D480081F31188BFF36F8F70476FF015007047CC
:103D58009C3B00200E461546002300B5E1EE103AC4
:103D6800EFF3148323F0040383F31488BFF36F8FF6
:103D7800BFF36F8F0C4BD0F8902098600B4B1A60F4
:103D8800D0F8803083F30B882C4686F3098800200E
:103D9800034B98472046002100220023014C20476E
:103DA800856205080D3501089C3B0020C8370020B6
:103DB8001022014B1A61704700ED00E0054B9A692B
:103DC8009B689A421FBF044A536843F0805353606C
:103DD800704700BF9C3B002000ED00E0084B9B684B
:103DE80083420BD1EFF3058343B1064B5A6842F087
:103DF80080525A605A6A22F400425A6246F052B817
:103E08009C3B002000ED00E025498A6882F8DDE04F
:103E18004FF030001044EFF3098C80E8F01F1EF0DB
:103E2800100F03D102F19C0080EC108A102080F35F
:103E38001288BFF36F8F1B4F4FF000668A698A6044
:103E48003E60D2F89000184C206092F9DDE0D2F87C
:103E580094000023C2F8943080F311881EF0100FEC
:103E680003D00023E1EE103A03E002F19C0090EC4D
:103E7800108AEFF3148323F0040383F31488BFF349
:103E88006F8F02F1300090E8F01F8CF3098802F17F
:103E9800000004B542F0EBF9BDE8044070470000AB
:103EA8009C3B002004ED00E0C837002000231021CF
:103EB8000348C2180133722B82F80013F9D17047F6
:103EC80000E100E008B5EFF30583064A103B02EB7A
:103ED800C30152F8330049688847BDE80840FFF736
:103EE8006DBF00BFAC0C002001480068704700009F
:103EF800C83700201FB50121094B0A4A0A4800F0BB
:103F08000FF90023064A0393084B0121019301A8E6
:103F1800D31A029300F00EF905B05DF804FB00BF58
:103F280000000C20000000200C440708C0130020EB
:103F38000A7A0B6810B562F304031C46CB68520971
:103F480023F01F0343EA4203044A43F00103C2F883
:103F58009800C2F89C40C2F8A03010BD00ED00E007
:103F680010B50A4BD3F89030C3F30723013B9842AE
:103F780008D901210346064A064841F0DAFF6FF0E6
:103F8800150010BDFFF7D4FFFBE700BF00ED00E010
:103F9800F3110808343E07082DE9F04F8946144606
:103FA80006464FF000084F4D85B0C84527DAD6F8C9
:103FB80004A0BAF1000F44D0BAF11F0F17D91AF0B4
:103FC8001F0F14D1D6F800B01BF01F0F0FD15846A1
:103FD80042F068F907460AEB0B00013842F062F933
:103FE800874210D06FF015073F4A3B4601E0434631
:103FF8003E4A01213E4841F09CFF6FF015042046DF
:1040080005B0BDE8F08F17F1160FEDD0BC42EBDD1F
:10401800C5F89870D5F89C10C5F89870D5F8A030F8
:1040280021F01F0143F01F0BD6E900321A449942D0
:1040380002F1FF3A1AD1D34507D13146F8B242F01E
:104048003AF908F101080C36AFE73146C5F898701F
:10405800D5F89C30E0B263F30402C5F89C2042F026
:104068002AF910F1160FC8D0441CEAE7C5F8987071
:10407800D5F8A020013B23F01F0302F01F021343D1
:10408800D3453146E0B2C5F8A030E8D042F013F984
:1040980010F1160FB1D0C5F89870D5F89C209DF88E
:1040A80008300BF1FF3B62F304038DF80830D5F8B4
:1040B800A0309DF808205B0863F347128DF80820AC
:1040C800D6E900321344009323F01F035B44A3EBAB
:1040D8000A03013023F01F036946C0B20393FFF7B8
:1040E8003FFFBEE700ED00E03F120808191208087C
:1040F800343E07080522044BC3F89420BFF34F8FC2
:10410800BFF36F8F704700BF00ED00E0BFF35F8F14
:104118000022024BC3F89420704700BF00ED00E076
:1041280010B5034C2278FFF737FF207010BD00BF91
:10413800814900202DE9F74F294D8A4606464FF060
:104148000008AB46274FD0451BDAD6F80490B9F1E2
:10415800000F3FD031680846019142F0A3F8019959
:10416800044609EB0100013842F09CF884424FF004
:1041780014021D4B08D002FB08F36FF015024BF830
:10418800032003B0BDE8F08F14F1160F2C60F8D0AF
:104198001978A142F5DD02FB08B0C7F89840C7F8C6
:1041A8009840D7F89C4000F10801007B64F30400B4
:1041B8000871D7F8A0000C79400860F347140C7117
:1041C800D7F89C1021F01F016960D7F8A01021F0E2
:1041D8001F01296108F1010814350C36B3E700BF47
:1041E800CC37002000ED00E081490020F0B55349AC
:1041F800534DD1F890302C68C3F307239C4287B005
:1042080000F299800020FFF781FF4E4BC1F8C030C3
:10421800844216D14C4D01A82C70FFF75DF800269A
:1042280007464A4CB74213D100202B784349D1F8AE
:104238009020C2F30722934277DBFFF75BFF002051
:1042480046E0696801EB0011FFF772FE0130DFE715
:104258000199300101EB0613DA682240B2F1807F40
:1042680052D00AD8B2F5001F34D0B2F5800F3ED034
:10427800B2F5801F12D00136D4E7B2F1006F43D0F7
:10428800B2F1805FF7D15A689B680958013B22F068
:104298001F00034423F01F03012032E05A689B6883
:1042A8000958013B22F01F0003440120844623F0F3
:1042B8001F0340EA4C10CDE902218DF8100002A935
:1042C80028780593FFF74CFE00282ADA6FF01500CE
:1042D80007B0F0BD5A689B680958013B22F01F00DF
:1042E80003444FF0020C012023F01F03E1E75A6852
:1042F8009B680958013B22F01F000344022023F069
:104308001F034FF0000CD4E75A689B680958013B1B
:1043180022F01F0003444FF0030C012023F01F0379
:10432800C7E72B7801332B70A5E7C1F89830C1F89F
:10433800A00001337BE74FF0FF30C9E700ED00E054
:1043480018440708AAFF4400814900200000F0FF34
:10435800F0B587B007460E4614460021102268467D
:104368001D465EF0D3FF02238DF80230054B2A4626
:1043780021466846CDE9047601933CF037FF07B043
:10438800F0BD00BFF762050808B5024B1B689847E7
:10439800002008BDE0370020034B044A18609378DA
:1043A80043F0020393707047E03700209C0100201F
:1043B80008B5054841F065F9002383F31188BFF378
:1043C8006F8F0423184602DF7112080808B50649E2
:1043D800064821F00701C1F1005202F5402240F0E1
:1043E80006FF002008BD00BF13EA0020E4370020C4
:1043F8004FF0FF324FF0FF33014807F083BB00BF97
:10440800AC010020014807F0EFBB00BFAC01002061
:1044180038B50546FFF7ECFF2A460821074840F063
:104428002CFE044628B925B1FFF75EFD0C22044B8B
:104438001A50FFF7E7FF204638BD00BFE4370020D9
:104448000C00000038B504460D46FFF7D1FF2146A1
:104458002B460822074840F092FE044628B925B1A9
:10446800FFF742FD0C22044B1A50FFF7CBFF204602
:1044780038BD00BFE43700200C00000010B504462A
:10448800FFF7B6FF21460348FDF78CFEBDE8104054
:10449800FFF7B8BFE437002070B541690446867A53
:1044A8000A4D59B1437ADB0706D42C2303FB065384
:1044B8005B6A1B689B689847002363612C20214630
:1044C80000FB0650BDE8704045F00DBCA811002067
:1044D8002C22024B02FB0030704700BFA8110020BD
:1044E8002C21827A054B01FB02339A6A1B7F801AC2
:1044F8001B3323F00303B0FBF3F07047A81100202F
:1045080038B52C24827A064B04FB02335B6AD3E964
:1045180001240C601568FFF7E3FF04FB005038BD69
:10452800A81100202DE9F04385B00546684690465D
:104538001C46039145F00DFEDDE90067EFF3118994
:10454800102383F31288BFF36F8F6B8B002B41D03E
:104558002A8B9A4225D900220023284607F094FB8B
:104568000446F0B189F31188BFF36F8F039B002BCA
:1045780041D032463B46684645F010FE2C21A27ACF
:10458800254B204601FB02335B6A03A91B681D68A3
:10459800DDE90023A847606170BB2046FFF77CFF78
:1045A80024E0698B4B1E6B8389F31188BFF36F8FEF
:1045B8002B7F2A8BAC6A1B3323F00303521A02FBAE
:1045C8000344154B154AEB1A9B105343A3722B7FD8
:1045D800E372CBE789F31188BFF36F8F2346424616
:1045E800284607F051FB04460028BFD10024204686
:1045F80005B0BDE8F0836361012300252381039B97
:1046080029466382E27A656004F118005EF07EFE56
:1046180063692582E360EAE7A8110020A38B2EBA1C
:10462800F8B500242C260F4D00B9F8BD476800F1F5
:104638000802D2E8EF3F591EC2E8EC1FBCF1000F98
:10464800F7D1DBB2012BF0D1837AC46006FB0353A8
:1046580044601B6A13B198473846E5E7FFF71CFF2B
:10466800FAE700BFA8110020F7B506460D46144624
:10467800124F384645F05AF9E0B1BB683146384622
:104688001B68AAB29847002802DB002003B0F0BDDF
:10469800002CFBD1AC42F8D22F1B042F28BF0427D3
:1046A80005F0BCFF3A46019001A930195EF008FEFA
:1046B8003C44EFE76FF01200E8E700BF103B070843
:1046C80038B5044608F0C8F8204641F08CFEA069C9
:1046D800C8B194F86C30DB070DD50221154A16488D
:1046E80041F07FFE6FF07705201D41F083FE08F052
:1046F800C7F8284638BD45F019F938B901210F4ADD
:104708000D4841F06EFE6FF01205EDE7204600F00F
:10471800ADFF05460028E7D10146242204F1280010
:104728005EF0F4FD94F86C3043F0010384F86C30CB
:10473800DAE700BF89120808E43E0708B312080840
:1047480070B5044608F088F8204641F04CFE94F80D
:104758006C30DA070DD40221254A264841F041FE83
:104768004FF0FF35201D41F045FE08F089F8284636
:1047780070BDC3F340019B0707D502211E4A1D489F
:1047880041F02FFE6FF07705ECE7A06943F0AAFA35
:104798000646A06943F036FB054628B10121174AB1
:1047A800144841F01EFEDDE7A36F4BB131462046A9
:1047B80041F0FAFF0546A0B1A06943F04BFBD1E7F1
:1047C800A06943F0C7FAA0670028EFD101210C4A7D
:1047D800084841F006FEA06943F03CFB6FF00B056A
:1047E800C0E794F86C3043F0020384F86C30B9E702
:1047F800D6120808E43E0708FC1208082213080825
:104808003E13080838B590F86C3004469B0708D466
:104818000221144A144841F0E4FD6FF07705284658
:1048280038BD41F0E0FD0021204601F0B9F820B183
:1048380001210E4A0C4841F0D4FDA06943F00AFB5F
:10484800054620B101210A4A074841F0CAFD94F8FB
:104858006C30201D23F0020384F86C3041F0CAFD4F
:10486800DDE700BF5A130808E43E0708811308086B
:104878009F1308082DE9F04385B006460C4690467C
:1048880041F0BAFD0546B8F1000F07D0304641F0B7
:10489800B8FD012810D1B5FA85F56D09013429460E
:1048A8003046E2B241F099FF814650B901212346D2
:1048B800324A334841F03DFB0024204605B0BDE8AC
:1048C800F0834768B8F1000F09D03868796801AB00
:1048D80003C33A7A01AF1A7007238DF80530F18DBA
:1048E8007B883046994228BF194642F0C8F80446EA
:1048F8000028E1D0038A428A4169D21AC36800F1CC
:104908000C085B1AD21A3B7839469A4228BF1A46D5
:10491800404641F03BFDD9F80C90B9F1000F08D1A1
:10492800218AF38D9942C8D94046C91A41F049FDF8
:10493800C3E7D9F8040083681B6B13B9D9F8009052
:10494800EBE7294698470028F8D0071F57F8041FB7
:104958000029F3D008780028F0D0628A238AA2EBD5
:10496800030C6269E3689B1AACEB0302904294BFA4
:10497800024692B2404641F009FDE7E7CF13080826
:10498800C43E070838B50446806F41F0E0FC054690
:1049980041F0C1FC2046294601F04AFA044638B1E4
:1049A80004480121044A41F0BBFA2846FFF738FEC3
:1049B800204638BDC43E0708F513080838B58021DD
:1049C8000446806943F0E9F9054678B10146204676
:1049D80001F02EFA044638B106480121064A41F092
:1049E8009FFA2846FFF71CFE204638BD6FF00B04DF
:1049F800FAE700BFC43E07081414080800232DE98D
:104A0800F04F93B005930B7E044633F080060F46B3
:104A180015460AD00121AD4AAD4841F081FA6FF040
:104A28000406304613B0BDE8F08F82B10846FFF7A0
:104A3800F7FD7B7EDA0704D49D07F2D53B7E002B79
:104A4800EFD1204613B0BDE8F04FFFF79BBF4A7E79
:104A580000F12809900705D5802B09D13846FFF7C2
:104A6800DFFDDEE7910700F03184002B40F02E8453
:104A7800D3071ED53B8A082B12D1FA68394613682A
:104A88000020A3625368C9F8043041F067FC059020
:104A980080B18F4801218F4A41F042FA059805E01C
:104AA8008B4801218C4A41F03BFA3846FFF7B8FDA4
:104AB8001EE00597FFF718FA002394F82850874A54
:104AC80015F0600F8350C5F341131CD0032B40F041
:104AD80064836FF08505FFF707FA804B1B58002B9E
:104AE80000F09A83002D00F0698305980028DDD135
:104AF800484641F0B9FD0346A069002B00F0218427
:104B0800802100F027BC484641F0AEFD94F82930DA
:104B1800002840F02C81013B0A2BDAD801A252F878
:104B280023F000BF6B4C0108DB4A0108F14C010877
:104B3800DB4A0108594B0108DB4A0108DB4A010836
:104B4800DB4A0108BF4B0108DB4A0108334C010866
:104B5800A069618D03697F2993F88030B9D8A28D47
:104B6800002AB6D1E28D002AB3D1EE06B1D194F86D
:104B78003020022A02D14FF0FF35ACE71D070BD5D4
:104B8800C9B241F0A7FD054648B1638D0121544AD9
:104B98004F4841F0CEF99EE7012384F8393094F864
:104BA8003030012B05D1638D1BB984F830300025D6
:104BB80091E70123F9E7204641F01EFC628D01468A
:104BC800FF2A86D8E38D002B83D194F82830D806A5
:104BD8007FF47FAF94F83030002BCCD092B9618D40
:104BE80094F838308B42E2D02046C9B200F0D8FEA3
:104BF800638D054668B1012100903A4A344841F076
:104C0800A2F968E72046D2B241F00DFE0028E6D1AD
:104C1800B1E7002B14BF02220122052184F83020BD
:104C280020461A4641F074FFC1E705F01F05012D23
:104C38007FF44FAFE38D002B7FF44BAF628DFF2ADB
:104C48003FF647AFA18DFF293FF643AF94F83030C8
:104C5800022B90D12046D2B2C9B241F094FE05464B
:104C680039E7E38DA68D002B7FF433AF94F830300D
:104C7800002B80D0012B02D1002E7FF47CAF15F0E1
:104C88001F0515D0022D92D1B4F82A80B8F1000F73
:104C98008DD1F6B23146204601F032F9421C054664
:104CA8003FF419AF42463146204641F0E3FC12E793
:104CB800002E7FF460AF638D012B7FF478AF94F8FA
:104CC8006C3066F3C30384F86C3070E73714080857
:104CD800C43E07086F140808581408080C000000A0
:104CE80091140808B3140808A38DE28DDEB2002AD7
:104CF8007FF4EFAE628D022A11D105F01F0535430E
:104D08004FEA13217FF4E5AE0122A06941F0C2FC0D
:104D180000287FF4DEAE012384F8393047E794F8A1
:104D2800301000293FF427AF012902D1002B7FF46E
:104D380022AF15F01F050FD0022D7FF438AF002ADF
:104D48007FF435AF3146204601F0B8F8431C0546DC
:104D58003FF4C1AE0122A6E7002B7FF40CAF012A75
:104D68007FF425AF94F86C3043F00803ABE70A2BC7
:104D780063D8DFE813F00B00620062006200620093
:104D880062003A006200DD016200F201E38D022B4D
:104D980053D194F83030002B4FD0012BA18D01D185
:104DA80000294AD115F01F050ED0022D17D0002674
:104DB8000221204641F063FE054618B131460C3009
:104DC80041F0F5FA0595F2E6002936D194F86C30F1
:104DD8009E0806F00206C3F300131E43E8E72046C8
:104DE800C9B241F070FE0646E2E7618DED064FEA72
:104DF8001123C9B207D0002320460AA90A9341F01B
:104E080082FC0A9DDEE7013B0E2B16D8DFE813F083
:104E18000F003000380015001500D20036001500CC
:104E28001500150015001500150015000F01204686
:104E380041F0E2FA18B1012818D00025C2E7266F20
:104E4800002EFAD0B4F82E8033782046984528BF33
:104E58009846414641F013FE05460028B2D0424626
:104E6800314605F10C0041F091FAABE7666FE7E7D0
:104E780000222046FFF7FEFC0546A3E70122F8E7DB
:104E88000A462046032141F043FB80460028D4D03F
:104E980041F0E5FBE58D98F81530B8B998F814603D
:104EA8008DF82930AE428DF8286028BF2E46D8F8F4
:104EB800103031461B882046ADF82A3041F0DFFD1E
:104EC80005460028B9D032460AA9CAE74FF0000AB9
:104ED800B44A8DF81130D8F808308DF810A01A406F
:104EE800B14B9A4255D1102106A804F09DF8061E30
:104EF80036DB0AAB102E984628BF1026AB4806AA08
:104F0800564503F1020334D8B6000236F6B28DF8DE
:104F18001060AE4228BF2E462046314641F0AFFD14
:104F28000546002889D0022EB34628BF4FF0020B51
:104F38005A46A6EB0B06C34600F10C0A504604A9D4
:104F480041F024FA730808EB56025A4528D1F007B5
:104F58007FF538AF504618F8031041F020FA31E7D2
:104F680058367FF46AAF0121914A924840F0D8FF41
:104F780063E712F8011B0AF1010A4FEA111C01F05C
:104F88000F0110F80CC0415C03F802CC03F8011CB7
:104F9800B6E798F81460D8F810808DF81060B8E774
:104FA80050461BF8011BCDE9022341F000FADDE968
:104FB8000223CAE7204641F01FFAD4E91C5300280F
:104FC80008BF1D460A2300268DF8283006232046F0
:104FD800CDF82A60CDF82E608DF8293041F011FA0D
:104FE80001287FF42AAF002D3FF4ECAE6B882046F1
:104FF800ADF82A302B798DF82C306B798DF82D305F
:10500800AB798DF82E30EB798DF82F306B7C8DF8DD
:105018003030E68D9DF828309E4228BF1E46314626
:1050280041F02DFD054600287FF44DAFCAE6204625
:1050380041F0E2F920B101287FF4FFAE636F00E090
:10504800236F002B3FF4F9AE5B88B3F5007F7FF642
:10505800F4AE594B04F14C060A9300238DF82C301A
:10506800E36C9E4208BF0023BDF82A2093B1597D06
:105078000F2908D1197D0A44ADF82A209DF82C2063
:1050880001328DF82C20226D9A4201D01B68EBE783
:10509800BDF82A20B4F82E802046904528BF9046B7
:1050A800414641F0ECFC054600283FF4C6AE9DF8A9
:1050B800282000F10C0A424528BF424650460AA95A
:1050C80041F064F99DF82830434594BFA8EB0308E4
:1050D800A8EB0808B8F1000F3FF474AED4F84CB050
:1050E800B3453FF46FAEBBF1000F3FF46BAE9BF8D6
:1050F80015300F2B15D19BF814205046424528BF78
:105108004246DBF8101041F041F99BF81430434552
:1051180094BFA8EB0308A8EB0808B8F1000F3FF408
:1051280051AE236D5B453FF44DAEDBF800B0DAE7D6
:1051380094F83030002B3FF480AEE18D01297FF4E4
:105148007CAE94F83860204641F099FC054600286A
:105158003FF438AE31460C30FFE605F01F05012D4F
:105168007FF46BAE204641F04CFB00283FF465AE5F
:10517800A38D4268FF2B3FF660AE12799A42FFF486
:105188005CAEDAB20F2A3FF658AEE18D01297FF402
:1051980054AE234493F83A60D5E7204605A941F078
:1051A800B2FA5CE500FF020000030200316A080859
:1051B800D6140808C43E0708050F050044F0C7FFC9
:1051C8000A220023FBF748FE644BD3E8AF1F41F2E5
:1051D8008732461A9642624A39D9D3E8EF6F8E422F
:1051E80004D1C3E8EC0FBCF1000FF6D12FD1D2E8FF
:1051F800EF3FC2E8E15F0029F9D123B10221594A02
:10520800594840F096FE0221584A574840F088FE17
:10521800FEF76AFE564B1D58002D7FF466AC7B7E68
:10522800E28DD9071BD5484641F01EFAB8B9BAB184
:105238002946A06942F09DFD0146059000283FF4EB
:1052480057AC204613B0BDE8F04F00F0F1BDD2E8EE
:10525800EF3F0133C2E8E13F0029D9D0F7E73AB977
:105268002046FFF7ABFB00287FF442ACFFF7E9BB11
:10527800484641F0F9F9059D18B92846FFF7D0F9D5
:10528800EEE7002D3FF434AC2946204600F0D0FD6F
:1052980008B128460AE4A069036993F8801011F060
:1052A80004017FF4CEAB42F078FD054600283FF4B8
:1052B8001FAC0146204600F0BBFD00283FF4C1ABFF
:1052C80001212C4A284840F02BFEE2E752077FF5DF
:1052D8000FAC002B3FF4C2AB3846FFF7A1F994F8A6
:1052E8003930002B3FF49DAB94F82930052B0CD1B5
:1052F800618DA069C9B241F0EDF9054628B1638D09
:1053080001211D4A184840F014FE94F82930032B57
:1053180011D1638D022B0ED1A18D00220E0A3146C8
:10532800A06941F0B7F9054628B101213346134A6F
:105338000D4840F0FEFD00232E4684F83930FFF773
:1053480070BBE38D002B3FF4DBAB0599003918BF28
:105358000121C90142F024FCFFF773BBF437002098
:10536800F0370020F8140808C43E07080C15080890
:105378000C0000003515080891140808591508088C
:105388000B7810B4062B14D10369D3F89C20EFF3E3
:105398001184102383F31288BFF36F8F00204B68AA
:1053A8001860506A60B9C2E9083384F31188BFF302
:1053B8006F8F0022002304485DF8044B44F0B5BB0E
:1053C80003605362F1E700BF2411002030B589B0B3
:1053D800002200230024CDE906236FF007034FF4D1
:1053E8008062CDE90334CDE90144154B1549009499
:1053F800154806F035FF1549134844F04EFD144B87
:1054080014498B4207D30020134B14498B420CD309
:10541800002009B030BD03F11402D2E8EF0FC2E852
:10542800E54F002DF9D11833EBE703F11402D2E868
:10543800EF4FC2E8E50F002DF9D11833E6E700BFBA
:10544800C154010800550020A0280020A22F0808F8
:10545800001300206013002060130020C0130020F8
:1054680038B50D4641F0CDF930B90121BDE83840D5
:105478000F4A104840F054BDC46804B938BD2B78B1
:10548800032B05D0052B0ED0022B08D02468F4E797
:10549800606883685B69002BF8D09847F6E7606816
:1054A80083689B69F7E760688368DB69F3E700BF97
:1054B80080150808D43E07082DE9FF4110274FF052
:1054C800FF334FF0FF32644801A906F0B7FA039B97
:1054D8001B69D3F89C40236A93B1EFF3118287F3D9
:1054E8001288BFF36F8F216A29B1606A0B68814205
:1054F800236208BF636282F31188BFF36F8FC9B953
:105508009DF80430062BDAD0072BD8D801A252F820
:1055180023F000BF61550108555501088955010858
:1055280067550108BD550108AB550108C754010866
:10553800515601080B7E20465D06D1F81E2002D187
:10554800FFF75CFAC7E741F0ACF9C4E70022012194
:10555800204641F0DDFAB2E700221146F8E794F858
:105568006C3043F0040384F86C3094F83030022B2C
:1055780003D1204601A9FFF773FF00220321E7E7C3
:1055880094F86C3023F0040384F86C3094F83030CD
:10559800022B03D1204601A9FFF762FF0022022156
:1055A800D6E794F83030022B89D1204601A9FFF7BD
:1055B80057FF84E794F86C30A66923F0040384F855
:1055C8006C30D6F808803369A033D3E8AF3F9A0728
:1055D8001ED53046D8F83C309847D8F824300021FA
:1055E800304698470546D8F840303046984795B138
:1055F8001A4A01211A4840F093FC0022042120464F
:1056080041F086FA002D3FF45AAF2A4607219FE75A
:105618004FF0FF35ECE72946204600F0C1F9054672
:1056280008B1104AE5E7A06942F0D6FB831E58424C
:10563800584194F86C3084F8305023F0680343EAFA
:10564800401384F86C30D8E70121074A044840F039
:1056580067FC0621029A7BE724110020AF15080891
:10566800D43E0708DD1508080916080838B50246AB
:1056780005460C49806942F00DFC044630B1012111
:10568800094A0A4840F04CFC204638BD85F83800E5
:10569800284600F043F904460028F5D0A86942F0EE
:1056A80028FCF1E78953010819160808D43E0708B1
:1056B800F8B501231D460C68002C35D063F07F0235
:1056C800D6B202F07F02103224FA02F7FF0716D58D
:1056D800046824FA02F7FF0708D433461348012167
:1056E800134A40F026FC6FF01500F8BD05FA02F2E7
:1056F80024EA020404600C6824EA02040C60DC401A
:10570800E6070ED5026822FA03F4E40700D4E5E7B9
:1057180005FA03F422EA040202600A6822EA040293
:105728000A600133102BC6D10020DEE7043F0708CA
:10573800401608082DE9F04F0026536891B0D46848
:105748000A900891069202930E96039674B9039BE9
:10575800029A09339BB293701B0AD370069B167189
:10576800DC68002C40F0C780A346AEE04FF0000A8A
:105778006068CDF83CA083681B6B002B00F0AC8000
:1057880008999847002800F0A7803546C4E903AA7D
:10579800A0F1040959F8043F0BB11A789AB9B54237
:1057A80040F29780E3680F9A1343E3606068836868
:1057B8009B6A002B00F0928098478346002800F0EF
:1057C8009080534A7DE05A780B2A08BF9D70D9F81B
:1057D80000305A78042A10D1E2680F990A43E2602F
:1057E800DA78002A5CD101229D702369AA4013430C
:1057F80001352361EDB2CDF83CA0D9F800707B7873
:10580800052BC7D16FF0120B4FF001080A9B9B695B
:10581800099379793A790E9B42EA0122ADF836204C
:1058280097F902205FFA88F1002AACBF424641F09E
:1058380080010493B7BF4BB24FFA88F321F080027E
:105848000793A8BF0793049BB8BF103223FA02F04E
:10585800C0072CD40F9B23FA02F20593D30726D452
:10586800BB79FA78099800930DF136030B9142F051
:105878000DF90B998346D0B9079BB970002B4FF0EF
:105888000103BCBF21F0800110318B4004980599B9
:10589800BDF8362019431843CDE90E01BA8079E7DF
:1058A8006A1E9A700FA90EA8FFF702FFA3E708F176
:1058B8000108B8F1100FACD1BBF1000F3FF46AAF8B
:1058C800144A0121144840F02BFB584611B0BDE89A
:1058D800F08F6FF0150BF3E7354667E76FF0850B30
:1058E8006FE76068089940F0ACFF039B2E460344BD
:1058F800246803932AE7E36804F10C01A3600EA867
:10590800FFF7D6FE08B924682BE76FF0150BDCE724
:10591800811608085D160808043F070870B58369F2
:1059280005461B69026F93F88030C3F34113022BBD
:105938000CD0032B0CD0012B0CBF10230823D371E0
:10594800EE6D3EB96E6DBEB9344611E02023F6E720
:105958004023F4E7324601212846FFF7EBFE0446D0
:1059680040B173685B790B4A01210B4840F0E1FABA
:10597800204670BD3668E4E7324600212846FFF726
:10598800D9FE044618B173685B79044AECE73668B7
:10599800D9E700BFA5160808043F0708C816080875
:1059A8002DE9F04105460E4640F026FD95F83830C1
:1059B800804633B3284640F024FF0746F0B101463D
:1059C800284640F08EFF10220446002105F13A00D7
:1059D8005DF09CFC002385F83830FF683FB984B13E
:1059E80019491A4840F0ECFE2046BDE8F081786875
:1059F80083685B6A03B198473F68EFE76FF03C0440
:105A0800EEE71EB985F838600024EDE732464146D6
:105A1800284640F0E2FE074690B10246284640F08C
:105A28008AFF04460028DFD185F83860FC68002C1E
:105A3800EAD0606883681B6A03B198472468F6E770
:105A48006FF03C04D0E700BF81130808BC3E07088C
:105A58002DE9F04105460F461446D2F8048040F07F
:105A6800B3FE95F86C30D9070BD54749474840F045
:105A7800A7FE6FF00F07281D40F0ADFE3846BDE8C1
:105A8800F081012F0AD1284640F0BBFC30B94049CB
:105A98003E4840F095FE6FF08507ECE798F8073030
:105AA8009A0607D5AB691B6993F880309B0701D428
:105AB8003849EDE71FB1012F06D03749E8E7EB6D0C
:105AC8002BBB05F1540603E06B6DABB905F15C0621
:105AD800002233680BBB002FD5E91C2308BF1346EF
:105AE8005B7C626803F10103DBB25371D5E91C12D8
:105AF80008BF0A46537422E09C4206D1274923482E
:105B080040F05EFE6FF01507B5E71B68DDE79C42C5
:105B180001D12349F3E71B68D2E79C4221D12368CE
:105B2800CAB972683360944200D17360002323605D
:105B380063685B7902211B4A144840F0FAF9A168AE
:105B4800B9B1284640F0FEFC074668B116490F482F
:105B580040F036FE8FE7136073689C4208BF72609E
:105B6800E4E71A461B68B5E7A06840F078FD88F8B6
:105B780006000023236073681BB9C6E900440027A8
:105B880079E71C607460FAE719170808BC3E070833
:105B98003B170808F5160808591708087917080860
:105BA80096170808B3170808D0170808F8B5054667
:105BB80000AF29B301290BD1184C194E2BE06368AB
:105BC80028461968FBF7A2F9B8B11834B442F6D3DD
:105BD8006C4688B06A46134BCDE905354FF400731F
:105BE800ADF81C30104B42F8103F00234FF4E2513F
:105BF8000E48FDF7D9F8A54600242046BD46F8BD55
:105C08000B4C0C4EE2E7636828461968FBF77EF9EF
:105C18000028F2D01834B442F5D3D9E76013002035
:105C2800C01300200718080803000001CC3E07082D
:105C3800001300206013002070B5012501F07F03D8
:105C480011F0800F18BF10339D4090F83030044693
:105C5800022B06D001210C4A0C4840F061F90020C3
:105C680070BD90F8386040F0C7FB324601462046C8
:105C780040F0B3FD0028F2D0C0680028EFD0836858
:105C88001D42EDD10068F8E725180808CC3E070842
:105C98002DE9F84305460846114616469846FFF78B
:105CA80085FF0446002843D0284640F0C3FD95F8F8
:105CB8006C30DA0702D5204A012109E0D4F80490B3
:105CC80004F11407D7E8AF3FDB070CD502211B4AC4
:105CD8001B4840F025F96FF00F04281D05F084FFDC
:105CE8002046BDE8F883D9F804301BB1AB4201D097
:105CF800144AE1E742463146284640F06EFDA0B11D
:105D08000023236003696BB9C0E90344D7E8EF3F78
:105D180043F00103C7E8E23F002AF7D10024C9F89D
:105D28000450DAE71C600461F0E76FF03C04D4E744
:105D38006FF01204D4E700BF191708084A180808BA
:105D4800CC3E07086C1808082DE9F04F83B000AF67
:105D58007B6097F830304C680E463B608146904631
:105D680040F04AFBA36801461B6B33B96FF015047A
:105D780020460C37BD46BDE8F08F204698470028DE
:105D8800F4D00024051F06F10C0A55F8041F09B1C8
:105D98000B782BB9002C14BF00246FF03C04E7E704
:105DA8004B78042B0ED1002C3CD18B787A68934227
:105DB800EBD1CB783A689342E7D10B79002BD7D057
:105DC8000124E2E7052BE0D1002CDED0B8F1010F69
:105DD80091F802B009D0B8F1020FF1D152465946F4
:105DE800D9F8180040F035FE04E05246D9F81800FA
:105DF80040F013FE04460028E2D06D468AB06A4699
:105E0800F368CDE907B3062307490990CDE90518DA
:105E180042F8103F00234FF441510448FCF7C4FFF7
:105E2800AD46A5E70024A3E7AC180808FC3E070820
:105E38002DE9F0410B7E0C465906054637D16BB368
:105E480040F01AFB40B11B4801211B4A40F068F89A
:105E58004FF0FF30BDE8F0812846D5F87080268ADB
:105E6800EF8D40F0C9FAF8B1421E534253419B01ED
:105E7800228A9AB1BE42324628BF3A46E98D9142FB
:105E88000CD9B2FBF3F103FB11223AB994F918309B
:105E9800002BBEBF637E43F0080363762146A869E2
:105EA800BDE8F04141F0D8BE98F80730E0E76FF060
:105EB8001500CFE7EC3E0708E818080870B5064655
:105EC80080690C4641F06CFE054638B10221234634
:105ED800094A0A4840F02DF8284670BD012214F0FE
:105EE800800F18BF24F08004736B18BF1034A240D1
:105EF8001A437263F0E700BFFC180808EC3E070875
:105F080070B5054680690E4641F075FE044638B105
:105F180002213346054A064840F00BF8204670BD7A
:105F2800314605F1340040F06AFDF7E71319080817
:105F3800EC3E070870B50646EFF31181102383F392
:105F48001288BFF36F8F1B4D2A6881F31188BFF346
:105F58006F8F526892F86C20D20705D4BDE8704064
:105F68000A22002306F02EB9EFF3118283F3128878
:105F7800BFF36F8F2C682CB1696823688C422B6043
:105F880008BF6B6082F31188BFF36F8F44B16068FC
:105F980004F10801C36998472146074843F062FDA8
:105FA8002B6833B13046BDE870400022002306F06C
:105FB800D1B870BDF8370020B010002030B585B0DA
:105FC800CDE90012054600220023144803A905F074
:105FD8009BFC0246E8B9DDE90001039B5D600833DC
:105FE80083E80300EFF31180102383F31288BFF3D3
:105FF8006F8F039B1A600A4A516861B9C2E900337E
:1060080080F31188BFF36F8F00220023054806F044
:10601800A1F805B030BD0B605360F1E7B010002067
:10602800F83700200000002073B5102504698DF8AA
:106038000710EFF3118685F31288BFF36F8F0122E3
:10604800206C0DF107013FF0E4FD86F31188BFF3E2
:106058006F8F012812D043F01AFFC8B10122104BEC
:10606800D3E8EF1F002903D1C3E8E02F0028F7D1B8
:1060780004D102210B4A0C483FF052FF237F2BB179
:106088000A22002304F1480006F064F802B070BD4B
:10609800A37E002BE2D000210A2044F000F8C8E7D4
:1060A800003800203D190808B43E070838B5002418
:1060B80005690E492B6C05F14800C3E90144DC6011
:1060C800AB6BC3E90144DC6043F0D5FE05F1780011
:1060D800074943F0A4FE074905F1280043F09FFE55
:1060E800284640F03AFD204638BD00BF216201082D
:1060F80069630108356401082DE9F341036906461F
:106108000D46D0F804801C690F7E002A32D00B8A15
:1061180071323E480BBF022101213D4A3D4A00939E
:106128003B463FF010FF30462F7E40F08AFD874205
:1061380004D1042104F1880040F037FE30462F7E58
:1061480040F08DFD874204D1052104F1880040F01C
:106158002CFE30462F7E40F066FD874203D104F1C5
:106168008C0005F029FE2946404602B0BDE8F04102
:1061780040F0A6BC40F065FDB84214D12A8AE9680F
:10618800A06B3FF046FD28B1236A1BB104F128003B
:1061980005F070FF04F18800042140F006FE04F1C8
:1061A800780005F067FF30462F7E40F058FD8742A3
:1061B80015D1236A1BB104F1280005F05BFF052106
:1061C80004F1880040F0F1FD237F9BB900234FF4D0
:1061D8007A7204F1480005F0BDFF012323773046A9
:1061E8002F7E40F020FD8742BDD104F18C0005F0E0
:1061F80081FDB8E7236C5A89DB889A42EFD00022E8
:10620800002304F1480005F0A5FFE8E7B43E0708BD
:106218005C190808801908082DE9F04750F8483C2F
:1062280000F140075B68054600213846D3F8009026
:1062380040F0F3FC002864D00121384640F0EDFC22
:10624800804600285DD155F8083C5A89DB889A4277
:1062580003D115F82D3C002B53D0D7E8EF4F44F06D
:106268002003C7E8E23F002AF7D114F0200448D100
:10627800484640F0F4FC002282460023224840F0C1
:106288004FF8064650B93846052140F08EFD28469D
:10629800BDE8F0470A22002305F05CBF80F818A08B
:1062A80015F82C3C33B1428AC16855F8080C3FF008
:1062B800D0FC0446214606F10C0040F061F85CB1C0
:1062C800D9F8040040F04FFDB4FBF0F303FB104491
:1062D800B4FA84F84FEA58183146484605F82D8C28
:1062E80040F0D6FB68B10121084A09483FF018FE82
:1062F8003046FEF795F93846BDE8F047052140F0ED
:1063080054BDBDE8F08700BFA8110020A1190808F6
:10631800B43E070838B503461B6940685D68AC6839
:10632800A37A84F8223094F82D3084F82330A376A9
:10633800696849B1237C3BB940F004F930B10121C7
:10634800054A06483FF0ECFD002038BD686840F07B
:1063580086F92074F8E700BFB3190808B43E0708A7
:1063680070B550F8782C00F11004526803460021EB
:106378002046156840F051FC00284DD001212046E8
:1063880040F04BFC002847D153F8402C68689388AC
:10639800918916695B1A9BB2F61A40F0E4FCB04288
:1063A8003AD8D4E8EF3F43F01002C4E8E12F0029BF
:1063B800F7D1DB0606D5BDE870400221174A184818
:1063C8003FF0AEBD284640F03CFC002206460023C4
:1063D80014483FF0A5FF0446F0B10676686840F01F
:1063E800C2FC638A984203D2686840F0BCFC83B25E
:1063F80021462846638240F04BFB68B1284640F0AE
:1064080020FC034606480121074A3FF092FD20463A
:10641800BDE87040FEF704B970BD00BFDD1908087B
:10642800B43E0708A8110020FD19080838B550F82F
:10643800083C044633B9BDE8384001212A4A2B48B4
:106448003FF06EBD50F8283C00F160055B68022102
:106458001A68002383828383284640F0DEFBB8B1A4
:1064680054E9023110699847637D1BB104F150006B
:1064780005F000FE0521284640F0CFFB98B9637F60
:106488006BB10022002304F1200005F063FE0AE04E
:106498000321284640F0C1FB0028E1D1E4E714F8C5
:1064A8000D3C002BEDD10221284640F0B6FB38B157
:1064B8002369DA885B899A4202D0204605F0DAFD22
:1064C8000321284640F0A9FB60B1A269938891890D
:1064D80012695B1A9BB29A4204D02046BDE8384044
:1064E80005F0C8BD38BD00BF221A0808B43E070829
:1064F800D3B5002600270446CDE9006705483FF0DC
:1065080013FF28B1230658BF0023047658BF03821F
:1065180002B0D0BD2C1200202DE9F04383B0002337
:106528004FF0010805691C4C1C4E02AF28602B7700
:1065380085F8203005F12409B442234601D3002010
:1065480019E095F820201034CAB16C4688B01B6851
:1065580002AA1349C2E905134FF400739383114B40
:1065680042F8103F104800234FF4E251FCF71CFC9E
:106578006FF00B00A5460437BD46BDE8F08385F8EB
:10658800208054F8043C4846009354F8101C54E901
:10659800032340F0D6FECFE7F0B0080800B10808A2
:1065A800841A0808030000010C3F07081FB5CDE94D
:1065B800010103924FF0FF324FF0FF3301A9034866
:1065C80043F0B3FA002005B05DF804FBF410002096
:1065D8001FB500230190CDE902334FF0FF324FF091
:1065E800FF3301A9024843F0A0FA05B05DF804FBA7
:1065F800F41000202DE9F041044617460E460068C5
:1066080040F007FD31463A468046FFF771FFD4F85F
:106618007B300546DB1B0146C4F87B30206840F020
:1066280037FA88B10B4A434601210B483FF081FCF9
:106638003146204640F0B8FD2846FDF7F1FF2046D8
:10664800BDE8F04140F07CBDA37F0133A377BDE8EE
:10665800F08100BFFD1908080C3F07082DE9F84F25
:106668000446006840F0EAFC4FF030090746E37F33
:10667800012B1ED82368D3F810B0D3F804A09BF8D8
:10668800616009FB06B62436304640F080FE31468C
:1066980002468046504640F0E7FC9BF81F3005460E
:1066A80033B1A8EB00023146504640F0DDFC054608
:1066B8000DB9BDE8F88F204640F093FC2A46014604
:1066C80006463846FFF714FF05460146206840F0A5
:1066D800DFF980B101213B46094A0A483FF029FC0D
:1066E8002846FDF79DFF3146204640F05DFDBDE898
:1066F800F84F40F025BDE37F0133E377B7E700BFEC
:10670800FD1908080C3F07082DE9F04FB94F89B06B
:106718004FF0FF324FF0FF33B74805A905F08EF967
:10672800059E069D3469002D40F09080257704F180
:10673800240694F820309D42C0F2828004F11803A8
:10674800D3E8EF2F22F00202C3E8E12F0029F7D1A6
:10675800D3E8EF1F21F00401C3E8E21F002AF7D1B4
:1067680004F11803D3E8AF3FDB07D1D5237F022B11
:1067780000F08E81032B00F0878153BBDDF814A055
:10678800DAF81050EB7F23BB504640F057FC8146A7
:10679800284640F026FC4FF400720146064648465B
:1067A800FFF7A6FE80460146504640F071F90028E2
:1067B80000F0668101214B46904A91483FF0B9FBB1
:1067C8004046FDF72DFF3146284640F0EDFC40F0ED
:1067D800B7FCA37F002B9BD1237F012B40F07D8149
:1067E800302304F1630694F86150304694F862103F
:1067F80003FB054500F060FA24350246314623695B
:10680800284600F077FA0646C4F88400284640F087
:10681800B4FD8146284640F0B5FD8046284640F044
:10682800B6FDE26D3044002A40F03B81002840F07C
:106838003381284640F0D2FD003818BF01202CE1F2
:10684800304640F091FD0135303672E7DDF81C80A6
:10685800D6F804A095F81890B8F1000F21D02B8A2B
:1068680018F1710F6648009308BF02214B4616BF06
:106878000121644A644A3FF066FB304695F8188067
:1068880040F0DCFB804540F0EF80E37F013BE3779D
:106898002046696940F088FC2946504640F010F9C6
:1068A8005EE7304640F0CAFB484540F09580237FBC
:1068B800D5F80C80B5F810B0002B49D1BBF11F0FEB
:1068C80042D1D8F80030BB423ED1414604F15403CE
:1068D80008F11C0251F8040B914243F8040BF9D15A
:1068E8000A881A808A7842219A70552384F873306E
:1068F800532384F8743084F87630A36DE26DC4F8BD
:1069080077300023C4F8803094F86030C4F87B20D6
:106918009A0684F875100FD194F8612094F8203005
:106928009A4209D294F86230013B0F2B04D8012314
:1069380084F87F302377A0E7206840F075FB0223B6
:1069480084F87F300423F5E7204640F0F9FB94E70C
:10695800032B92D1302394F8619003FB0949D4F8B2
:10696800803009F124095B44C4F88030BBF1000F82
:1069780016D0484640F00BFD90B141465A4648466D
:1069880040F017FD804628B902215B461F4A1C4883
:106998003FF0CFFAD4F87B30A3EB0803C4F87B3080
:1069A800D4F88020E36D9A420DD2484640F0EFFCBF
:1069B80000287FF462AFD4F88020E36D9A4202D2B7
:1069C800206840F047FB484640F008FD003818BFF3
:1069D800012084F87F00B5E7304695F8189040F01C
:1069E80018FB81457FF449AF237F052B10D184F82C
:1069F8001C8042E755534243F4100020FD19080853
:106A08000C3F07085C190808801908089B1A080831
:106A1800022B7FF432AF4FF030092A8AD4F8803045
:106A280094F861801344C4F8803023681969D3F856
:106A380004B091F8613009FB031124310846039131
:106A480040F0A5FC03990246584640F00DFB00288B
:106A58007FF413AFD4F87B3013B1206840F0E4FA28
:106A680009FB08402430AFE7304695F8188040F01D
:106A7800D0FA804502BFA37F03F1FF33A37707E76E
:106A8800EB7F0133EB77A4E62046FFF7E7FDA0E6AE
:106A9800204640F099FB9CE6022084F87F000423FE
:106AA8001AE094F9601040B90029206802DA40F031
:106AB800BBFABEE640F0CEFABBE6002914DA9042F3
:106AC80002D8B9F1000F06D1206840F0ADFA0223D0
:106AD80084F87F30E3E702232377237F022B0ED14C
:106AE800204640F071FB13E6904202D8B8F1000F3F
:106AF80003D1206840F0AEFAE9E70323ECE7032B63
:106B080003D12046FFF7AAFD02E6042B7FF400AE6E
:106B1800A37F2BB101211D4A1D483FF001FAF7E57B
:106B2800206840F076FA8046204640F05AFA05463A
:106B3800024604F1730304F17F0153F8040B8B42FE
:106B480042F8040BF9D11B782946137040460D22F0
:106B5800FFF7CEFC0646014620683FF099FF78B162
:106B68000C4A434601210A483FF0E3F93046FDF755
:106B780057FD2946204640F017FB40F0E1FAC7E5EB
:106B8800A37F0133A37705232377C1E5C11A08083A
:106B98000C3F0708FD190808802938B50D4614462A
:106BA80021D083290DD019BB80235371832303205F
:106BB800117193710023E07023706570A370043025
:106BC80038BD0223137101235371002393710A23E3
:106BD800D37108224168A0185CF0CFFB064B0E2049
:106BE8001B882382E6E7044B02201B889380E1E799
:106BF8006FF08500E4E700BFE36808082DE9F0417D
:106C08008769D0F82480BA4228BF3A46B2FBF8F424
:106C18000646C269234600683FF0F7FA0546C0B940
:106C2800B7FBF8F7A7420BD1002205213068FCF723
:106C3800E7FB28B101210A4A0A483FF071F901250A
:106C4800F3692344F3613DB10020074BB362BDE80B
:106C5800F08100240125E7E7706A6043F7E700BF89
:106C6800E21A08080C3F07080203000C81420B4691
:106C780007B509D302210D4A0D483FF05AF96FF0C4
:106C8800150003B05DF804FB6AB101391144814273
:106C980001D28B4207D90221009305481346054AC1
:106CA8003FF051F9EBE70020EBE700BFF91A0808BD
:106CB8000C3F0708101B08080C290346084616D184
:106CC8001B78252B12D009D8122B10D8084A42FA63
:106CD80003F313F0010F08BF0620704703F0FD020D
:106CE800282A03D05A2B08BF0A2070470A20704769
:106CF800F6FFFBFF2DE9F041984690F82C3086B05E
:106D080023F00C0380F82C300023C0E9043383619E
:106D1800062A04460F460B7840F010810BBB4B79CE
:106D28005B0724D490F82C309F070DD402234FF42E
:106D380068521946002584F8283084F8291062859D
:106D4800284606B0BDE8F08140F07DFA0028EDD174
:106D5800002319461A46EDE70223052145F20232BF
:106D6800E8E7032B36D14E7916F0040604D0022347
:106D780005214FF41052DDE790F82C308DF80760AC
:106D880043F0040380F82C307023ADF8043090F8F9
:106D980029300D7903F00F038DF806300A23122DE0
:106DA80028BF12258DF80B30438D2A465BBA404622
:106DB80001A98DF808608DF809608DF80A600396BE
:106DC800ADF81030ADF81260ADF814605CF078FAE8
:106DD800A662B5E71B2B00F0898009D8122B1AD0C0
:106DE8001A2B61D00121B24AB2483FF0A2F8BEE79F
:106DF8001E2BF7D14B795E07B9D40B7913F0030337
:106E080000F09780012BA3D190F82C3043F00103B8
:106E180080F82C309CE74B795E07A8D490F82C308A
:106E280043F0040380F82C304A7812F002061FD190
:106E3800D5078B7822D5B1F8035042461946FFF79B
:106E4800ABFE6DBAADB285420BDAB7F803506DBA36
:106E5800ADB200231A4684F8283084F82960628588
:106E68006EE742462046B978FFF796FE051EF0DA2F
:106E7800022305264FF410520025ECE72BB102211E
:106E88008D4A8C483FF055F8F2E7B1F80350414677
:106E98006DBAADB240F00DFA232DD6D94146204641
:106EA80040F007FA2425D4E74D7915F004057FF45E
:106EB8005EAF90F82C3043F0040380F82C308B78C8
:106EC8003F2B0ED1CE78002ED2D10D790323042D7D
:106ED80028BF042540462A4601A901935CF0F0F931
:106EE800B7E7022305264FF41052B4E74B79590748
:106EF8003FF53DAF3B791A090CD19A070AD5DB0754
:106F080015D494F82C3003F00303032B3FF424AF7B
:106F1800002305E094F82C209707C2F34003F0D52E
:106F280094F82C2063F3410284F82C2010E7012305
:106F3800F6E790F82C2063F30002F5E70A2A7FF4BD
:106F480051AF2A2B1AD8222B7FF64CAFA3F123027C
:106F5800072A3FF647AF01A151F822F0DB6F01087D
:106F6800ED6D01085D700108ED6D0108ED6D01081A
:106F7800C5700108ED6D01081D7101085A2B7FF4D9
:106F880031AF4D7A15F004057FF4F1AE90F82C304E
:106F980043F0040380F82C308B783F2B40F0DD80E1
:106FA800CE78002E40F0D9804FF4C063CDE9013689
:106FB800B1F8075040466DBAADB2082D28BF082574
:106FC80001A92A465CF07CF93246334684F8282029
:106FD80053E07B7A13F004037FF4C9AE01AEADF839
:106FE8000430B370082390F82C208DF8073042F055
:106FF800040280F82C2040F026F90028B5BF4FF095
:10700800FF3302220322236A8DF80C20A8BF1BBA83
:107018000293636A31461BBA8DF80D30C3F3072219
:10702800C3F307438DF80F3094F82C308DF80E20F9
:1070380043F0040384F82C30B7F8075040466DBA83
:10704800ADB20C2D28BF0C252A465CF039F9002377
:10705800A36275E67E7A16F004067FF488AE90F88F
:107068002C3043F004039D0780F82C3009D4022605
:107078004FF46853002584F8286084F829606385F4
:107088005EE640F0E0F80028F1D1236A03B1013B45
:1070980094F82C10626A1BBA12BA41F0040184F801
:1070A8002C100825C8F80030C8F804200023E2E7AF
:1070B800571B08080C3F07083A1B08087B7A580733
:1070C8003FF555AE94F82C30D7F8026043F004032E
:1070D8009907B7F8075084F82C307FF527AE20467B
:1070E80040F0B1F800287FF421AE6DBA36BAADB2DF
:1070F8002A463146206AFFF7B9FD20B1022305214F
:107108004FF4045216E6174B2361636AE6616B433A
:10711800A3611DE67B7A5A073FF529AE90F82C301B
:10712800D7F8026043F00803B7F8075080F82C300E
:107138009B077FF5FBAD40F086F800287FF4F6AD9D
:107148006DBA36BAADB22A463146206AFFF78EFDCF
:107158000028D3D1044B6361D7E7022205264FF4F8
:10716800105333E71D730508056C010810B5046951
:107178000346204640F8143B0122002142F0D7FD87
:1071880004F12C00024942F04AFE002010BD00BF65
:107198002573010838B503461B6940685C681B699C
:1071A80025685A681AB19A680AB1DA683AB9134870
:1071B8000121134A3EF0B4FE6FF0150038BD1033BC
:1071C800D3E8EF1F41F00101C3E8E21F002AF7D11D
:1071D800216909B90020F1E72B7A002BFAD13FF099
:1071E800B1F928B10121074A04483EF099FEF1E7B8
:1071F80020693FF034FA2872ECE700BFF43E070834
:10720800721B0808B319080838B504694068006893
:1072180004F11005D5E8AF5FED071FD40BB15D6829
:107228003DB9104A104801213EF07AFE6FF0150072
:1072380038BD90F820501DB1DD680DB90B4AF1E753
:1072480085791DB19D690DB9094AEBE7C4E90212B8
:1072580063600274120A42740020E9E76FF0770055
:10726800E6E700BF9C1B0808F43E0708BB1B08089C
:10727800DA1B08082DE9F347D0F804A00669884608
:1072880015467768DAF8044006F11003D3E8AF3FF3
:107298009B073BD5236960685B68D3F800903FF093
:1072A800ABF800220023012829460CBF99F81B904F
:1072B80099F81490DAF80C00CDE9002342463FF023
:1072C80033F8054650B90121124A13483EF028FE0A
:1072D8006FF00B04204602B0BDE8F087014680F845
:1072E800189020463FF0D4FB044618B12846FDF715
:1072F80097F9EFE7FB69002BECD14FF0FF324FF025
:10730800FF3306F1140004F031FDE3E76FF00C04DD
:10731800E0E700BFFB1B0808F43E070870B550F80B
:107328002C3C5C6865681C38D0E8AF3F9B0725D5C6
:107338002B6968685B681E683FF05EF800220128C8
:107348004FF00003A0680CBF96F8296096F82260F9
:107358003EF0E6FF044630B9094A0121BDE8704015
:1073680008483EF0DDBD0146067628463FF090FB12
:1073780020B12046FDF754F9034AEEE770BD00BF7F
:10738800161C0808F43E0708301C080807B5084A08
:1073980092E80300CDE9000106488268126822B12C
:1073A8006946904703B05DF804FB6FF05700F9E7B2
:1073B800303F0708883907081F2808B5034606D94B
:1073C80009480121094A3EF0B4FD002008BD01200A
:1073D800074A00FA03F3D16833EA0101F6D01269CB
:1073E800934318BF0020F1E7CC3D0708651C080847
:1073F80000200246012100F01F021F2808B501FAEB
:1074080002F2034606D90648064A3EF092FD6FF09E
:10741800150008BD044B0020DA601A61F9E700BFC7
:10742800CC3D0708651C0808002002462DE9F041FC
:10743800054600264FF001080E4F6B78F4B2A342C0
:1074480001D8BDE8F0812B781C442046FFF7B4FF33
:1074580068B12046FFF7CEFF57F834303BB107EB51
:10746800C40204F01F04516808FA04F09847013672
:10747800E3E700BF44380020014B1954704700BFB0
:10748800480C0020034670B1B0FA80F2C2F11F0226
:10749800D2B206498856064AD2F880100B43C2F881
:1074A8008030FCF7B1BBFF22F3E700BF480C002097
:1074B80000200246034AD2F8803023EA0003C2F8CB
:1074C8008030704700200246032921D8DFE801F008
:1074D800020C10190F4B1A6822EA00021A605A6847
:1074E80022EA00025A6070470A4B1A680243F5E71D
:1074F800084B5A6802435A601A6822EA00021A6066
:107508007047044B1A6802431A605A68104358605F
:10751800704700BF0020024630B5B0B1B0FA80F322
:10752800C3F11F03DBB20B4850F833408C4204D13F
:1075380000EBC3056D68954205D044B940F8331097
:1075480000EBC3004260002030BDFF23EBE76FF083
:107558000F00F9E74438002060B1B0FA80F3C3F1B6
:107568001F03DBB20021044A42F8331002EBC302C6
:1075780051607047FF23F5E744380020C300074AED
:10758800C0F38100183052F8202003F018000F23B0
:107598008340134023FA00F0704700BF00200246E2
:1075A800F8B504690D4600AFA034D4E8AF3FC3F383
:1075B8008003994218D1164A164B6E4688B00029A6
:1075C80018BF13466A461449CDE905134FF40073F2
:1075D800ADF81C30114B42F8103F00234FF4E45132
:1075E8000F48FBF7E1FBB5464DB1D4E8EF3F43F058
:1075F8000403C4E8E23F002AF7D1BD46F8BDD4E849
:10760800EF3F23F00403C4E8E23F002AF5D0F6E791
:10761800A51C0808AD1C0808B41C080803000001D4
:10762800A43E07082DE9F0470546894690461F46BF
:10763800D0F808A040F063F90446D0B1067FF307FC
:107648000AD590F8203018480121184A3EF071FCFC
:107658006FF07700BDE8F0873B464246494640F068
:107668000CF948B994F820300121114A0E483EF02F
:1076780060FC6FF01200EDE79DF8203026F006065A
:1076880084F82180678484F824302677DAF8183063
:10769800214628469847B0FA80F3227F5B0963F3B6
:1076A80000022277D6E700BFA43E0708C61C0808D8
:1076B800E01C080870B50546866840F020F90446C5
:1076C800D8B1037FDB0709D490F820300C4801219A
:1076D8000C4A3EF02EFC6FF0770070BD0146F3694E
:1076E8002846984738B1237F03F00103227F63F3CC
:1076F80000022277F1E70346F8E76FF01200ECE7A3
:10770800A43E0708021D08082DE9F3411746D0F8E2
:1077180008800546D8F83C300E46984700220023DA
:1077280039460B48FCF7FEFE044670B901213B467A
:10773800084A094800963EF006FC2846D8F840302A
:107748009847204602B0BDE8F0810676F5E700BF0D
:10775800581200201D1D0808A43E070813B5036928
:107768000C46D3F8A40091F8201041F031FD94F8AC
:10777800203048B101210090084A09483EF0E3FB57
:107788006FF0040002B010BD5B0601D10020F9E7DC
:10779800237F43F002032377F8E700BF4B1D080857
:1077A800AC3E0708F8B591F9203091F82060002B1D
:1077B80001DB0020F8BD7306FBD047684C8CB7F896
:1077C8004830C4F30A04A34294BF03330334006966
:1077D8008CBFA3089B08D0F8A440402B98BF5B003F
:1077E800D4F8E8049D008AB9A84224BF401BC4F815
:1077F800E80491F820100022204601F07F0141F0B2
:107808007BFD0028D5D06FF00400D3E7BA68121AC0
:10781800AA4207D20A4832460A4940F0D2FB6FF022
:107828000B00C7E720469AB206F07F0141F064FDDD
:107838000028E8D1D4F8E8342B44C4F8E834B8E791
:10784800AC3E0708791D0808F7B5466803697468EF
:10785800D3F8A45064009834A1B20746A40028467F
:1078680041F069FDC5F8E8440124102200212846AA
:1078780041F042FDD5F8E8344033C5F8E834736880
:107888009C420ED3284641F0B5FB054680B1174906
:107898000246174840F095FB6FF00404204603B0F9
:1078A800F0BDE1B20022284641F026FD0134E6E7AA
:1078B80002460146009040233846FFF7B3FE0446CF
:1078C80028B12A460B490A4840F07BFBE6E7024606
:1078D8000090402380213846FFF7A4FE044608B1F3
:1078E8008022EFE73069FCF78FF9D7E79C1D08087D
:1078F800AC3E0708B11D080838B504460369D3F83B
:10790800A45043681869FCF78DF900212046FFF759
:10791800D1FE38B10C490D4840F058FB6FF0040413
:10792800204638BD20468021FFF7C4FE04460028C3
:10793800F0D1284641F07BFB02460028F0D00449EC
:10794800024840F03EFBE9E7CB1D0808AC3E0708BB
:10795800EE1D080838B503690546D3F8A44020464B
:1079680041F0C4FC024630B10D490E4840F029FBF5
:107978006FF0040038BD0021142042F090FB20462F
:1079880041F0B7FC04460028F2D101462846FFF72B
:1079980007FE2246022128463FF0EBFF2046E9E792
:1079A800021E0808AC3E070870B50369456804461E
:1079B800D3F8A40041F009FB024618B11A491B4844
:1079C80040F0FFFA6668F069D8B143689847044602
:1079D800B8B117490246154840F0F3FA002C19DBF4
:1079E80000F0F8FB024618B11249104840F0E9FAD5
:1079F8002869FCF72BF910B12869FCF713F9002066
:107A080070BD0D48716983685B6843B90B490748C5
:107A180040F0DCFA0A49054840F0D8FAE0E7984710
:107A28000028DDD0F2E700BF221E0808AC3E070898
:107A3800381E08088B1E080888390708561E0808CB
:107A4800721E08082DE9F04103690646D3F8A450D0
:107A5800476800F08BFB044638B12E4902462E4891
:107A680040F0AFFA2046BDE8F08176682B4896F8DA
:107A78004A30D0F80880012B13D97169D8F818302A
:107A8800083153B92649244840F0A0FA254922482C
:107A980040F09CFA6FF00404E4E722469847002877
:107AA800F0D1D8F8003071690BB91F49EBE71B48D2
:107AB800984704460028F8D1F06950B10368984700
:107AC800064630B119490246134840F07AFA002EAA
:107AD800DCDB40F2E442002128465BF017FC3B68FF
:107AE80028462B607B682B7140232B723B6B6B7293
:107AF8007B6BEB7102F03AFE024620B10C49064856
:107B080040F05FFAC6E7284641F091FA0028A9D06C
:107B1800C0E700BFA91E0808AC3E07088839070857
:107B2800C61E0808201F0808E81E0808031F0808C2
:107B3800381F08082DE9F04F064600274FF0280A9D
:107B48004FF0400BD0F810904568D9F8A4808BB05E
:107B58006B68BB4256D800274FF0280A4FF0400BFD
:107B68006B68BB4200F2858099F8803023F06A0385
:107B780043F06A0389F880306B6B2BB999F8803031
:107B880043F0010389F88030C8F8E46408F5C0615F
:107B980008F5BA600823042241F0B4FFD5E91012B1
:107BA80008F59E684FF0000A4FF0000B6FF00703CE
:107BB80001200027CDE90330CDE906AB4046CDE9E9
:107BC8000177514B009604F04BFB3168404642F078
:107BD80064F9EB6898473946A86909AA40F040FE5D
:107BE800041E07DB099B3A461979186840F04AFEDB
:107BF800041E6BDAA31C69D044492246444840F06D
:107C0800E0F930E00AFB07F1EB6B17F0800F0B444B
:107C18009A7E07F07F000CBF42F0400242F020023B
:107C28009A769A7E83F8207050B942F001029A76CB
:107C3800EB6B5FB1EB6BB5F848200B441A8307E098
:107C480022F00E0242F00E029A76F3E7A3F818B07B
:107C5800EB6B304619443FF064FE044638B12D49B9
:107C68002B4840F0B3F920460BB0BDE8F08F013740
:107C78006EE70AFB07F1AB6B67F07F020B4483F8F2
:107C880020209A7E7C0642F020029A760BD1D2B24E
:107C980042F001029A76AB6B67B1AB6BB5F848203E
:107CA8000B441A8308E09A7E22F00E0242F00E027C
:107CB8009A76F2E7A3F818B0AB6B304619443FF058
:107CC80030FE04460028CAD1013749E7A86A08B936
:107CD8000024C8E7283541F029FE30B90E490C4880
:107CE80040F074F96FF01504BDE74FF4B011284661
:107CF80040F026F90028EBD00849054840F066F91D
:107D08006FF00404AFE700BFF17D0108681F0808A1
:107D1800AC3E07084C1F0808861F0808A21F080861
:107D280073B5D0F8A46008460C4615463FF0F0FD40
:107D380018BB94F82030298A802BEA680B4602D1B8
:107D4800402928BF4023D018C91AE8602982304644
:107D580094F8201041F022FA58B194F8203001210B
:107D68000090074A07483EF0EEF86FF0040002B0B2
:107D780070BD012120463FF0CFFD0020F7E700BF8E
:107D8800BF1F0808AC3E070813B591F820300C4611
:107D9800D0F8A400DBB9537EDB071ED4538AC0F8A1
:107DA800EC34538A402B28BF4023D26894F8201023
:107DB80041F0CFF968B194F8203001210090084AC9
:107DC80008483EF0C0F86FF0040002B010BD538AB6
:107DD800EBE7012120463FF09FFD0020F5E700BFBB
:107DE800F01F0808AC3E07082DE9F347074603696A
:107DF800D3F8A4604FF0FF334FF0FF3201A906F526
:107E0800BA6003F01BFE9DF80430012B5FD0022BF3
:107E180007D0002BEED1384606F29C413FF0DCFD3E
:107E2800E8E79DF80590D6F8E48449F0800A5146C1
:107E380040463FF064FD054600213FF06DFD2846B1
:107E48003FF08AFD04460028D4D019F07F0F18D1DE
:107E5800038AB3B1402B28BF4023C2688021304633
:107E68001D4641F09BF9024620B13F493F4840F08A
:107E7800A8F8BFE7238A5B1B2382E3682B44E360EF
:107E8800B8E720463FF06CFD814660B120463FF0E0
:107E98006BFDE26800235146304641F07FF9024607
:107EA8000028A7D0E1E728463FF052FD4A460146A0
:107EB80040463FF06AFD28463FF04EFD0246002846
:107EC80098D02946D8F81000FFF72AFF92E79DF8C6
:107ED8000590D6F8E48449464046BDF806A03FF030
:107EE8000EFD05463FF038FD044648B920494A468C
:107EF8001E4840F066F8214628463FF00DFD79E718
:107F080051460C303EF03CFAB9F1000F17D1BAF1E6
:107F1800400F14D1228AD6F8EC349A420FD2E06886
:107F2800638A61699B1A411A5B1A402B024428BF75
:107F38004023304695F8201041F00BF95AE72846BF
:107F48003FF006FD0022014640463FF01EFD284650
:107F58003FF002FD024628B12946D8F81000FFF785
:107F680013FF47E70146C7E720200808AC3E07088B
:107F780049200808F7B591F82150036905F0030571
:107F8800D3F8A4706B1E022B4FF001020C4688BF79
:107F98000025FFF707FC064698B9628C2B46384641
:107FA80094F82010C2F30A0241F077F848B194F827
:107FB800203001210090044A04483DF0C4FF6FF0CE
:107FC8000406304603B0F0BD62200808AC3E07083E
:107FD80013B503690C46D3F8A40041F04BF840B13F
:107FE8000121009023460448044A3DF0ACFF6FF09D
:107FF800040002B010BD00BFAC3E07088B20080883
:1080080037B5036905460C46D3F8A40091F820104B
:1080180041F077F8024630B92146284603B0BDE85A
:108028003040FFF7BFBB94F8203001210090044A8C
:1080380004483DF088FF6FF0040003B030BD00BF76
:10804800B9200808AC3E070873B5036905460C4615
:10805800D3F8A40091F8201041F0F1F858B194F841
:10806800203001210090164A16483DF06CFF6FF051
:10807800040002B070BD237F60F3410323772046DC
:108088003FF06AFC064608B90020F2E720463FF0B8
:108098003FFC94F92030002B07DA0028F4D132464F
:1080A80021462869FFF73CFEEEE70028ECD132466E
:1080B8002146286902B0BDE87040FFF765BE00BFE1
:1080C800E3200808AC3E070837B50D46044641F0E2
:1080D8005DF801238DF805508DF80430ADF80600E1
:1080E8000022002301A904F5BA6041F01EFD18B171
:1080F800024903483FF06AFF03B030BD1321080866
:10810800AC3E0708002307B5ADF8063002238DF80A
:1081180005108DF804300022002301A900F5BA608B
:1081280041F003FD18B1034903483FF04FFF03B086
:108138005DF804FB13210808AC3E0708002307B5C7
:1081480001930022002301A900F5BA6041F0EDFC7B
:10815800002803DA034904483FF038FF03B05DF80C
:1081680004FB00BF13210808AC3E070838B54FF0E0
:10817800FF324FF0FF33124803F0F8FD0446C0B950
:10818800104D2B685A1C2A6083B90F4BDA6802F429
:108198004032B2F5003F0ED26FF0040401210B4AC1
:1081A8000B483DF0BDFE2B68013B2B60044803F0F3
:1081B800A1FD204638BD1A6942F080521A61F5E7E0
:1081C80084110020A43A002000080246462108082D
:1081D8008C3E070810B54FF0FF324FF0FF330A48C6
:1081E80003F0C4FD044660B9084A1368013B1360F4
:1081F80023B9074A136923F080531361024803F037
:1082080079FD204610BD00BF84110020A43A00204B
:1082180000080246074B1A6822F004021A605A68DE
:10822800D207FCD40222DA601A6842F001021A600E
:10823800704700BF00040340044B1A6822F0010293
:108248001A601A68D207FCD4704700BF00040340C4
:108258000D4A0E49936813F4000308D0936813F489
:1082680000030CD1D2F8F42051F82300704790682D
:10827800000207D4D2F8F430C3F30333F4E7936869
:108288001B0FF1E79268EFE7000C02463048070839
:1082980038B50B880D46C3F30B03122B144636D89A
:1082A80013B96FF0850031E0013B112BF9D801A219
:1082B80052F823F0378301086B830108058301080E
:1082C800AB820108AB820108538301084D83010882
:1082D800AB820108AB8201083183010831830108B0
:1082E8003183010831830108318301083183010892
:1082F8005783010837830108378301084FF4FA4090
:1083080020602B68B3F5805F2ED2002038BD882B03
:108318000AD003F67473C3F30B031C2BC1D8164A97
:1083280022FA03F3DB07BCD5144B1868E8E7FFF71C
:108338008FFF4FF42023A0FB0303400B40EAC34008
:108348004008DDE7FFF784FFDAE70D48D8E7FFF7D5
:108358007FFF4FF42023A0FB0303400B40EAC340F8
:10836800CEE74FF40040CBE7C3F313330133B0FB40
:10837800F3F02060C9E700BF11011111C806002001
:10838800006CDC0237B5A84CA84BE26902F00C027D
:108398001341D80700F14381FFF75AFF236AA44A23
:1083A80003F00F03D35C20FA03F5A24BDA6842F41A
:1083B8004032DA60DA681104FCD59F48854201D260
:1083C80003F03EF8984CD4F8943043F00403C4F812
:1083D8009430D4F8943003F004030093009BFAF728
:1083E800D9F9D4F8F03023F0180343F01003C4F897
:1083F800F030D4F8F03043F00103C4F8F030D4F88A
:10840800F0309A07FBD5D4F8F03043F08003C4F875
:10841800F030854CD4F8F0301B05FBD5FAF7D8F9C5
:10842800A36843F40003A360A36823F0704343F0F8
:108438008043A360236843F040032360236843F02C
:1084480008032360236843F001032360764B1A680E
:108458005407FCD5D3F8942050070BD4D3F89420B4
:1084680042F00402C3F89420D3F8943003F00403D4
:108478000193019B6C4CFAF78DF9D4F8F03043F076
:108488008063C4F8F030D4F8F0301901FBD5FAF75E
:108498009FF9236843F480532360634B1A6892045E
:1084A800FCD5DA6902F00C020C2A1AD11A685405B4
:1084B80007D41A6842F480721A605B4A1368580538
:1084C800FCD5594BDA6922F0030242F00102DA6165
:1084D800DA6902F00C02042AFAD11A6A22F00F02B1
:1084E8001A62514B1A6822F080721A609A6A22F056
:1084F800030242F001029A624E4AD16821F48021B7
:10850800D160D46814F48044FBD19A6A464922F4B5
:1085180070429A62494B4A4A1B699342B6BF494A1C
:10852800102393FBF2F38A6A03EBD37322F47042AD
:108538005B1042EA03338B623E4BDA6842F48022D6
:10854800DA60DA685104FCD5FFF782FE3E4AA0F5EE
:108558007413A3F51063934205D93C4B394A03447D
:1085680093425ED20C24304B9A6A22F470629A626B
:108578009A6A22F00C0222439A625A6B6FF308023D
:1085880042F04F025A639A6A22F010029A625A6BBA
:1085980022F4FE0242F480325A639A6A42F40032AC
:1085A8009A625A6B22F0FE4242F080725A639A6ACB
:1085B80042F480229A621A6842F080721A601A683D
:1085C8009201FCD5DA6A22F00302DA621A6B22F011
:1085D80003021A631A6A22F00F021A621A6A22F058
:1085E80070021A621A6A22F4E0621A625A6A22F067
:1085F80070025A62DA6942F00302DA610A4AD36900
:1086080003F00C030C2BFAD10B4CA54202D32046E5
:1086180002F016FF00200E4B1C6003B030BD002096
:10862800BCE66FF02100F8E7000C0246FEEFFFFF02
:10863800A26A080800080246006889093048070845
:108648000020A10700127A0000093D00FFED85FF18
:10865800C8060020192808D8054BC34013F0010F9D
:108668000CBF6FF08500002070476FF085007047E1
:10867800CEFC060208B5074841F058F938B106485B
:10868800FBF78AFE0448FAF735F8002008BD6FF0BA
:108698001200FBE7643B0708A58601080A2838B5DD
:1086A8000446074D04D1AB680D2128465B689847FE
:1086B800AB6803485B68E1B29847204638BD00BF05
:1086C800643B0708064A11680B6823F004030B6033
:1086D8005068044B196883685B6803B11847704792
:1086E80078050020E405002010B5094BD3E90040C7
:1086F800084B196883681B6803B19847236843F0DF
:1087080004032360236843F00803236010BD00BFFF
:1087180078050020E405002008B5EFF31181102347
:1087280083F31288BFF36F8F0120094B93F8482019
:1087380083F8480081F31188BFF36F8F32B9FFF7D0
:10874800D3FFBDE808405E20FBF75EBA08BD00BF56
:108758007805002038B543680569394868601968A4
:1087680083681B6853B19847044650B101212346DA
:10877800344A35483DF0DDFB204638BD6FF05704DC
:10878800F4E7012205F10800114641F0D0FA012270
:10879800214605F1200041F0CAFA05F138002B49BD
:1087A80041F03DFB072385F86130042385F86230EA
:1087B8000F2385F84C300C23224685F84D3021468E
:1087C8005E2085F85E4085F85F4085F8604085F852
:1087D800494085F84A4085F84B403DF040FD1C4B28
:1087E8001C491B681A681D6922F07C4222F07F022E
:1087F8008A42D86806D14AF2B0218D4202D1164980
:10880800884211D0196821EA0201144A0A431A6001
:108818004AF2B0221A61104ADA601A6822F08042DD
:108828001A601A685200FCD41A6842F004021A60EE
:108838001A6842F008021A60FFF76EFF9CE700BF53
:108848008839070891210808C43D07082F820508C0
:1088580078050020000DF000BB7C0100000DF04001
:10886800F8B58378C678EFF3118E102484F3128854
:10887800BFF36F8F057890F801C05B1B33409A42B5
:1088880088BF9AB2AF1837402C4607708EF311880C
:10889800BFF36F8F8F188F421BD165450CD1EFF353
:1088A8001181102484F31288BFF36F8F0478447009
:1088B80081F31188BFF36F8F01799B1A994294B2A3
:1088C80005D341F0E4FA68B1084803F0D3FB204629
:1088D800F8BD00EB040E9EF805E0013401F801EB49
:1088E8003440D8E7FFF718FFF1E700BFB0050020D4
:1088F80070B50D4614460CB9204670BD4FF0FF32D6
:108908004FF0FF330B4803F031FA224629460A4854
:10891800FFF7A6FF064630B94FF0FF324FF0FF339E
:10892800064803F023FA0348A41B03F0E3F9A4B2B2
:108938003544E0E780050020D60500209805002092
:1089480010B51D4B01461B68EFF31184102282F30A
:108958001288BFF36F8F5A68500605D45A68D20739
:108968001DD46FF00A0015E01A6842F080421A60C0
:108978001A6822F080421A600A221868400005D45A
:108988005868400602D458684007E7D5013AF4D140
:108998006FF0040084F31188BFF36F8F10BD5A681D
:1089A8009207F5D4586810F04000F1D19B680B602D
:1089B800002BEFD1D5E700BF780500202DE9F7435C
:1089C800D8078846144605D43148FFF749FF03B055
:1089D800BDE8F083002A37D0EFF31185102383F325
:1089E8001288BFF36F8F5E20FBF730F906465E20D2
:1089F800FBF718F985F31188BFF36F8F0EB9FFF7EE
:108A080073FEDFF89490D9F800305A68510713D4F0
:108A18005B685A0610D44FF0804325461D4FC7F8AF
:108A28008831D9F800305B68DB070FD4BFF34F8F6C
:108A380020BF40BF20BFF4E701A8FFF781FF002453
:108A480016B35E20FBF7E0F82046C0E701A8FFF761
:108A580077FF4FF080420346C7F8882188B9291F5D
:108A6800019A89B2002DEBD0A94203D1002BD8D0AE
:108A78000192D6E7013DADB208F805200123120A9C
:108A8800F0E7002DCDD1DBE7FFF71CFEDCE700BFE8
:108A9800C105002000E100E0780500202DE9F7433A
:108AA80001A8FFF74DFF002843D10427804601465F
:108AB800264C019A94F84B3094F84CC094F84AE04C
:108AC800A3EB0E053CEA05055FFA82F91ED194F87E
:108AD800601094F85F6094F861508E1B35EA0606C2
:108AE8002AD108B184F84B30B8F1000F00D00192B8
:108AF8005E20FBF797F8FFF7E5FD002384F8483080
:108B0800134803B0BDE8F04303F0F4B8E01880F868
:108B18004E90012001330CEA0303013F4FF0010896
:108B28004FEA1222CCD108B184F84B3001920029C7
:108B3800E6D103B0BDE8F083661801310D4086F830
:108B48006390012184F86050E7E700BF78050020B2
:108B58009805002000487047D4450708044BB3F82F
:108B6800A0379B020B60002318464B60704700BF7C
:108B78000000FA0B07B50346054A00910548012194
:108B88003DF0E1F96FF0150003B05DF804FB00BF9C
:108B9800F7210808DC3D070873B506466422002360
:108BA800684641F0D6FADDE9004533691B681A6A60
:108BB80012F0FA0212D01A6A02F0FA021A626FF080
:108BC800040002B070BD22462B46684641F0E6FA22
:108BD800DDE9003213430CBF0122002233691B6810
:108BE800186A10F48030ECD0002AECD00A23012156
:108BF800024A03483DF09DF9E1E700BF2122080839
:108C0800DC3D070838B5036905461C6849B1FFF71C
:108C1800C3FF58B12869043003F06CF86FF0040002
:108C280038BDA36A002B06DB0020F9E7A36A43F0EE
:108C38000043A362F8E7034BA36003F18833A36002
:108C4800F2E700BF2301674573B5012306460D46C9
:108C580014463FF0B7FB50B90A482B4601210A4A8F
:108C680000943DF070F96FF0150002B070BD3CB192
:108C780022462946304602B0BDE870403FF07FBB2F
:108C88002046F2E7DC3D070835220808F7B51C4600
:108C980017460123224605460E463FF093FB58B976
:108CA800012100943346154A15483DF04CF96FF000
:108CB8001504204603B0F0BD002CFAD028693FF017
:108CC80030FB00212846FFF79DFF98B9314623461F
:108CD8003A46284600F0B8F8064601212846FFF72C
:108CE80091FF002E14BF344604462869043003F06F
:108CF80001F8DEE76FF00406EFE700BF602208081E
:108D0800DC3D07082DE9F84F494B17461B680D460F
:108D1800824603F001084FF0000BFFF78DFA013F80
:108D2800DFF82091434E2F44AF420CD3DAF81030CD
:108D38001C68A36A002B0EDA01213F4A3F483DF028
:108D4800EFF86FF0040BB8F1000F01D0FFF762FAEB
:108D58005846BDE8F88F5046FFF71EFFB0F1000BEC
:108D6800F1DBDAF810301B681B6C9B0252D54FF60A
:108D7800FD70B9F8A010226C4B1E9BB2834202F41E
:108D8800801250D8B5EB412F2CD26B0B002A43D15F
:108D9800A26A22F40062A262A26A504642F002026B
:108DA800A262A26A22F47E72A262A26A42EAC303A3
:108DB800A362A36A43F48033A362A36AFFF7ECFEBD
:108DC800DAF8103083461B681B6C13F4001FA36A83
:108DD80014BF334023F002030028A362B3DB05F578
:108DE8000055A1E7B5F5801F0BD332B1A36A23F470
:108DF8000063A3626B0B803BCEE7A36A43F4006376
:108E0800F7E701212B460E4A0C483DF092F86FF027
:108E1800150B98E76B0BBFE7B5F5801FE6D2A26A82
:108E280042F40062B7E7B5F5801FAED3DDE700BFB7
:108E380000040340FDF7FFFFB1220808E43D0708DE
:108E4800BE2208080007FA0B2DE9F84F00249846BF
:108E5800324B0D461F6806469146A346FFF7ECF9CC
:108E680007F0010705F10065D8450DD93369D3F836
:108E780000A0DAF82830002B0CDA0121284A29480A
:108E88003DF04EF86FF004040FB1FFF7C3F9204628
:108E9800BDE8F88F3046FFF77FFE041EF4DB2BF0A9
:108EA80003024A44111F0B460C3253F8040F00BB4F
:108EB8009342FAD1DAF8283043F00103CAF828308F
:108EC800DAF828302B4651F8040F914243F8040B86
:108ED800F9D13046FFF760FEDAF82830041E23F097
:108EE8000103CAF8283005F11005CDDB0BF1100B92
:108EF800BAE7284600230468013408D005F178450C
:108F08000121094A07482B443DF013F8BAE7013319
:108F1800042B00F10400EED1CCE700BF00040340AD
:108F2800B1220808E43D0708D722080830B5104CDC
:108F3800104D0C60236813B12B68136030BD0369B2
:108F48001B68196C1B6C9B020FD54FF6FD700A4B02
:108F5800B3F8A030591E89B281428CBF4FF4807398
:108F6800DB0823604FF40053636001232B60E4E7C0
:108F7800AC3A0020A83A00200007FA0B2DE9F84384
:108F8800D0F8049090460746D9F808000D461E46CA
:108F98003EF043FCB8F5001F044616D12846D9F820
:108FA8000840FEF7EBFA84420CD129463EF035FC26
:108FB8000446FEF77FFA2046FEF7CEFA0021204647
:108FC800FEF782FA0020BDE8F883B8F5800F20D0BC
:108FD800B6F1806F19D0B6F1C06F18D0B6F1007F26
:108FE8001AD102263A4620460E49FEF795FAB0B93C
:108FF8002846D9F808103EF015FC20463146FEF701
:1090080063FA2046FEF73EFADCE70126EAE7032684
:10901800E8E76FF08500D6E76FF01500D3E76FF04B
:109028000F00D0E7358505080C291FB528BF0C218E
:109038000C460A4BD3F8082712BA0192D3F8042732
:1090480012BA0292D3F800370A461BBA01A9039351
:109058005AF036F9204604B010BD00BF0000FA0BE4
:1090680080B500AF8AB06A46094B0791CDE9053053
:109078004FF40073ADF82030064B42F8103F002340
:109088004FF411510448F9F78FFEBD4680BD00BF6B
:109098000523080804000001143E07082DE9F743DA
:1090A80098460B7A164643F00403046907460B7288
:1090B8000D460B460122B2421AD904F118094FF0A5
:1090C800FF324FF0FF33484602F050FE38463FF07B
:1090D8008EFA041E2DDA012123461A4A1A483CF05A
:1090E80028FF484602F006FE204603B0BDE8F0839C
:1090F8000AD2197A187D81EA000C1CF0010F01D000
:1091080040071CD589071AD401320C33D2B2D2E7F2
:10911800012E0CBF002305F11403CDE900383846B1
:1091280095E80E003FF006FB041E04DB013E0C35FB
:10913800F6B2002EECD138463FF05BFAD1E76FF07B
:109148001504D1E719230808143E070808B50121BA
:10915800034A04483CF0E4FE6FF0040008BD00BF79
:1091680035230808143E07080023F7B5426804466B
:10917800066923480F46D568516892680193836849
:10918800012ADB6833D908314BB91E4A01211E4830
:109198003CF0C6FE6FF00404204603B0F0BD01AAFF
:1091A80098470028F1DB376306F118074FF0FF32C4
:1091B8004FF0FF33384602F0D9FD2B68204623F0E4
:1091C80001032B6096F862103FF0D4F9204601990C
:1091D80000F0BEF8041E06DB96F861301BB12B6860
:1091E80043F001032B60384602F084FDD4E70BB945
:1091F800064ACBE701AA98470028D4DAF8E700BF67
:109208008839070853230808143E070881230808EB
:10921800F8B504464668056900274FF0FF3200217B
:10922800284640F084FD20463368984785F86070EA
:1092380085F86270012205F11800114640F077FDAB
:10924800204600F051F8B368012B25D831691F4B2F
:10925800994230D014D81E4B99422ED01D4BCB1AB0
:10926800594259418900204641F01001FFF77CFF1F
:10927800041E26DA0121184A18483CF051FE13E072
:10928800174B99421BD003F5C31303F5206399428A
:109298000CBF0A210021E6E712487168836808318B
:1092A8009B691BB96FF004042046F8BD3A469847FD
:1092B8000028CBDAF6E70621D5E70221D3E7082113
:1092C800D1E70123002485F86030EDE740420F0024
:1092D800A0860100801A0600AF230808143E07087C
:1092E80040E133008839070837B545680021286A06
:1092F80001AA3FF0B5FA041E07DB019B0022197989
:1093080018683FF0BFFA041E08DA012123460C4A08
:109318000C483CF00EFE204603B030BD0A48696890
:1093280083681B683BB90121084A06483CF0F8FDF0
:109338006FF00404EFE7984704460028EBD0F2E703
:10934800D3230808043E070888390708F1230808CA
:109358002DE9F04F4FF00C0E44680369002085B0EA
:109368000393A36AE568DFF82881DFF82891DFF81E
:1093780028A1DFF828B10293029B8342039B1B6B51
:1093880001930DD1C3F34202012A39D0022A66D0D3
:109398003A4A3B4801213CF0C3FD6FF015001DE03F
:1093A8000EFB00F7D4F824C0364A0CEB07067368A6
:1093B80093421DD015D853451CD0A3EB0B02534242
:1093C80053419B00019A534013F00E0F16D15CF8DD
:1093D80007308B4212D1B36800202B6105B0BDE87D
:1093E800F08F434508D04B450CBF0A230023E9E71B
:1093F8000623E7E70223E5E70823E3E70130BBE7B5
:1094080041F25C2E4FF47A6C40F2E2474FF4FA7660
:1094180002201D4B421EB1FBF2F2B3FBF2F2BCFB81
:10942800F2F4013CFF2C23D8BEFBF2F808F1FF3818
:10943800B8F1FF0F1CD8B6FBF2F9B9F10F0F17D826
:10944800B7FBF2F2013A0F2A12D8023848EA094368
:1094580043EA007343EA025343EA0423BCE740F2B9
:10946800145E4FF4167C4FF4FA7740F27716CFE784
:1094780001301128CED1054A8BE700BF3B240808EC
:109488000C3E070840420F0000CA9A3BB624080861
:1094980040E13300404B4C00A0860100801A0600D2
:1094A80043681B6803F1080252E8002F42F00102EA
:1094B80003F1080040E800210029F3D1174A93423C
:1094C8001ED002F1805293421AD0154A934217D007
:1094D80002F18052934213D0124A934210D002F103
:1094E800805293420CD0104A934209D002F1805224
:1094F800934205D00D4A934202D0B3F1502F03D1C5
:109508005A6842F040025A6053E8002F42F48072D1
:1095180043E800210029F7D1704700BF0038014017
:109528000044004000480040004C0040005000400B
:1095380043681B6803F1080252E8002F22F0010279
:1095480003F1080040E800210029F3D1174A9342AB
:109558001ED002F1805293421AD0154A934217D076
:1095680002F18052934213D0124A934210D002F172
:10957800805293420CD0104A934209D002F1805293
:10958800934205D00D4A934202D0B3F1502F03D134
:109598005A6822F040025A6053E8002F22F4807281
:1095A80043E800210029F7D1704700BF0038014087
:1095B8000044004000480040004C0040005000407B
:1095C8000129034608461AD002290BD0C9B91B68DD
:1095D8000D4A934217D002F180529B1A18BF0123FB
:1095E800180370471868084B98420AD003F1805353
:1095F80098420CBF4FF400504FF440507047002081
:1096080070474FF4005070470024004638B51D4697
:10961800094B6C0833F812200023F7F71DFC0902E8
:1096280041EA1061000220182A464FF0000341F178
:109638000001F7F711FC38BDC80208082DE9F0470A
:1096480082B0436880460C461D6800AF002945D0AB
:10965800586819698368DB686BB13A1D9847061E1C
:109668000CDA0121344A35483CF05AFC30460837B8
:10967800BD46BDE8F0876FF05706F2E7304B9D42D4
:1096880003D003F180539D422BD10026D7F80490D4
:10969800DFF8BCA0234648460021B2B2FFF7B6FF68
:1096A800A0F5407050452BD90136102EF2D16D46E9
:1096B8008AB0D8F800306A4622490794CDE90513E4
:1096C8004FF40073ADF820301F4B42F8103F0023D1
:1096D8004FF411511948F9F767FBAD466FF01506BD
:1096E800C4E72B6823F400432B607B6803EB540327
:1096F800B3FBF4F30F2BDAD99BB2EB600026B5E786
:10970800EB6A484623F00F033343EB620F4B33F801
:10971800162000231946F7F79FFB002306464FF44F
:10972800807C194660082246E6FB0C01F7F794FB9B
:10973800C0F31300E860E1E7812308089C3E0708AE
:1097480000240046FA24080804000001C80208089A
:10975800FFFC0F002DE9F84307460E7940683B6986
:10976800012E0D460468D3F8008014D0B31ED3F13F
:10977800000949EB03094FEA89296979FFF720FFB6
:10978800AA790346022A09D0042A01D0002E6AD0F9
:109798004FF4805005E04FF4C069EEE7002E5FD02B
:1097A8000020A6F1030CBCF1010F04D86FF085036B
:1097B8001846BDE8F8830EB1042AF7D0B3F5805FE8
:1097C80053D0B3F5405F52D0002B0CBF01230323C5
:1097D8009942EBD149463FF0A9F88242E6D1EB79AC
:1097E80053B3012B45D1244B9C4225D003F1805320
:1097F8009C4221D0214B9C421ED003F180539C42B5
:109808001AD01F4B9C4217D003F180539C4213D0AF
:109818001C4B9C4210D003F180539C420CD01A4B35
:109828009C4209D0B4F1502F06D0184B9C4203D06B
:1098380003F180539C42B9D12368294623F00103E0
:10984800236038463FF0F4F903460028AED1226879
:1098580042F00102226095E8030088E80300A7E7C8
:109868004FF08050AAE73046A8E70023B0E702236C
:10987800AEE7032BB7D099E7003801400044004019
:1098880000480040004C00400050004000240046C2
:109898002DE9F04383B0D0F804908046D9F804004D
:1098A800D9F81010836800AF1B687BB1984705464C
:1098B80070B90021D9F824003A1D3EF0D1FF051EE9
:1098C8000EDA28460C37BD46BDE8F0836FF0570521
:1098D8000121644A64483CF023FB002DF1DBE8E7F2
:1098E8007B680022197918683EF0CCFF051EE8DB7A
:1098F800D8F80460D8F8103034681D68236823F05D
:1099080001032360B06840F011F838B90121574AC3
:1099180055483CF005FB6FF01205D2E7D6E9020185
:109928008368DB6803B1984754E8003F43F00C03B1
:1099380044E80032002AF7D1294640463FF078F93A
:10994800054610B16FF01505BBE7337E1BB1A36860
:1099580043F00803A360737E1BB1636843F40043BC
:109968006360B37E1BB1636843F480336360F37E46
:109978001BB1636843F400336360337F002B5AD014
:109988003B4B9C423CD003F180539C4238D0394B2E
:109998009C4235D003F180539C4231D0364B9C42D7
:1099A8002ED003F180539C422AD0344B9C4227D0BE
:1099B80003F180539C4223D0314B9C4220D0B4F118
:1099C800502F1DD02F4B9C421AD003F180539C423C
:1099D80016D06C4688B06A46D8F800302A49CDE9D6
:1099E80005134FF40073ADF81C30284B42F8103FB4
:1099F80000234FF4E2511C48F9F7D6F9A546A1E730
:109A0800D8F804301A68936843F480439360236855
:109A1800727F23F0787343EA425323602368B27F4E
:109A280023F4F81343EA02432360F37F1BB1A368CE
:109A380043F40043A36096F820301BB1236843F039
:109A480000532360236843F001032360E3699A020B
:109A5800FCD5E3695B02FCD54046D9F82830984725
:109A68002FE700BF112508089C3E07083125080884
:109A7800003801400044004000480040004C0040CD
:109A880000500040002400464C250808030000014F
:109A980070B50B68064698883FF0A6F904280C466E
:109AA800D1E91B15034610D002280AD1012A01D991
:109AB800012D0AD8328E92B209B105B10A80022569
:109AC80008E0032A12D9032D12D9326B09B105B166
:109AD8000A600425B5FBF3F5226F2AB1954213D924
:109AE800164917483FF0BCF9284670BD012A02D92B
:109AF800226F012ADED896F83020D2B201B10DB912
:109B08000125E9E70A70FBE7521B22677AB9A26DC3
:109B180004F15C010832A265E26D04F15800013AD3
:109B2800E26504F170023FF03BF9E066DCE7E26EC3
:109B3800002AD9D005FB0322E266D5E7A925080843
:109B48006C3E07082DE9F84306460C4604274FF0FB
:109B5800020891F87C90236898883FF045F904281A
:109B68000346626E17D002280FD1B9F1010F02D94E
:109B7800A16E01290FD8002A39D0A16E01B1118830
:109B880089B2B8FBF3F531840CE0B9F1030F1FD9A2
:109B9800A16E03291FD9CAB1A16E01B11168B7FB23
:109BA800F3F53162A26E2AB1AA4224D21F49204895
:109BB8003FF056F9636F5B1BA9EB050515F0FF092C
:109BC800636701D0002BC6D1BDE8F8831146E6E7EC
:109BD800B9F1010F02D9A16E0129CCD84AB1A16E01
:109BE80001B11178C9B2012586F82010DAE71146CB
:109BF800C6E71146F6E7521BA2667AB9226D04F150
:109C0800540108322265626D04F15000013A626520
:109C180004F168023FF0C4F86066CBE7626E002A80
:109C2800C8D005FB03226266C4E700BFA92508085F
:109C38006C3E070808B502B933B1044804493FF03F
:109C48000FF96FF0850008BD1846FCE76C3E070861
:109C5800C72508082DE9F047044600AF00693FF022
:109C68003FF9012160683FF026F9002802DA10F177
:109C7800860F15D165680021284626693FF01BF933
:109C8800041E0BDB3248A96883681B685BB19847E0
:109C9800044658B12F4930483FF0E2F804EAE4702E
:109CA800BD46BDE8F0876FF05704F3E74FF00108B1
:109CB800B5680835D6E9023203EBC203A5F10802FC
:109CC8009342EBD955F8080C3FF030FE034615F8DF
:109CD800041C55F8080CBBB96C468AB06A46006883
:109CE80007914FF400711D4DADF820101C49CDE9C6
:109CF800055042F8101F4FF411511748F9F754F85E
:109D0800A5466FF01204C9E735F8023CD0F810E018
:109D1800DA0754BF43F4B01383F4D013DEF800C05D
:109D280023F4801208FA01F9DB074CBF4CEA090357
:109D38002CEA0903D0F808A0CEF80030DAF8003091
:109D48009847002805F10805B4DA0446A6E700BFDD
:109D580088390708F52508086C3E07081026080802
:109D6800040000012DE9F04F87B080460E469B465F
:109D78009146056900AF32B92BB9002630461C3729
:109D8800BD46BDE8F08FB3889A0400F123814FF0F7
:109D9800FF324FF0FF3305F1100001F0E7FF6E606E
:109DA8000023C5E9113385F84C30D8F81030D8F8BD
:109DB80004A0FB601B68DAF800409E42B28840F0BD
:109DC8001581130508D5B9F1000F00F00C814FF487
:109DD800C12120463EF0D5FFB0883FF005F8034684
:109DE800B9F1000F40F07581C5F8509000226A65FE
:109DF80005F1540105F1680205F15000FB603EF0E1
:109E0800CFFFFB686866BBF1000F40F06B81C5F8B7
:109E180058B00022EA6505F15C0105F1700205F110
:109E280058003EF0BDFF00210B46E866686D2964C6
:109E3800834240F0608100231A46D5F85CC0624531
:109E480040F0608199422CBF29662B66AB6E3BB906
:109E58002B6F2BB96B6F1BB9AB6F002B00F03F82D8
:109E680023687B60E3683B60D8F80430BB601B68FC
:109E7800FB60FA681B68D26803F4006302F4C0222E
:109E8800134340F04681494630463EF0C7FF5946E5
:109E9800814630463EF0C2FF81454E46B8BF064671
:109EA800002EC0F2B580BB681B6AB342C0F03B818C
:109EB800FB68D8F810101B68DB0702D5F8683EF07D
:109EC80085FFFB68FA685B686FF30F0333435360E1
:109ED800C1E91D66D8F804301B681A6842F001020F
:109EE8001A60DA68500200F12581D8F810603068ED
:109EF800002840F028817B6803F400693B6803F47C
:109F0800C02349EA0309AB6E2BB92B6F1BB96B6FE2
:109F18000BB9AE6F3EB3294620463FF003F863699C
:109F280013F4787300F01C816E468AB06A46934930
:109F380005919349CDE906134FF40073ADF820302D
:109F4800904B42F8103F00234FF411518E48F8F718
:109F58002BFF6369B5465A0603D5A36943F040034E
:109F6800A3616FF00406D8F80430D8F810901C6884
:109F78006369D90700F15F81E3685A0240F1728191
:109F8800824920463EF03BFF002800F057812368B5
:109F9800D80740F1538163689BB26BB9D9F8003098
:109FA8009B88C3F34513192B06D821FA03F3DB0763
:109FB80002D520463EF00AFF2368E26803F40063F6
:109FC80002F4C0221343B3F5C02FDAD120463EF085
:109FD800FDFED6E7AB69002B7FF4D9AE6B689E42D5
:109FE8007FF4D5AEDCE64FF4C021F2E6DAF81010C3
:109FF800C2F34513022918D0032919D0012931D1F8
:10A00800043B1C2B8CBF00230123ABB96FF08506E2
:10A0180095F84C3013B1002E3FF4AFAE00236B60BF
:10A0280005F1100001F066FEA8E6043B0C2BE9E7F9
:10A03800082B01D0102BE9D1100448BFE36854481D
:10A0480042BF23F4601343F40023E3608368DAF823
:10A058000810DB685BB94F494B483EF001FF6FF0D1
:10A068000406D5E74C4948483EF0FAFECEE707F12A
:10A07800140298470028EEDB00217B69306823FA38
:10A0880001F2824240F22D8101310929F7D16C4653
:10A098008AB06A4607931B0A089305233F49CDE90E
:10A0A800051042F8103F00234FF421513648F8F7C5
:10A0B8007BFEA5463BE04FF4C02143E11BB1E368BA
:10A0C80023F0105366E1E36823F0105343F0005384
:10A0D80060E1D9F800202A65002A3FF487AED9F854
:10A0E800042084E6DBF80020AA65002A3FF491AE3C
:10A0F800DBF804208EE62A6D02EBC30252680133B6
:10A10800114495E6A86D00EBC20040680132034493
:10A1180095E6B3F5C12F30460CBF494659463EF087
:10A128007DFE0646BCE61E4917483EF099FE6FF0D4
:10A1380015066DE71A6842F400721A601A689105EC
:10A148003FF5D3AEFAE7037D002B3FF4D4AE0121EF
:10A1580008303EF09DFE336818693FF0C1FBCAE63F
:10A16800B9F5C12F7FF4CFAEAB6EDBB10021226809
:10A17800E36800295CD102F40069C0E6B426080847
:10A18800906A0808040000016C3E070800020202F9
:10A19800883907085C26080834260808BF260808F6
:10A1A800882608082B6F002BE0D0DAF800603046CC
:10A1B8003EF025FE01460028F9D130463EF006FE65
:10A1C8002B689888C30712D40B46D5F85CC0634542
:10A1D80024D13EF009FE91FBF0F300FB131323BBDF
:10A1E800B1FBF0F173686FF30F03194371604FF41B
:10A1F800C02130463EF0C5FD336843F001033360AB
:10A20800F3685A02B2D5336843F400733360336895
:10A218009B05ABD473691807A8D4F8E7AA6D02EBBD
:10A22800C302526801331144D1E76FF015019EE76C
:10A238006FF0150697E694F8303099E6D8F810A034
:10A24800DAF8003073B11A7D62B1998811F4805B35
:10A2580008D118693FF044FBDAF800005946083085
:10A268003EF016FE6369990542BFA36943F4007383
:10A27800A361A36943F01003A361A36943F04003FA
:10A28800A361A36943F00803A36163686FF30F0335
:10A298006360D9F800309B88DA0402D420463EF087
:10A2A80095FD99F84C3033B9C9F8406009F1280098
:10A2B80001F020FDACE6D9F8443023B131464046E0
:10A2C800D9F848209847D9F800309B8813F40053F0
:10A2D8007FF49EAEC9F8043009F11000E8E71E4685
:10A2E80096E620463EF072FD4B4AA36852F82120BC
:10A2F80023F070431343A3609AF82530DB0703D596
:10A30800E36843F40043E360B38813F0020FE368A3
:10A3180014BF43F0007323F00073E360B38813F0B5
:10A32800040FE36814BF43F0807323F08073E36085
:10A33800B18811F4006105D0B9F1000F3FF4BBAE4C
:10A348004FF4C12120463EF01CFDB38813F0100FD6
:10A35800E36814BF43F4000323F40003E360A36835
:10A3680023F48003A360B388327D03F0010322B98C
:10A378009AF8252091077FF5A1AE33B9E368DA0092
:10A388005EBF236843F480532360E36823F01053CF
:10A3980043F08063E360B388204913F0010FE3685A
:10A3A80014BF23F4800343F48003E360B288A368F6
:10A3B800C2F34512043A51F8222023F01F03134335
:10A3C800A360E368DAF81C2023F00F031343E3606B
:10A3D800E368DAF8182023F0F00343EA0213E36095
:10A3E800B288DAF81430C2F345120732D20893FB68
:10A3F800F2F3012BB8BF0123FA68094982F87C30CF
:10A40800DBB2A268013B51F8233022F4F072134307
:10A41800A360FB681E60DFE404470708BC47070821
:10A428007C4707084FF0E02310B599691C699B69C0
:10A4380000B103600B4A0C481268002908BF114696
:10A44800002B08BF134614F4803F01D1994205D26E
:10A458000168114401604FF0E02109690068104467
:10A46800C01A10BD983B00208C3B002010220B4BDB
:10A47800002083F823204FF4C862094B1A604FF478
:10A488007A52084B1A60084B43F67F6218604FF007
:10A49800E0235A61072298611A61704700ED00E0D5
:10A4A800943B0020983B00208C3B0020684620F01D
:10A4B80007018D46F1B53EF077FD04460020FFF711
:10A4C800B1FF1348134A0368D2E900515B1941F1FF
:10A4D8000001C2E9003100274FF47A520E4D07609F
:10A4E800D5E900619B1BB3FBF2F002FB00F39B195B
:10A4F80041F10001C5E90031084B21461F6002F017
:10A50800A7FBF9F75BFCBDE8F1408546704700BF43
:10A518008C3B00208830002080300020903B0020B9
:10A528002DE9F341804601A8FFF77CFF0027284961
:10A53800284AD1E90034C318274844F100041760B9
:10A54800D0E90020B3EB020CC1E90034234E64EBE0
:10A558000004234BBC42356818681ADB4FF47A5E56
:10A56800204B1B6813EB0803A3FB0E3247EB0708CD
:10A578000EFB0822B3EB0C0362EB040298429741EE
:10A5880007DAB3F1807F72F10002A8BF6FF07F4352
:10A5980018464FF0E0230022306001389C6958616A
:10A5A8009A61114A536803F0807343F00073536053
:10A5B800019BD1E90020A34238BF5B191B1B9A18E5
:10A5C80040F10000C1E9002002B0BDE8F08100BF01
:10A5D800883000208C3B002080300020983B0020F1
:10A5E800943B0020903B002000ED00E010B5084BA4
:10A5F80000201C68074B1B68E41AFFF713FF4FF491
:10A608007A532044B0FBF3F0034B186010BD00BF31
:10A618008830002080300020903B002038B53EF084
:10A62800C3FC064B044600201D68FFF7FBFE84F3BD
:10A638001188BFF36F8F284438BD00BF88300020D1
:10A6480030B53C4AD369916A13F00C0305D00C2B42
:10A658003FD101F0030101293BD19168090254BFA0
:10A66800D2F8F4209268344954BFC2F30332120F6F
:10A6780051F82200002B5AD02E49B7EE006A8C6A96
:10A688008B6A8D6AC3F303238A6B013307EE903A12
:10A69800C2F3CC03C5F30012534306EE903A04F01C
:10A6A8000304022CB8EEE77AFAEEE96A1FD0032C0D
:10A6B8001DD04B6BC3F3080307EE903AF8EEE77A28
:10A6C80077EEA67A06EE900A77EE867AB8EE666A94
:10A6D8001AE0D26902F00C02042A06D0082B27D00F
:10A6E80000200C2B23D10020C6E71448F9E74B6B58
:10A6F800C3F3080307EE903AF8EEE77A77EEA67A06
:10A7080077EE867A9FED0E6A0A4BC6EE076A5B6B98
:10A7180067EEA67AC3F30663013307EE103AB8EE84
:10A72800C77AC7EE876AFCEEE67A17EE900A30BD64
:10A738000248FCE7000C0246304807080024F400F1
:10A748000024744B08B5FFF77BFF054B054A1B6ACD
:10A7580003F00F03D35CD840034B186008BD00BF5B
:10A76800000C0246A26A0808C8060020F7B504468D
:10A7780010B390F89534056803F0FF021BB980F810
:10A7880094243EF020FC032384F89534324B20684F
:10A798009D4204BF0023A3713EF029FE237C251DA2
:10A7A8008DF8003095E80E0020683EF0DCFD01468B
:10A7B80030B1022384F895340125284603B0F0BD52
:10A7C80020683EF01AFE0028F3D1012702462679B8
:10A7D80004F11403C1B28E4203F1240321D80021ED
:10A7E8000A4604F51573C8B2864203F1240326D835
:10A7F800237C8DF8003095E80E00206800F00AFCF4
:10A8080005460028D5D10123607484F89534237B4C
:10A81800012B02D120463EF092FD20683EF0F6FF63
:10A82800CBE723F80A0C43E9072203F8237C03F853
:10A83800241C03F8202C43F8142C0130CAE743E900
:10A84800072203F8232C03F8240C03F8202C43F8E0
:10A85800142C0131C7E700BF000004422DE9F04F76
:10A86800066889B0044630463FF00CF8039000288B
:10A8780040F06F8120683EF0D7FF002800F0698122
:10A88800D6F808382068C3F30D23C4F8D4343EF052
:10A89800CBFF870748BF226806F5006542BF5369AA
:10A8A80003F00203536120683EF0BEFFC0062DD5B9
:10A8B8002268936923F010039361D6F8208008F486
:10A8C800F013B3F5802F08F00F0740F0458147F6E5
:10A8D800F07318EA030F14D0242303FB0747C8F3C7
:10A8E8000A194A463046D7F860123EF02EFFD7F8CC
:10A8F80060324B44C7F86032D7F868324B44C7F827
:10A9080068322268936943F01003936120683EF02F
:10A918008BFF010300F1338120683EF085FF42037D
:10A928000CD520683EF08CFF27464FF0000A0490B3
:10A9380006F5106B049B002B40F0EB8120683EF07D
:10A9480073FF002813DA6B6823F001036B6094F837
:10A95800CC34012B40F085820021204684F8CC14A9
:10A968003EF000FD2268536903F0004353612068FC
:10A978003EF05AFF03050AD5AB68DF0702D520462B
:10A988003DF099FB2268536903F400635361206822
:10A998003EF04AFF000115D52268536903F00063B1
:10A9A800536194F8CC34002B40F05F820121236876
:10A9B80084F8CC145B6D2046C3F38303C4F8D03409
:10A9C8003EF0D0FC20683EF02FFFC10433D56B6801
:10A9D800102123F001036B6020683EF03CFD4FF628
:10A9E8007F3106F5106322790398824200F2418292
:10A9F800EB6943F00113EB61E37B002B00F0568217
:10AA0800D5F8843043F00B03C5F884306B6C43F001
:10AA18000B036B64D6F8003804F29C4223F4FE63FF
:10AA2800C6F80038A179206800F0E4FC2268536970
:10AA380003F48053536120683EF0F6FE820416D575
:10AA480020683EF023FF20683EF050FDE071276843
:10AA5800FFF778FEE2790146384600F06BFA2046A7
:10AA68003DF0F1FA2268536903F4005353612068FA
:10AA78003EF0DAFE030707D520463DF03AFB226890
:10AA8800536903F00803536120683EF0CDFE0706C2
:10AA980000F1178220683EF0C7FEC0020CD5A04620
:10AAA800012706F512692379BB4200F22882226841
:10AAB800536903F48013536120683EF0B5FE8102A8
:10AAC8002AD523464FF0010C06F5326120796045FE
:10AAD8001DD993F87C720868012F40F0268200285F
:10AAE80080F22382D4F8D42482EA1040C20700F10D
:10AAF8001C8283F87B72B06940F08000B061706995
:10AB0800000600F112826B6843F400736B602268E0
:10AB1800536903F40013536120683EF085FE410039
:10AB280007D520463DF0BBFA2268536903F08043FD
:10AB3800536120683EF078FE42070AD523685D68B5
:10AB48006B0702D520463DF0B0FA226853682B43C4
:10AB5800536009B0BDE8F08FB3F5402F7FF4D1AE54
:10AB68000822304604F29C413EF0EFFD242303FB0B
:10AB78000747D7F86832C8F30A184344BFE6206885
:10AB88003EF056FEA2460027049006F53068049B66
:10AB9800002B3FF4C1AE049BDB0779D55FFA87FB36
:10ABA800594620683EF054FE10F0010F81461FD030
:10ABB8000123C8F80830206894F806C000F530630F
:10ABC80003EB4713BCF1010F016C9A6840F08B80CE
:10ABD80012F0080F07D0B348814209D9120407D5EB
:10ABE8004FF4004203E012F0200F5AD020229A605E
:10ABF80019F0080F21D00823C8F808302368A9499C
:10AC08001A6C03F5306303EB47138A42986804D93A
:10AC1800000444BF4FF40040986020460592FDF7B9
:10AC28008DFA059A9F498A4207D9A179012904D149
:10AC3800206804F29C4200F0DDFB19F0100F1CBFE5
:10AC48001023C8F8083019F0020F14D073691906D8
:10AC580042BF6B6843F480636B609AF85732012BEC
:10AC680006D10023594620468AF857323EF000FAAA
:10AC78000223C8F8083019F0200F1CBF2023C8F899
:10AC8800083019F4005F1CBF4FF40053C8F80830AF
:10AC9800049B01375B08049308F120080AF1240A91
:10ACA80075E7DFF800C2614501D9120498D41A6922
:10ACB800DAF87432C2F312029B1ACAF868326FB912
:10ACC800D4F864222AB9012104F29C4200F092FBD4
:10ACD80004E0D4F860221A44C4F860225946204699
:10ACE800FDF7F2F984E7DFF8C0C1614507D1110427
:10ACF8003FF576AF9206F1D520229A60EEE7002F55
:10AD0800ECD1D4F86432002BE8D1394604F29C42E5
:10AD1800DCE7049BDA0740F19B805FFA8AF3194667
:10AD2800206807933EF09DFD10F0010F804620D06B
:10AD380001216B6B0AF00F0201FA02F223EA020307
:10AD48006B63CBF80810A17901290DD1D7E9072346
:10AD580013443B62BAF1000F06D1636A23B9206835
:10AD680004F29C4200F046FB20465FFA8AF1FDF7A8
:10AD7800C9F918F0080F1CBF0823CBF8083018F0E1
:10AD8800100F1CBF1023CBF8083018F0400F1CBF61
:10AD98004023CBF8083018F0020F10D05146304647
:10ADA8003EF059FBFB7D012B06D100232046FB75A5
:10ADB8005FFA8AF13EF05DF90223CBF8083018F00B
:10ADC800800F45D0D7E909329A4241D8A3EB02084F
:10ADD800FB692168984528BF984601F5106308F17A
:10ADE800030803EB4A1305914FEA98080693069B5C
:10ADF8009969D7E9093289B2414527D393420BD8DB
:10AE08000121059B0AF00F00D3F83428814022EA7B
:10AE18000102C3F834281BE0A3EB0209FB69079A77
:10AE2800994528BF9946A37905980093396A1FFA6E
:10AE380089F33EF077FC3B6A09F103084B443B6217
:10AE4800BB6A4FEA98084B44BB62D0E79342D7D914
:10AE5800049B0AF1010A5B08049324370BF1200BC9
:10AE680068E520463DF036F97CE520463DF023F9BB
:10AE7800A8E599601A68203322F4001243F8202CC0
:10AE8800C3F8E811D3F8E02122F40012C3F8E02156
:10AE9800D3F8E02142F00062C3F8E021039A0132BE
:10AEA8000392A0E50A30544F0A31544F6B6943F4BA
:10AEB800005343F02B036B612B6943F00B032B61A9
:10AEC800A8E501222427B36904F2572023F0800360
:10AED800B36106F53263217991427FF6DBAD07FB5A
:10AEE80002F1415C012907D1196841F0006119603C
:10AEF800196841F08041196001322033EBE798F876
:10AF08003C30D9F80020012B09D1002A07DA67F074
:10AF18007F01204688F83B30C9B23EF0C0F90137BE
:10AF280008F1240809F12009BDE50CF1010C2433CE
:10AF38002031CBE5022A4AD1274B284A0B449342B9
:10AF480039D9274B274A0B44934236D9264AA1F5CB
:10AF58007403A3F51053934231D9244AA1F18373A2
:10AF6800A3F5E74393422CD3214B224A0B44934247
:10AF780029D9214B214A0B44934226D3204B214AFD
:10AF88000B44934223D3204AA1F1B773A3F5585336
:10AF980093421ED31D4B1E4A0B4493422CBF0623DB
:10AFA8000723C26822F47052C260C26842EA83234F
:10AFB800C360002070470F23F3E70E23F1E70D234A
:10AFC800EFE70C23EDE70B23EBE70A23E9E7092377
:10AFD800E7E70823E5E700BF405327FFFF340C00ED
:10AFE800401E1BFF3F420F007F4F120020D6130068
:10AFF80060B6E5FE5FE3160000D3CEFE40771B0087
:10B00800C05BB3FEC091210020753800E05459FEA2
:10B01800E09C410084B02DE9F843044609A880E883
:10B028000E00002319469DF824809DF82E7003F128
:10B038004002013304EB82020F2B5160F7D104F573
:10B048000066002F64D1736843F002037360A36B3A
:10B0580023F40013A363236843F0400323602368A9
:10B0680043F080032360002503212046C4F8005ED6
:10B078003EF035FA102120463EF0EDF90146204613
:10B088003EF00CFA0843C0B2401B18BF01202A4604
:10B098004FF090414FF0006C4FF67F3E356104F55C
:10B0A80010637561F561A84537D800224FF09045C7
:10B0B80011464FF0006C4FF67F3E04F53063904523
:10B0C8003DD8336923F4807333610023A3616FF0A3
:10B0D800804363619DF826301BB9A36943F01003D0
:10B0E800A361A2691F4B1343A3619DF82A301BB1CA
:10B0F800A36943F00803A361012F01BFA36943F0CB
:10B10800804343F00403A361BDE8F84304B07047EB
:10B11800A36B43F40013A363A5E7D3F80090B9F138
:10B12800000F0ADA3DB9C3F800C01A610135C3F847
:10B1380008E02033B7E71960F7E71A60F5E7D3F8B6
:10B148000090B9F1000F0ADA3AB9C3F800C01961E2
:10B158000132C3F808E02033B1E71D60F7E7196052
:10B16800F5E700BF00383C8030B54A780B78012AF3
:10B1780000EB431300F5006029D1D3F80029002A19
:10B188000BDAD3F8002942F00062C3F80029D3F89B
:10B19800002942F08042C3F8002901240A78C56BCF
:10B1A80002F00F0204FA02F225EA0202C2630978E9
:10B1B800C26901F00F018C4022EA0402C261D3F88F
:10B1C8000019174A0A40C3F80029002030BDD3F8F7
:10B1D800002B002A0BDAD3F8002B42F00062C3F8E8
:10B1E800002BD3F8002B42F08042C3F8002B012437
:10B1F8000A78C56B02F00F0204FA02F225EA02424D
:10B20800C2630978C26901F00F018C4022EA044246
:10B21800C261D3F8001B034A0A40C3F8002BD4E7E5
:10B22800007833EC0078F3EFF7B54B7891F800C06D
:10B23800012B6D4D6D4E00EB4C1440F089800F6969
:10B2480004F510633FBB1F693D401D611D6945F44E
:10B2580000251D611D693540012A1D614DD1CA694E
:10B2680002B15A610B79012B0CD1D0F8083813F4CC
:10B27800807FD4F800390CBF43F0005343F080536B
:10B28800C4F80039D4F8003943F00443C4F800394D
:10B29800002003B0F0BD1F693E401E611E693540A5
:10B2A8001D610D698E68BCF1000F0CD1B54288BFD5
:10B2B8000E611D6945F400251D610D691E69C5F300
:10B2C80012053543C8E73544013DB5FBF6F5484F4F
:10B2D800D3F810C0AEB207EAC54545EA0C051D61B2
:10B2E8000D79012DE9D11D6925F0C0451D611F6942
:10B2F800750705F0C0453D43DEE7D4F8003943F053
:10B308000443C4F800390B79012B0DD00B69002BCD
:10B31800BED001230A78D0F8344802F00F029340D7
:10B328002343C0F83438B3E7D0F8083813F4807FE3
:10B33800D4F800390CBF43F0005343F08053C4F8ED
:10B34800003900920B8A0A78C9683EF0EBF99FE74A
:10B35800D4F8107B04F530633E401E611E69354009
:10B368001D610E698D68BCF1000F27D106B10D6112
:10B378000D621E69C5F3120535431D611D6945F44B
:10B388000025012A1D6102D1CA6802B15A610B79F0
:10B39800012B0CD1D0F8083813F4807FD4F8003B87
:10B3A8000CBF43F0005343F08053C4F8003BD4F87B
:10B3B800003B43F00443C4F8003B69E7002ED8D0B3
:10B3C8002E44013EB6FBF5F6B6B275430D62084D44
:10B3D8001F6905EAC6453D431D610D6A1E69C5F32F
:10B3E80012053543CDE700BFFFFF07E00000F8FF77
:10B3F8000000F81F30B5114C056C00F53063A5420C
:10B4080003D9D0F8004B002C16DB00241C611C6902
:10B41800012944F400241C611C6944F018041C61CF
:10B428001C6944F0C0441C6101BF5A61D0F8003B5C
:10B4380043F08023C0F8003B002030BD0A30544F51
:10B44800A8B1304BDA6802F44032B2F5403F10D16F
:10B458002D4B984250D92D4B98424FD92C4B98429E
:10B4680035D92C4B984216D92B4B984231D901200B
:10B478007047DA6802F44032B2F5003F0DD1274B2D
:10B48800984239D9264B984238D9264B98421ED92A
:10B49800254B9842EBD803231CE0DB6803F44033C8
:10B4A800B3F5803F0AD1214B984225D91B4B9842CE
:10B4B80024D91F4B98420AD9194BEAE71D4B9842E9
:10B4C8001AD91D4B984219D91C4B9842CFD8022340
:10B4D80000E004231A490A6822F00F021A430A609E
:10B4E8000A6802F00F0293420AD0086800F00F00C1
:10B4F800C01A18BF012070470023EBE70123E9E7D2
:10B5080000207047000802460048E8010090D00378
:10B5180000D8B8050020A1070068890940787D0196
:10B5280080F0FA02C068780400E1F50520BCBE008E
:10B5380060343C0200127A000024F40000366E01E8
:10B548000020024010B50446F7F760FB03480121CC
:10B55800034A3AF0E5FC20463EF0F3F94C3E070872
:10B56800052708082DE9F84304460D4600AFEFF318
:10B578001188102383F31288BFF36F8F04282A4A97
:10B5880098BF2A4BE9468AB09668117C98BF53F851
:10B5980020306A4688BF264BCDE9073140F2013397
:10B5A8002448ADF82430244BCDE9050442F8103F77
:10B5B80000234FF431512148F7F7F6FBCD4645B14A
:10B5C800EB69C3F3080323B101211D4A1B483AF074
:10B5D800A7FC2EB130463EF063FC08B1037803B9EE
:10B5E8001848E9468AB06A46174B0790CDE90536F0
:10B5F80040F20133ADF82030144B42F8103F0023DD
:10B608004FF411510D48F7F7CFFB2946CD46204698
:10B61800FFF798FF88F31188BFF36F8F3046F8F76C
:10B62800DDFBBD46BDE8F8839C3B00207048070859
:10B63800152708082B270808050000014C3E0708B5
:10B64800532708082327080874270808040000015E
:10B6580038B50A4B53F82040013053F82050A54222
:10B6680000D838BD606830B1037EDB0701D43EF0F6
:10B6780045F90834F3E723689847FAE78448070848
:10B68800012270B52C4B2D4C2D4D86B01A70AC4252
:10B698001CD30320FFF7DCFF0420FFF7D9FF294C58
:10B6A800294D2646AE4204F1300413D301F0D4F8F4
:10B6B800244CAC422AD301F0E3F839F028FB234AA2
:10B6C800938923F00103938106B070BD54F8043BBD
:10B6D8009847DCE754F80C3C059354F8103C049365
:10B6E80054F8143C039354F8183C029354F81C3C47
:10B6F800019354F8203C009354E90A2354E90C01BF
:10B70800F5F77EFD54F8303C5E65CAE7D4E90A23B4
:10B71800B3F1FF3F08BFB2F1FF3F05D052EA030182
:10B72800206803D100F078FD3034C2E708491830AA
:10B7380001F0A6F9F8E700BF824900202C3C070871
:10B74800303C0708303C0708603C0708703100208F
:10B75800C79F0508E02370B5134E012203FB00665E
:10B76800002386B0CDE904230F220193CDE90232EC
:10B7780018234FF4A0720D4D0D4903FB00550446E4
:10B7880002FB00110B4B30460095F5F739FD337C71
:10B798002C7423F004033374074B013403EBC423E4
:10B7A800EE606B6006B070BD903000209C3B0020BE
:10B7B80000690020DD9A0508006100207FB500209F
:10B7C800FFF746FF2D4B03F5006282F3088883F3E9
:10B7D8000A88F0232A4C2B4D84F822300023E37783
:10B7E80023766376A37684F82030636A43F4E023F3
:10B7F8006362F8F79DF9F8F7DBFA4FF0FF33A362BD
:10B80800E362F8F7F3FCF8F775FBF7F761F91E4800
:10B8180000F0DEFCF7F712F81C4CAC422AD30120EA
:10B82800FFF716FF02201A4CFFF712FF01F00CF881
:10B83800184B00259C61184B45F6E06205930123DF
:10B848001649CDE903532046154BCDE9015500951E
:10B85800F5F7D6FC0646237C204623F00403237420
:10B868003EF053FB2846FFF775FF314620460C4A49
:10B87800F8F770FA54F8043B9847CEE700610020C7
:10B8880000ED00E02C3C070850320020283C070857
:10B89800703100209C3B00204C0B0808406A0020B7
:10B8A80089B6010838B5064C064DAC4201D30020D4
:10B8B80038BD2046D4E901123EF08DF81434F4E77F
:10B8C800CC100020E010002030B5054B85B0DDE934
:10B8D80008450293CDE900453EF03BF805B030BD80
:10B8E8008350050838B5064C064DAC4200D338BD28
:10B8F80020463EF095F80028F9D11C34F5E700BF42
:10B90800B0100020CC10002073B50C46EFF3118165
:10B91800102585F31288BFF36F8FC5685DB1256068
:10B928002B68C360836901338361002081F3118828
:10B93800BFF36F8F11E052EA030603D16FF00B00DB
:10B948002560F3E7CDE900230246083000F088FEC1
:10B9580018B9034B9B685B69236002B070BD00BFD8
:10B968009C3B0020F7B50E4604469DF82010EFF3E7
:10B978001187102080F31288BFF36F8F256AE06863
:10B98800854245D22568AC4219D0C5B128463EF05B
:10B99800ACF805F1180001F003F93146A2686869AE
:10B9A80057F08EFC00232846C5F8983000F0D4FCE8
:10B9B80004F10800394600F0DBFD002036E0A268FB
:10B9C800D9B13146E06957F07BFCE369A2681344BA
:10B9D8006269E361934201D12369E361236A10211B
:10B9E8000133236204F124003EF050FC0028DFD12B
:10B9F80087F31188BFF36F8F18E0A0692369314678
:10BA0800984208BF6069801AA06157F059FCE5E7C1
:10BA180052EA03010CD0084904F1080089684E6114
:10BA2800CDE900233946224600F01AFE03B0F0BDE6
:10BA38006FF02200DCE700BF9C3B0020F7B504460E
:10BA48000846EFF31186102181F31288BFF36F8F38
:10BA5800216A00293BD0A268A16957F031FCA3698B
:10BA6800A268256813446269A361934204BF2369ED
:10BA7800A361236AAC4203F1FF33236236D0284620
:10BA8800002D34D000273EF030F805F1180001F001
:10BA980087F86969A268E06957F012FCE369A2684F
:10BAA800284613446269E361934204BF2369E36152
:10BAB800236A01332362C5F8987000F04DFC04F145
:10BAC8000800314600F054FD384603B0F0BD52EA94
:10BAD800030111D00A4989684861CDE9002331463C
:10BAE800224604F1080000F0BBFDEEE7002086F3D3
:10BAF8001188BFF36F8FE8E76FF02200F7E700BF08
:10BB08009C3B00202DE9F341044617461E46EFF3FF
:10BB18001188102383F31288BFF36F8F304BC268EC
:10BB28009B6872B18068984217D057EA060216D10E
:10BB380088F31188BFF36F8F6FF00F0002B0BDE874
:10BB4800F08193F90E1001322161C4E9023288F3C1
:10BB58001188BFF36F8F0020F0E72169F3E793F9AD
:10BB68000E1090F90E30994230DA9942A8BF194662
:10BB78003EF013F8054622464146CDE900761948BD
:10BB880000F06EFD0028E6D0EFF31186102383F352
:10BB98001288BFF36F8FA068D0B1236821699C42D7
:10BBA8000AD04BB193F90E309942A8BF19466FF0ED
:10BBB8007F039942B8BF19463DF0EFFF40B13146C7
:10BBC800084800F0D5FC6FF00A00B7E70025D2E777
:10BBD800002DF4D186F31188BFF36F8FF3E700BF10
:10BBE8009C3B002083490020F8B583680546002B5C
:10BBF80040D0234A926893423FD1C368012B03D9AE
:10BC0800013BC3600020F8BDEFF31187102383F3D5
:10BC18001288BFF36F8F016980683DF0BEFF2C6802
:10BC2800A54207D10023C5E9023387F31188BFF382
:10BC38006F8FE7E7002CF5D0D4E9003200261360B7
:10BC48005A60237CC4E9006623F002032374A660CB
:10BC580004F1180000F0A4FFAC6094F90E302046FF
:10BC68002B61C4F8986000F077FB3946054800F06E
:10BC78007FFCC7E76FF01500C5E74FF0FF30C2E75C
:10BC88009C3B00208349002073B51546EFF31186CD
:10BC9800102282F31288BFF36F8F0468B4B123684F
:10BCA800426823F00303944208BF4360036023689B
:10BCB8009B0704D0656820463EF014FB2C4686F3AB
:10BCC8001188BFF36F8F204602B070BD55EA03029A
:10BCD800F5D000F1080231461046CDE9005300F0D6
:10BCE800BFFC0028EFD1024B9B685C69EBE700BF03
:10BCF8009C3B002070B5EFF31186102383F3128864
:10BD0800BFF36F8F0468A0421CD0DCB1D4E90032C5
:10BD1800002513605A60237CC4E9005523F0020310
:10BD28002374A56004F1180000F03AFF2046C4F817
:10BD38009850656100F010FB3146BDE870400A4834
:10BD480000F016BCD0E902329A4218BF0133022132
:10BD5800836010303EF09AFA0028EDD186F31188FE
:10BD6800BFF36F8F70BD00BF8349002013B5EFF399
:10BD78001181102484F31288BFF36F8F846844B153
:10BD8800013C846081F31188BFF36F8F002002B0FB
:10BD980010BD52EA030406D181F31188BFF36F8FF7
:10BDA8006FF00F00F3E7CDE900230246014800F0E9
:10BDB80057FCECE783490020F8B50546EFF31187F7
:10BDC800102383F31288BFF36F8F00262C68A542D7
:10BDD8001AD0CCB1D4E90032002613605A60237C13
:10BDE800C4E9006623F002032374A66004F1180076
:10BDF80000F0D6FE6FF00A0366612046C4F898305A
:10BE080000F0AAFA0126E1E700230221AB6005F160
:10BE180010003EF03BFA28B926B987F31188BFF322
:10BE28006F8FF8BD3946BDE8F840014800F0A0BB67
:10BE3800834900202DE9F04F04464FF0FF3A4FF0B8
:10BE4800FF3B614E85B0EFF31187102383F312880F
:10BE5800BFF36F8FD4F8E4505DBB022104F1FC00FE
:10BE68003DF075FF00287FD004F1F409D4F8F450B0
:10BE78004D4500F08680002D00F08380D5E9003222
:10BE88004FF0000813605A602B7CC5E9008823F046
:10BE980002032B74C5F8088005F1180000F080FE35
:10BEA80001232846C5F89830C5F8148000F054FAE4
:10BEB800DCE7D4F8E8202B689542C4F8E43008BFE2
:10BEC800C4F8E830D4F8FC3043F00203C4F8FC307E
:10BED800EB6823F0040343F00103EB606B6887F31E
:10BEE8001188BFF36F8F28469847EFF31187102307
:10BEF80083F31288BFF36F8FEB68D80623F0010233
:10BF08004AD4EA60EB689A0717D5306823F0020331
:10BF1800EB6090B10022036878B141688D4249D145
:10BF28000368002A40D172683360904200D1736080
:10BF3800002340F8083BFFF7DDFED4F8FC3023F07F
:10BF48000203C4F8FC30DB053CD4D4F8E430003BF1
:10BF580018BF012387F31188BFF36F8F002B3FF4BD
:10BF680072AF3DF0BEFF6EE7D4F8FC30D90608D5B5
:10BF7800C4F8FC0087F31188BFF36F8F05B0BDE8E4
:10BF8800F08F00233946CDE900AB029304F1EC02AF
:10BF98000E4800F08BFC56E723F01103EB6005F127
:10BFA8001000FFF7A7FEADE713607368984208BF5B
:10BFB8007260BDE702461BB1196818460B46ABE72D
:10BFC8001946FAE70023C5E7C43B0020834900204F
:10BFD800F8B5C36804469A070E46C3F3400542D431
:10BFE8005F0742D40B680BB983680B60E368D80716
:10BFF80042BFA36802253360376858BF012557B38D
:10C008001B4B9A68D7F8E0309A421ED13DF03FFFAB
:10C0180080F00100C0B2D7F8FC30D907C3F3800222
:10C028001CD5F2B1F8B100232360D7F8E83073B912
:10C03800C7E9394438463DF0B4FEE36843F00403E9
:10C04800E3603368A3602846F8BD0020E3E71C607E
:10C05800C7F8E840EEE76FF0150506E06FF0120547
:10C0680003E01B07DFD56FF00F0500233360EAE715
:10C078009C3B0020014601483DF0EDBE50330020B6
:10C08800F0B50446002089B00E9DC4E9390004F1DA
:10C09800EC00C4E93B0004F1F400C4E93D0055B3E9
:10C0A8002879002840F2011008BF0120C4F8FC00DC
:10C0B80000204FF0FF364FF0FF37CDE90330CDE9D0
:10C0C8000100CDE9066720460C4B009400F0C8F843
:10C0D80055B1296811B120463DF0DFFE6B791BB1DF
:10C0E800A38943F00103A381204600F095F8C4F822
:10C0F800E04009B0F0BD0120D8E700BF3DBE01080F
:10C1080037B501900846EFF31184102181F31288A6
:10C11800BFF36F8FC16811F01E0F16D153EA0205E5
:10C1280008D101A9FFF754FF84F31188BFF36F8F7B
:10C1380003B030BD41F00801C16001991030816140
:10C14800034900F09DFC0120EEE70020ECE700BF6A
:10C15800EB9D050801460148FFF7D2BF5033002088
:10C16800F0B585B00C4617461D460190EFF31183D4
:10C17800102181F31288BFF36F8F204603A9039320
:10C188003DF0F0FD55EA0703039E09D1204601A9B9
:10C19800FFF71EFF86F31188BFF36F8F05B0F0BD60
:10C1A800E3683A4643F00803E360019B0449A3624D
:10C1B80004F110002B4600F063FC0120EAE700BF01
:10C1C800EB9D050801460148FFF7CABF5033002020
:10C1D8000123037483810023C0E92033C0F88C3025
:10C1E800014B9860704700BF9C3B002008B500F0E9
:10C1F80069FA70B1074B9B68DB7B53B9EFF3118089
:10C20800102383F31288BFF36F8FBDE8084000F056
:10C21800C5BA08BD9C3B002038B50446EFF311852C
:10C22800102383F31288BFF36F8F037C5B070FD54E
:10C23800183000F0B5FC237C204623F00403237457
:10C2480000F08AF82946BDE83840044800F090B963
:10C2580085F31188BFF36F8F38BD00BF8349002075
:10C26800F0B5002587B00595109DDDE91276049597
:10C278000F9D044603950E9D02950D9D01950C9DFD
:10C288000095F4F7BDFFB6F1FF3F08BFB7F1FF3FD8
:10C2980005D056EA070305D12046FFF7BDFF204623
:10C2A80007B0F0BD3A46334604F11800014900F0E2
:10C2B800E7FBF4E7C79F05086FF00A01094A93688E
:10C2C800C3F898100849C3F894004B6843F08053AA
:10C2D8004B60002383F31188BFF36F8F9368D3F803
:10C2E800980070479C3B002000ED00E038B5184CE2
:10C2F800A168206A0B68814214BF1A460022496867
:10C308000B605960A368216A2AB9124AC3E900215F
:10C318000B6023620AE092F90E5093F90E008542F1
:10C3280012DD5168C3E900210B605360E569094BD0
:10C338009D4200D005B9E568A3689D4202D0284611
:10C348003DF0FAFEA56138BD8A42DED01268DBE70F
:10C358009C3B0020B83B002070B590F91020037C6E
:10C36800002A2FDBD9062DD11A4C63F07F03224611
:10C37800037452F81C3F216A934207D1C0E9002197
:10C38800086020620FE09942F8D01B68002BF5D0B6
:10C3980093F90E6090F90E50AE42F4DD5968C0E989
:10C3A800003108605860E569954200D005B9E56834
:10C3B800A3681A7CD20606D1DA897F2A03D9AA692A
:10C3C8000AB9A36170BDAB4202D028463DF0B4FE65
:10C3D800A561F7E79C3B002038B590F9102001468D
:10C3E800002A037C04DA03F07F0303743DF07BFD2D
:10C3F8000D4D2A4652F81C4FAB68944200D004B940
:10C40800EC688B4207D01A7CD20604D1DA897F2ADD
:10C4180001D9A2692AB1A34202D020463DF08CFE80
:10C428002346AB6138BD00BF9C3B0020002A2DE9A4
:10C43800F8430CBF4FF010084FF00808027C044680
:10C4480018EA020F0D4665D148EA0203D2090CD159
:10C458000374B8F1080F7ED1A36813B120463DF0EC
:10C468004AFD102704F118060FE003F07F03037458
:10C478003DF039FDEDE785F31188BFF36F8FEFF3DA
:10C48800118587F31288BFF36F8F304600F088FB61
:10C498000B30F0D0A66D04F15807B74211D04FF019
:10C4A800000976B130463DF026FDC6F8989006F1B1
:10C4B800180000F075FB3046FFF74EFFA66DB74237
:10C4C800EFD1294B9B689C4245D1EFF30587003F8C
:10C4D80018BF0127DFF890904B4653F81C6F9E4217
:10C4E80000D00EB9D9F80C60D9F80830B34202D0A0
:10C4F80030463DF021FEB8F1100FC9F8186009D098
:10C50800204639F0B9FE204600F066FA17B1174800
:10C51800FFF75EFE144B9B68A3421ED1EFF3058321
:10C52800DBB9A289D20711D585F31188BFF36F8FC4
:10C5380083F31188BFF36F8F0423184602DFEFF3EC
:10C548001185102383F31288BFF36F8F2846BDE847
:10C55800F843FFF7B1BE0027BCE785F31188BFF3A6
:10C568006F8FBDE8F88300BF9C3B0020503200204D
:10C5780049B9EFF3058030B9054B9A699B689A422F
:10C5880001D0FFF799BE81F31188BFF36F8F704711
:10C598009C3B002070B50F4D06462B4653F81C4FA8
:10C5A8009C4200D004B9EC68AB681A7CD20604D16E
:10C5B800DA897F2A01D9A2692AB1A34202D020468A
:10C5C8003DF0BAFD2346AB613146BDE870400248F4
:10C5D800FFF7CEBF9C3B00208349002070B5EFF3E6
:10C5E8001186102383F31288BFF36F8F1A4CA1684A
:10C5F800206A0B68814214BF1A46002249680B6002
:10C608005960A368216A2AB9144AC3E900210B605A
:10C6180023620AE092F90E5093F90E00854216DD66
:10C628005168C3E900210B605360E5690B4B9D42DB
:10C6380000D005B9E568A3689D4202D028463DF0C0
:10C648007BFDA5613046BDE87040FFF735BE8A42E4
:10C65800DAD01268D7E700BF9C3B0020B83B002027
:10C66800F8B5DDE906670C461146EFF305833BB1E3
:10C67800002383F31188BFF36F8F0423184602DF6A
:10C688000D4B0E4A98681060EFF31182102282F366
:10C698001288BFF36F8F9D6828463DF045FC3246EF
:10C6A8003B4605F11800064900F0EAF92046BDE8C6
:10C6B800F840FFF701BE00BF9C3B0020CC3B0020A8
:10C6C800C79F0508F8B50446EFF31187102383F3D5
:10C6D8001288BFF36F8F037C49B203F01F02002A50
:10C6E8000CBF0126002635D103F07F032A4D0374C1
:10C6F8003DF0F9FB2A46037C817363F07F030374E2
:10C7080052F81C3F286A934207D1C4E9002004600C
:10C718002C620DE09842F8D01B68002BF5D093F9F5
:10C728000EC08C45F6DD5968C4E900310C605C60C8
:10C73800EC69944200D004B9EC68AB689C4202D022
:10C7480020463DF0F9FCAC6187F31188BFF36F8F89
:10C758003046F8BD9B071CD585683DF0C4FB817346
:10C768002B689D4209D16B68C4E900531C606C605A
:10C77800EAE76A689A42F6D01B68002BF3D093F96F
:10C788000E208A42F5DD5A68C4E9003214605C6004
:10C79800DAE78173D8E700BF9C3B0020034648B91D
:10C7A800EFF3058232B9064A91699268914201D045
:10C7B800FFF782BD83F31188BFF36F8F704700BF07
:10C7C8009C3B0020F8B550EA010305460C4603D10E
:10C7D8003DF087FB0020F8BDEFF31187102383F3AA
:10C7E8001288BFF36F8F144E144BB0681860FFF7B0
:10C7F800F3FDB0682A4623461149183000F040F985
:10C80800B36804461A7CC3F8947042F004021A74A0
:10C818006FF00A02C3F898200A4A536843F080531D
:10C828005360002383F31188BFF36F8F3DF08BFCB7
:10C83800201A20EAE070CEE79C3B0020CC3B002089
:10C84800C79F050800ED00E0024B03F11C02C3E995
:10C85800072270479C3B0020EFF31181102383F3DC
:10C868001288BFF36F8F054B9A68D37B013BD37354
:10C8780081F31188BFF36F8F704700BF9C3B002086
:10C88800EFF31180102383F31288BFF36F8F034BEC
:10C898009A68D37B0133D373FFF77CBE9C3B00209F
:10C8A800014B9868704700BF9C3B0020D3B5DDE979
:10C8B8000667089CCDE90067FFF7D2FE1CB1034B61
:10C8C8009B685B69236002B0D0BD00BF9C3B002021
:10C8D800027C034612F01F0210D10A4988420DD08B
:10C8E8000949086868B1D9897F2909D893F90E20C0
:10C8F800064B1B689A42B8BF00207047002070475B
:10C908001046704790300020CC060020D03B002015
:10C918000122044BC01A044BC0105843034B1A544D
:10C92800704700BF30330020ABAAAAAA8349002071
:10C93800F8B50B4B04461E7C18230A4D0A4F03FB1F
:10C948000655284600F02CF934B1BB5D2846E21A9A
:10C958000649D31700F094F80023BB55F8BD00BF73
:10C968009C3B0020303300208349002019C901086E
:10C97800F8B5EFF31187102383F31288BFF36F8F95
:10C98800124E134BB5681868A84206D13DF0D4FB87
:10C9980087F31188BFF36F8FF8BD00221A60337CCC
:10C9A8000C4AD35C002BF3D02846FFF791FF0446CE
:10C9B8000028EDD02B7CDB06EAD1FFF797FCB369A2
:10C9C800AB42E5D12046FFF7B3FFE1E79C3B0020EF
:10C9D800CC3B002083490020EFF31181102383F31F
:10C9E8001288BFF36F8F0A4A536A834207D1DB6FFD
:10C9F800536281F31188BFF36F8F70471346002B82
:10CA0800F7D0DA6F8242F9D1C26FDA67F1E700BF77
:10CA18009C3B0020024B1868984208BF00207047D2
:10CA2800D006002008B50246FFF7F4FF6FF000417A
:10CA3800C8B18A4215D2D0E90230B0F1FF3F08BF31
:10CA4800B3F1FF3F03D16FF00040801A08BD8B425D
:10CA580070F1000001DB0548F7E79A4201D2981A05
:10CA6800F4E70020F2E78A42EDD3EFE7FEFFFF7F0D
:10CA7800024B186808B1FDF7B9BD7047D806002009
:10CA8800B3F1FF3F08BFB2F1FF3F2DE9F84F04466D
:10CA98009A461546984679D00161EFF3118710231D
:10CAA80083F31288BFF36F8FBAF1000FDFF8E890B5
:10CAB80023DBFFF7DDFF374B06461A68003A18BF3D
:10CAC800012245194AF10003521943F10003D9E93B
:10CAD8000051551943EB01080121DFF8C090C4E962
:10CAE8000223FFF797FFD9F804A0D0B9C4E9009A48
:10CAF800CAF80040C9F8044025E06FF00102D9E9FE
:10CB08000013521A4FF0FF3161EB0303521B63EB22
:10CB18000A03012A73F10001BCBF0122002300218E
:10CB2800DBE7D0E9022ED4E9023C93427CEB0E0B02
:10CB380023DAD21A6EEB0C03C0E902234368C4E976
:10CB480000031C604460FFF765FF84420DD1114B60
:10CB58001B68013309D111B9FFF78AFF0646304631
:10CB6800FFF760FF0021FDF7DBFC87F31188BFF3B7
:10CB78006F8F28464146BDE8F88F9B1A6CEB0E0272
:10CB88005045C4E90232B1D00068AEE70025A84696
:10CB9800EFE700BFD806002048330020D006002069
:10CBA800F8B50446EFF31186102383F31288BFF318
:10CBB8006F8F026872B3FFF72DFF184B5B689C42BA
:10CBC80008D0D2E90231D4E90275DB1941EB05013D
:10CBD800C2E90231D4E900320025844213605A6068
:10CBE800C4E900550ED000200D4A136823F0010156
:10CBF8008C4204BF43F00103136086F31188BFF32E
:10CC08006F8FF8BDFFF734FFFFF70CFF2946FDF7DC
:10CC180087FCE8E76FF01500E6E700BFD0060020C4
:10CC2800D43B0020EFF31182102383F31288BFF363
:10CC38006F8F064B40F001001B681B1A5842584181
:10CC480082F31188BFF36F8F704700BFD43B002079
:10CC580000232DE9F0470C46334E344DDFF8D490CD
:10CC6800334F30602B60D6F80080B8F1000F10D138
:10CC78004FF0FF3340462B60FFF7D4FE4146FDF7E7
:10CC88004FFC84F31188BFF36F8FBDE8F047FFF7BF
:10CC98006FBEFFF7BFFE6FF0004330B1D0E902125C
:10CCA800994272F10002B8BF0B464345194684BF4A
:10CCB800434641464FEAE37C38B18268B2EB030A47
:10CCC800C26862EB0C0EC0E902AEA8EB01014FF09E
:10CCD800000A4FF01008D9F800203160D218D9F8AE
:10CCE800043043EB0C03C9E90023FFF793FE002847
:10CCF800B9D0D0E902120A43B5D1D0E900210A60BF
:10CD080051600269C0E900AA386084F31188BFF352
:10CD18006F8F9047EFF3118488F31288BFF36F8FFA
:10CD2800C7F800A0E1E700BFD83B0020D8060020E4
:10CD3800D43B00204833002010B5EFF311841023B2
:10CD480083F31288BFF36F8FFFF792FE054AD2E98B
:10CD58000031C01841F1000184F31188BFF36F8FCF
:10CD680010BD00BF483300202DE9F0410446EFF321
:10CD78001186102383F31288BFF36F8F03682BB1DA
:10CD880086F31188BFF36F8FBDE8F081FFF74AFF84
:10CD980007460028F4D1D4E90A586A1C48F1000370
:10CDA800022A73F1000324D33DF0D1F9281848EB87
:10CDB8000101012871F1000142DB3DF0C8F96FF073
:10CDC8000203281848EB010183426FF000438B41AE
:10CDD8003BDB3DF0BCF96FF001022D1848EB010375
:10CDE8004FF0FF31521B61EB030320461949FFF74F
:10CDF80047FE236B01332363236A63B186F31188EB
:10CE0800BFF36F8F20469847EFF31186102383F303
:10CE18001288BFF36F8F54F8185FA542B0D0002D69
:10CE2800AED028463DF0A6F80023C5F8983086F322
:10CE38001188BFF36F8F2846BDE8F0413DF065B813
:10CE48006FF001024FF0FF33CFE73A464FF000434F
:10CE5800CBE700BF71CD0108B3F1FF3F08BFB2F1C6
:10CE6800FF3FF8B5044616461D4618D0EFF3118764
:10CE7800102383F31288BFF36F8FFFF791FEDDE96C
:10CE88000623C4E90A2300233246236320462B469F
:10CE98000349FFF7F5FD87F31188BFF36F8FF8BDDE
:10CEA80071CD010870B50546EFF31184102686F39D
:10CEB8001288BFF36F8FFFF773FE20B184F31188D8
:10CEC800BFF36F8F70BD6B6A63B184F31188BFF3D2
:10CED8006F8F28466B6A9847EFF3118486F31288A0
:10CEE800BFF36F8F05F118003DF07EF80028E5D0FC
:10CEF8003DF00BF82146BDE870400148FFF738BB0C
:10CF080084490020034610B5EFF31184102282F300
:10CF18001288BFF36F8FC16001218160006883426E
:10CF280005D184F31188BFF36F8F002010BDD0E9BD
:10CF3800003213605A600023C0E900333DF060F905
:10CF480021460248FFF714FBEFE700BF84490020A1
:10CF5800F8B507460C4616463CF099FF08B1002084
:10CF6800F8BD0E4B9B68D3F88C50002DF7D0221DCE
:10CF7800F5D2EFF31184102383F31288BFF36F8F78
:10CF8800284647F00401B04784F31188BFF36F8F38
:10CF98000028E4D040F8045BE2E700BF9C3B002097
:10CFA8000146024A0020FFF7D3BF00BF7D500508A5
:10CFB80007B5064B4FF44062009305494FF0FF3325
:10CFC8000448FFF75DF803B05DF804FB9C480708C8
:10CFD80020C9002050330020F0B504468BB03DF046
:10CFE800DDFB042C2BD0344D286818B116F0EEFB6D
:10CFF80000232B601CB3314B9C4220D0002601AB90
:10D0080002932F4B214602A8039301963FF073FB2E
:10D0180001983146013016F0B9FB0246286070B11C
:10D0280006AF384601993FF0C0FE264B214604A8BA
:10D03800059304973FF05FFB2A68019BD65402F0E2
:10D048009DFD43F0DEF83DF074FB01F031FD002258
:10D058001D4D1E4BD5F8F0401A7084B1204613F0D0
:10D0680013FC30B3A06805F055F9D5F8F040002C52
:10D07800F4D1D5F8F0301C46DB68002BFBD1C5F89D
:10D08800EC400025124C01F0B9FF11F061FB13F0E0
:10D09800EBFC206816F09AFB25600E4C206816F011
:10D0A80095FB25603DF059F90BB0BDE8F0403DF027
:10D0B80037BBE468DBE700BF383D0020A040002014
:10D0C80013A305082BCD050828400020844900201B
:10D0D800183C0020143C0020002270B50446154B73
:10D0E80000EB8105C3E900229A60264630683EF0CD
:10D0F8008FFF022804F1040418D130680E4C206018
:10D1080098B10E483DF083FC20683DF04CF90C487E
:10D1180002F096F901F0E0FD064920683DF03EF97D
:10D128000023236001F0D8FD012070BDAC42DCD1A2
:10D138000020E3E7E03B0020103C0020B26A08082A
:10D14800D195080873B506463DF0EAFA09F05EFA8B
:10D1580016F01EFA054616F027FA0446641B002549
:10D1680009F05CFAA4F5806009F05EFA01F0A0FC11
:10D1780000F026FC6B464FF4006230461F490095CC
:10D188003DF0C7F801461E4B1E4C1860009B194421
:10D1980006F070FB4FF4005201AB30461A49019576
:10D1A8003DF0B7F80146194B1860019B194413F07C
:10D1B8003DFB06F0AFFB2946D4F8E80009F088F8F3
:10D1C8001621D4F8E8003FF043FB6621D4F8E800C4
:10D1D8003FF03EFB40F6B651D4F8E8003FF038FB8C
:10D1E800294604F1D80009F073F8094804F026F933
:10D1F8000122084B1A7002B070BD00BFDF27080873
:10D20800143C002028400020F6270808183C00207D
:10D21800240C0808844900202DE9F0410928054616
:10D22800A4B000F0878001F05DFC044640B1002DF9
:10D2380040F08380424BD3F8F040003C18BF0124F3
:10D248002846FFF77FFF3DF075FA002C6CD002AC42
:10D258003C4F01F0A7FD4FF4007120463FF08AFDD6
:10D268003C6001F047FC0121054600F180083DF0D3
:10D27800CFF9354B354A364936483FF079F806A894
:10D2880000F00AFB344933483FF097F8002606AC13
:10D2980014F8012B31492F4801363FF08EF8202E23
:10D2A800F6D12F492B483FF063F842F0ABFF02213B
:10D2B8002C48FFF711FF00233B6001F079FD0123A3
:10D2C8004046294A0EA943F022FFA0B9029842F02D
:10D2D80067FA039A0446014601AB01320EA844F0EE
:10D2E80036F840B9039A019B9A4204D12146049822
:10D2F80056F014F8A0B14FF47A703DF0DDF90A2326
:10D30800194A0EA9404643F002FFDDE9032101ABAB
:10D318000EA844F0D0F80EA844F03AFA01F0C8FB81
:10D32800002128463DF074F9104C6068FFF754FE60
:10D338000023636024B0BDE8F081002480E700BFCB
:10D3480028400020DC3B0020102808082328080873
:10D35800712808086C5B07081F8D0808BD95080828
:10D368008D300808D848070881280808E03B0020C5
:10D378002DE9F04F8146AA4E89B0002842D00024FA
:10D38800202725463368B3F5007F00F0B480B9F153
:10D39800000F40F0B48001264FF4405302933DF053
:10D3A80087F90390002C40F05B814FF4C87BA046BE
:10D3B8000BFB06F3012603F59C5A04930AF1080AAD
:10D3C80001F0EAFD01F04AFC05460190002800F052
:10D3D800998047F0100701F0F5FB924E306828B1AC
:10D3E80003781F4002D116F0F1F93760B8F1000F49
:10D3F80004D0002001F0FAFC01F0F2FC284609B044
:10D40800BDE8F08F01F054FB01F046FC054600280A
:10D41800B5D1844FFFF796FE3DF093F93B68002B9A
:10D4280055D01A7822F020021A703B689A681C7846
:10D43800127892B1586808B104F000F83B680121ED
:10D448009B6807A80793FFF747FE98B93B68986859
:10D458003DF0DDFA744801F0F3FF04217348FFF74B
:10D468003BFE38B908217248FFF736FE10B1714803
:10D4780001F0E6FF336818052BD500F0BFFF01283F
:10D4880027D16D484FF0000801F0DAFF6B4B706848
:10D4980083F80080FFF7A0FD3A68C6F804802AB137
:10D4A8001378990644BF43F02003137033681A05B4
:10D4B80011D500F0A3FF441E18BF0124302733689C
:10D4C80003F48073002B0CBF254601245AE72C4631
:10D4D800C3E75B48D6E71BB9242704F00104EEE74D
:10D4E80014F0020418BF83F480634FF0280718BFB4
:10D4F800C3F38024E3E702264FF440134EE70326E4
:10D50800504B4BE73DF05CFA059080B13DF077FA5F
:10D5180068B101F0C1FB054648B93DF05EFA042840
:10D528007FF45BAF032000F06FFF059D55E7F4B96A
:10D538003DF046FAE0B101F0AFFBC8B942483CF013
:10D5480032FF01F067FB00283AD0404801F078FF2D
:10D55800B9F1000F02D03E4801F072FF484601F0D1
:10D56800EBFE3C483DF053FA3B4801F069FF0124CB
:10D578003DF026FA2040C4B22EB101F08DFB10B95F
:10D5880003F05AF806463DF093F8039B049AC31A31
:10D598009A42054623D9B3FBFBF20BFB1235632DE8
:10D5A80010D9B8F1000F04D0002001F01FFC01F0E1
:10D5B80017FCC5F5C8706EB3B04228BF304629E0E5
:10D5C8002648C3E7B8F1000F04D101F029FC0298FE
:10D5D80001F00CFC0123C5F164000193EBE79A45C7
:10D5E80007D23DF065F8CDF804800390DDF804809B
:10D5F800E6E6B8F1000F04D0002001F0F7FB01F0D7
:10D60800EFFB039B5344581B16B1B04228BF30466A
:10D618000028EBD015F0ECFF16F034F8E6E700BF71
:10D62800E03B0020343D0020D7950808C84807088B
:10D63800A8480708448C0808B38B080884490020C8
:10D64800CD8B080800303000B26A0808A793080894
:10D65800448E0808A2290808BC8E0808D393080835
:10D668004FF00008B9E600BF07B5114B186820B1A4
:10D6780003B05DF804EB3DF0CAB90E4B1A68920589
:10D688000FD59A68002A0CDD596851B109680C3326
:10D69800C9880948009109493EF06AFE03B05DF85F
:10D6A80004FB074803B05DF804EB01F0C9BE00BFF6
:10D6B800103C0020E03B00206C5B07088F2808081E
:10D6C8004F920808F7B515F047FF01F073FD3CF0DD
:10D6D80044FE15F0F9FF3DF04DF801F01FFD5048EC
:10D6E8003CF061FE3DF09DF901F06CFB01F05CFD42
:10D6F800B0FA80F00021400901F00EF910B90820B5
:10D7080001F058FD01F050FD18B901F059FD01F084
:10D7180051FD42F076FD3DF00CF83DF009F802F0BD
:10D7280067FB3F483CF03FFE002000F06DFE01F033
:10D738003BFD08B901F04CFA0125012001F0CCF9B4
:10D74800012001F0C3F901F02FFDFFF765FD3CF062
:10D75800E8FF012001F0B4FA4FF480742846314EF6
:10D7680014F4106754D015B92F4801F069FE3578C4
:10D77800002D3ED101F018FDFFF7FAFD0028EFD18A
:10D7880001F012FD044601F093F92046FFF7DAFC98
:10D798003CF0D7FF012001F02DFA01F005FD28B972
:10D7A800224B012101A80193FFF796FC01F038FBF9
:10D7B8001F4801F01BFB01F013FB3378012B1AD132
:10D7C80001F0F0FA00F0A4FC044601F0F1FA04209C
:10D7D800FFF702FC01F024FB002001F007FB01F039
:10D7E800FFFA012001F00EFA032000F00DFE0020E0
:10D7F800B6E70025C4E70F4B0F4F3B6001F06CFA0A
:10D8080000F00CFD002304463B6001F065FADEE7FA
:10D81800002CB3D03EF019FE384603B0F0BD00BF6F
:10D82800B26A080885490020CA7F080898280808AD
:10D8380030303000A0280808103C002008B513F04C
:10D8480033F800F027FB0421074842F07FF83CF04A
:10D85800BAFF01F007FC02F00DFA04F0E5FABDE8A2
:10D86800084013F035B800BF18410020014B187864
:10D87800704700BF844900209FED010A704700BF30
:10D888000000000000487047006889099FED010A00
:10D89800704700BF3333534038B505462021FBF7A6
:10D8A800C3FB041E11DA2146094837F0EAFE0024BA
:10D8B80021462022074837F0E4FEC4F12002281947
:10D8C8000021BDE8384055F021BD1F2CF0DD38BDE2
:10D8D800302908084A2908080428034607B506D845
:10D8E80001460E4803B05DF804EB01F0EBBA0621DF
:10D8F80068460B4A33F0E8FA052801DD38F0F4FCF5
:10D90800442200F108036B44411C684603F8082CC4
:10D9180001F0D8FA03B05DF804FB00BF71290808CC
:10D9280076290808F8B5244DAB7DDB0731D52E687C
:10D93800706801282DD9B168431ECA5C0A2A28D10B
:10D948004A1E002B01DC1A4608E0D45C0A2CFAD0E7
:10D95800013BF6E78C5C202C02D101329042F9D8C9
:10D96800002B0CDD541CA04209D15C1E0C448C42D7
:10D9780005D014F8017D0A2F0BD0202FF7D00144D1
:10D98800D21A11F8023C94083A2B00D10134013C18
:10D9980000D2F8BD0422304608493FF0C2F90421FC
:10D9A800064801F08FFA2B6904332B61AB7D43F0F5
:10D9B8000203AB75EBE700BF1C3C0020E1680808D8
:10D9C80020220021014855F0A1BC00BFE040002002
:10D9D800002238B50B4C0546A26062754FF0FF3245
:10D9E8006B680846C4E9032363602560A1613CF0C5
:10D9F800DAFC6B680BB90123A375BDE83840FFF763
:10DA080091BF00BF1C3C0020F8B503780446DBB189
:10DA18000E4FD7F8B80018B12146F3F777FA98B146
:10DA28002046F3F785FA461C304641F0BCFE054611
:10DA380050B13246214655F043FC05491C22081DC9
:10DA480055F04BFCC7F8B850F8BD00BF284000207F
:10DA5800E04000202DE9F347A44C06462368D3E9AB
:10DA680001103EF092FDA5688146042D00F20E8259
:10DA7800DFE815F005002A013301CE010702731E05
:10DA8800042B15D8D4E900325B689A4200F08180F3
:10DA9800012E0FD123686568986826698119284482
:10DAA8003CF064FC761B00250746A846A5606BE1A0
:10DAB8000D2E11DC022E13DDF31E0A2B10D8DFE821
:10DAC80013F068000F00C1010F000F006F000F0076
:10DAD8000F000F0024005D001B2E5ED07F2E5FD04C
:10DAE800A37D9A0740F19780092E00F08B80202EA5
:10DAF80040F0BF804FF000080321206884F81680AA
:10DB08002F463FF0FEF903266DE079483CF04BFCC8
:10DB1800A0693CF048FC2268636821699068C91ACA
:10DB2800184401F0CFF900252368D3E901103EF02D
:10DB38002CFD484503D203216E4801F0C3F9236840
:10DB48002769D3F80880D3F80490781908EB0901FD
:10DB580040443CF00BFC0646A9EB070108EB070024
:10DB680001F0B0F9236822695B689B1A5B1B981B5C
:10DB7800FFF7B2FE23692B44236145E05E483CF081
:10DB880012FC20683FF046F963682E461844FFF7F8
:10DB98003BFF304602B0BDE8F0870123A36033E0C5
:10DBA8002669626896422FD92B462068B11AD0F8A8
:10DBB80008C08B4203EB02071CD1042BB4BF01271A
:10DBC8000427F71B3B461CF80320194602F0C00245
:10DBD800802A03F1FF33F6D0761A32467F1A4FF0C7
:10DBE80001083FF095F9F01BFFF776FE23699B1BB0
:10DBF8002361CCE01CF80770202F01D10133D8E74E
:10DC08000127DEE70023A375A37D4FF0FF3623F03D
:10DC18000203A375BDE7092E2BD123685A68C2B148
:10DC28009B682269134413F8010C07F075F980B159
:10DC38000426324B01930025019B21695A1C01924D
:10DC480029441A78206801353FF04FF9B542F3D1DD
:10DC58006AE7236860689D682169294A091A01AB47
:10DC6800284408F0D1FD06460028CDD0431CE2D157
:10DC78004EE71F2EC8DD06F0C0032068802B08BFC2
:10DC88008368276912BFF3B2DB5D217D03F140028F
:10DC980008BF0131D2B214BF0021C9B2372A97BFD9
:10DCA800E5250025DB0803F0060398BF1D41217513
:10DCB8003246394498BF05F003053FF01CF9237D2F
:10DCC800AB42A1D101352FE74F2E04D05B2E40F097
:10DCD800DD80022362E7042360E7A6F13003092B05
:10DCE80010D803236675A3608EE700BF1C3C002094
:10DCF8007B29080884290808A2290808E168080877
:10DD08006C5B07080023413EA360072E3FF67CAFFB
:10DD180001A353F826F000BF41DD0108A1DD010889
:10DD2800E1DD010805DE010811DC01084DDE01080E
:10DD380011DC01089DDA0108E368062B3FF764AFA0
:10DD4800534D03F1010A2D3305EB8305AB68002B16
:10DD58003FF45AAF2668D4F80480B06821690144BA
:10DD680040443CF003FB07463046C6F80480A968E7
:10DD7800C4F80CA03FF0ACF84FF0010822686368C3
:10DD880026695568F61AED1A002E3FF72CAFB8F140
:10DD9800000F7FF4C9AE26E0E568002DFFF634AF2A
:10DDA8002668D4F80480B0682169013D01444044E4
:10DDB8003CF0DCFA71680746A1EB08013046E560E3
:10DDC8003FF09FF8E268002AD6DB314B206803EB6E
:10DDD8008203D3F8B810CDE7236825695B689D42B4
:10DDE8002CBF00250125002D7FF70EAF236829469B
:10DDF80098682369184401F065F8BBE622696368EE
:10DE08009A427FF601AF00250126A8462F46EAE68A
:10DE18007E2E3BD1637D313B072B37D801A252F8C8
:10DE280023F000BF9DDA010895DE01085BDE0108DA
:10DE38004DDE010895DE010895DE01089DDA01082E
:10DE48004DDE010823685D682369ED1A0023A3608D
:10DE5800C9E7206821694368994217D20122856879
:10DE68005B1A0D4415F8016F06F0C006802E01D12B
:10DE78009A4204D13FF04CF80023A36053E60132E4
:10DE8800F0E7462EDED0482E3FF404AE002385E6A8
:10DE9800284000202DE9F04F8BB068460A4BCDE9A9
:10DEA80000451968CDE90267091A8908CDE904898E
:10DEB800CDE906ABCDF820C0CDF824D041F046FD21
:10DEC8000BB0BDE8F08F00BF2840002070B5067881
:10DED80004461EB14FF0FF35284670BD3CF074FC77
:10DEE800C31E012B05460CD801210C48217000F0F7
:10DEF800E9FF032DEED10A48836E60309E6013F06F
:10DF0800E5FFA388013B9BB2A380002BE4D101214C
:10DF1800044800F0D7FF6388A380DDE78829080854
:10DF280028400020A62908082DE9F0431D460023B3
:10DF380097B0044603A817460493884613F0ACFF2D
:10DF480007F001060346002877D1F90665D5D4E91C
:10DF58000121DC2041F0B5FF0446B8F1010FD4F8E7
:10DF6800009007D14FEA09114FF4397041F00601CA
:10DF780005F038FD2146424601A813F0C3FB494687
:10DF8800C7F3800201A80FF015FCB8F1010F044691
:10DF980001D1FFF753FC380602D4032000F0E6F95C
:10DFA80014B120463EF08AFA4FF0FF3000F0DEF957
:10DFB800012004F039FB10F0D1FC1EB101214548C5
:10DFC80000F080FF0024FDB12C60ECB14FF0FF336E
:10DFD800049FAB6038466F603FF071FAA0B16946A4
:10DFE800384601AA3FF09AFA019B6BB15A68AA60B9
:10DFF800002285F82C20186840F0D6FE2022014621
:10E0080005F10C0055F0B9F91EB10121314800F0B5
:10E0180059FF204617B0BDE8F0837A0605D594E885
:10E028000E00DC2041F005FF96E7BB0695D520469B
:10E0380040F09AFE41F053FF8EE74FF0FF3000F0BA
:10E0480095F9022004F0F0FA790602D5A368206851
:10E0580098471EB101211F4800F034FF049C204658
:10E0680007F05AFA1C490DF091FDF0B104983FF001
:10E078003BFA0E2817D0C20705D4830708D10268D7
:10E08800164B9A4204D141F01DFB40F480749AE784
:10E0980001460022124807F05BFA124910483EF088
:10E0A800E7F80120F1E70020EFE70F4B9C420DD085
:10E0B80004990B483EF01FFB049B0C4918680DF0AF
:10E0C80065FD002814BF822401247CE74FF4006416
:10E0D80079E700BF88290808E86B0708A85E0708E1
:10E0E8006C5B07088D300808A0400020C46B070847
:10E0F80008B503784BB901210170044800F0E2FE2D
:10E108003CF062FB03380128FAD808BD88290808C2
:10E11800F0B58BB0202106A83EF02CFE002536482D
:10E128003CF041F9079535483CF03DF93CF04CFB93
:10E13800431E032B43D8DFE803F002353F47079916
:10E148000229ECD1089B1A78052AE8D15F78412F7B
:10E1580005D02B4800F0B6FE00230793E3E78024A0
:10E168000126284800F0AEFE03216846ADF80040BD
:10E178008DF8026000F0A6FE002301AA0392224A4D
:10E1880031460492214A03A805923A468DF8043094
:10E19800ADF80640ADF80840FFF7C6FEC305DBD56D
:10E1A8000BB0F0BD1A483CF0FEF806A83EF004FE9D
:10E1B8000020184B1870F3E700230793B6E7C1B2A5
:10E1C80006A83EF036FEB1E713483CF0ECF8079B92
:10E1D80043B90F483CF0E7F806A83EF0EDFD4FF4D0
:10E1E8008070DDE700231122012106A8FFF79CFEBD
:10E1F80010F4106F96D0D3E78A2908082A31080846
:10E20800383F0708A5290808D5DE0108F9E0010804
:10E21800A229080885490020A829080870B598B0DF
:10E22800202101A83EF0A6FD474E48483CF0BBF827
:10E2380047483CF0B8F845483CF0B5F8B28A0023A6
:10E2480002B1B38205A80293069313F025FE044693
:10E2580088B9404901A83CF097F8012805462BD118
:10E268003A483CF0A0F801A83EF0A6FD20463A4BFB
:10E278001D7018B070BD022004F0D6F933483CF088
:10E2880092F8069935483EF036FA029B002BD5D015
:10E2980001A83EF0BFFD08F0F9F958B10A2101A81C
:10E2A8003EF0C7FD2E4901A83CF06EF80328C2D005
:10E2B8000428EDD100212CE0851E032DE5D801A30B
:10E2C80053F825F0DDE201083FE20108E5E2010824
:10E2D800F7E201081D483CF066F8A6E71B483CF049
:10E2E80062F801A83EF068FD4FF48070C1E71D4850
:10E2F8003CF059F8002302933CF066FAC1B20329B6
:10E308008DF8031097D004290CD110483CF04BF835
:10E3180001210023162201A8FFF706FE10F4106F52
:10E328008CD0A6E701A83EF084FD9DF803300D2BA4
:10E3380003D10D483CF037F8DEE701210DF1030069
:10E3480000F0C0FDD8E700BF28400020A229080837
:10E3580023280808AB290808854900206C5B0708B2
:10E36800E7290808B0290808E0290808014B1860BF
:10E37800704700BFDC060020024B986A003818BFBF
:10E3880001207047284000202DE9F04106460D463F
:10E3980000270DB9BDE8F08133780A2B16D1AFB943
:10E3A8000121104800F08EFD012406EB04084346C5
:10E3B8001FB998F800200A2A01D0A54208D1304692
:10E3C800214600F07FFD46462D1BE2E70024ECE7DE
:10E3D8001F7808F10108A7F10D035F425F4101347E
:10E3E800E5E700BFEC290808024B034819783EF01E
:10E3F800EFBD00BF8649002050520708014B18782E
:10E40800704700BF86490020014B1870704700BF55
:10E41800864900206FF013030B41DB0710B5024655
:10E428000C4615D50B490C483DF0C7FF022C03D00C
:10E43800052C0BD0094900E0094907483DF0BDFF0C
:10E44800BDE81040074904483DF092BF0649F4E78B
:10E4580010BD00BFDF9308086C5B07080991080826
:10E46800BD9008088D300808C89008082DE9F04FBD
:10E4780099B000AF81460C46904600F03BFB28B9A6
:10E48800012528466437BD46BDE8F08F01239F4A21
:10E4980007F10801803042F03AFE0028F0D1D7E9B0
:10E4A8001002D7E906139A4208BF884200F02C816F
:10E4B80097F83930002B40F0278107F108003BF02E
:10E4C800DEFF5B28064606D1D7E9062307F10800D8
:10E4D80043F057FAE3E7002EF6D009F1FF3A1AF8AD
:10E4E800015F2DBB304606F017FD20B107F108008B
:10E4F8003BF0C5FF06463D2E1CD107F108003BF056
:10E50800BEFF22280CBF0123002388F8003040F00A
:10E51800CB8007F108003BF0A3FF222829D016D8AA
:10E5280028B30A2823D0C1B220463BF0C0FFF0E749
:10E53800B54206D00A2EB2D007F108003BF0AEFF74
:10E54800ADE707F108003BF08BFF0646C7E75C28FC
:10E55800E9D107F108003BF083FF7628E3D861286A
:10E568001CD80A2803D0552854D00028DBD105250B
:10E5780009E007F108003BF082FF0A2803D02328AE
:10E5880007D00028F3D1EDB207F1080043F000F9F5
:10E5980077E707F108003BF081FFF4E7A0F1620399
:10E5A800142BC0D801A252F823F000BFADE6010831
:10E5B8002FE501082FE501082FE5010819E60108F4
:10E5C8002FE501082FE501082FE501082FE50108CF
:10E5D8002FE501082FE501082FE501080DE60108E0
:10E5E8002FE501082FE501082FE5010809E60108D4
:10E5F8002FE5010811E6010891E6010815E6010872
:10E608000D2090E70A208EE709208CE70B208AE787
:10E618000C2088E74FF0080909F1080323F00703E5
:10E628006E46ADEB030DEA46E8460DEB090B07F124
:10E6380008003BF015FF08F8010BD845F7D1002377
:10E64800391D0AF809301022504632F0DBFC7B688D
:10E658000146434524D1B0F5881F1ED27F2816D91C
:10E66800B0F5006F15D3B0F5803F2CBF042303230A
:10E67800227B22B16268134422689A420BD9204651
:10E688003EF0DEFBB54644E74FF00409C4E701233A
:10E69800EEE70223ECE76360F4E70225B54672E78C
:10E6A800B54664E708203EE70A283FF460AF002833
:10E6B8003FF45DAF00250D281CD00ADC092819D0CD
:10E6C8000A2812D088B1C1B220463BF0F0FE0025DE
:10E6D80015E020280ED02328F5D1636807F108003B
:10E6E8005B1B63603BF0DAFE02E063685B1B636000
:10E6F800002548E7C1B220463BF0D9FE013507F1B5
:10E7080008003BF0ADFED6E704253DE7EE290808F2
:10E7180030B587B00D4610220DF1070302A93BF072
:10E72800D1FE044648B99DF8073083B9094902A8C3
:10E73800F2F7ECFB20B901232B70204607B030BD5F
:10E74800054902A8F2F7E2FB08B92C70F5E70524A1
:10E75800F3E700BFFD290808022A08082DE9F0415F
:10E768008EB002AC0F46302221460DF103033BF078
:10E77800A9FE054628B99DF80380B8F1000F04D01A
:10E78800052528460EB0BDE8F0812046F2F7D0FBFB
:10E798002618A6420CD99DF808302B2B01D02D2B1A
:10E7A80006D12D3BD3F1000848EB03080DF109040D
:10E7B800311B022923DD2378692B15D163786E2B51
:10E7C8001DD1A378662B1AD14FF0FF43E01C0193AB
:10E7D800B042D5D1DDED017AB8F1000F01D0F1EEEC
:10E7E800677AC7ED007ACCE76E2B08D16378612B86
:10E7F80005D1A3786E2B02D1054BE01CE7E7204634
:10E8080001AA13F01BFC0028BAD08442E0D1B7E774
:10E818000000C07F70B5054688B004A80C462021CA
:10E828003EF0A8FA28460DF1060204A9FFF71EFEDD
:10E83800064630B99DF8063033B104A80AF06EFADE
:10E848002060304608B070BD28460DF10701FFF77B
:10E858005FFF38B99DF80730002B0CBF1E233E23FD
:10E868002360EEE7284602A93BF051FE18B902984A
:10E8780040F0EBFEE4E7284603A9FFF76FFF88B9ED
:10E88800DDED037AF4EE677AF1EE10FA7DBF17EE4C
:10E89800903A23F0030343F00203034B78BFA3F13C
:10E8A800FF43DDE70526CCE70200400000B597B03E
:10E8B80002460A236946044842F029FC684642F0A9
:10E8C80067FF17B05DF804FB4014002010B5064C34
:10E8D80023783BB14FF47A72044B1A6000F0E8FBDE
:10E8E8000023237010BD00BF87490020E0060020E8
:10E8F800074B1A685AB11A68012A09BF05491A68EC
:10E908000A704FF47A7218BF02F1FF321A6070472A
:10E91800E0060020874900202DE9F0414FF000086B
:10E92800514EADF5287D0746504C30460D46A6F8A9
:10E93800048000F0CBFB06F18000C4F8048042F0AC
:10E94800E2FB0D2802D127B91DB98BE0002D00F09C
:10E9580087804FF40073002200930721444828ABB6
:10E9680016F03EF800287DD100F0A2FB414940484E
:10E9780015F04EFF002875D13F493D4843F0D6FABF
:10E9880000286FD13D48FFF791FF3D48FFF78EFF04
:10E998003C48FFF78BFF3C48FFF788FF3B4934486A
:10E9A80043F0C4FA3A4B03AA03F13807154618682E
:10E9B8005968083303C5BB422A46F7D11B88354A34
:10E9C8002B80392302AD12A92B6029480A2342F073
:10E9D8009EFB2B462A6803A912A842F06CFD12A8D8
:10E9E80042F0D6FE2C48FFF761FF2C4B03AA03F137
:10E9F800100C174618685968083303C763453A4628
:10EA0800F7D1186899889B793860BB711623B9804B
:10EA1800234A2B6012A90A23154842F078FB03A960
:10EA28002B462A6812A842F046FD12A842F0B0FE12
:10EA38001C490F4843F07AFAA0B900F039FB1A4B89
:10EA4800012523600023E360184BC4E90156C3E99C
:10EA58003B443CF080FE28460DF5287DBDE8F0815A
:10EA68000028ECD00020F7E7C0130020383C002035
:10EA7800401400208B350808082A0808142A0808BA
:10EA8800272A08083E2A0808482A0808552A080894
:10EA98007B2A0808592A0808EE290808B52A080810
:10EAA8006D2A0808762A0808240C0808284000203F
:10EAB8004FF47A7208B5044B1A6000F0F9FABDE811
:10EAC800084014F0E9BB00BFE006002001460148F9
:10EAD8003BF076BDC0130020014601483BF08EBDD7
:10EAE800C0130020024B5868003818BF0120704737
:10EAF800383C0020034B04485B68002B08BF00200B
:10EB0800704700BF383C0020C013002008B544F00F
:10EB180076FD3BF088FF00F0ABFFFFF7D7FE44F02F
:10EB280070FD3BF080FF002041F06DFB034BC3E913
:10EB38000001BDE8084044F063BD00BF5034002028
:10EB480008B5FFF7D5FEBDE8084000220149024894
:10EB58003BF053BE15EB01084C3C002010B5074CA8
:10EB680002F0C0FA23680BB914F02EFD23680133B4
:10EB78002360BDE8104002F0CFBA00BF483C002037
:10EB880008B502F0AFFA074B1A6812B11A68013AD1
:10EB98001A601B680BB914F025FDBDE8084002F0A7
:10EBA800BBBA00BF483C002008B5FFF72DFC044B5A
:10EBB80003F178029A62BDE8084014F0E3BC00BF94
:10EBC800284000200022014B1A6070475C3C00205E
:10EBD8000122034B1A700022024B1A60704700BFD3
:10EBE800884900205C3C00200022014B1A707047C5
:10EBF80088490020024A136803431360704700BF26
:10EC0800603C0020024A136823EA0003136070473F
:10EC1800603C0020014B1878704700BF88490020ED
:10EC280038B50B4B1B7893B10A4B1B687BB90A4C60
:10EC380025683BF03DFD2060236813B92368013344
:10EC4800236025B9BDE838400120FFF7ADBF38BDC6
:10EC580088490020603C00205C3C002010B50C4C2A
:10EC6800206890B10B4B1B6883B93BF021FD2368EA
:10EC780083422368A0EB030040F2EE2388BF00F133
:10EC8800FF30984294BF0020012010BD0020FCE70F
:10EC98005C3C0020603C0020024B1868003818BF1C
:10ECA800012070475C3C0020034B1B7813B90348D4
:10ECB8003BF0ADBE704700BF89490020CC2A080848
:10ECC80010B10122024B1A70024800F041B900BF8E
:10ECD8008A490020643C0020F8B5234B1E7826B1F1
:10ECE800BDE8F8400120FFF7EBBF204B20481E701D
:10ECF8003CF075FE1E483CF058FE78B33BF060FED1
:10ED080080F00105EDB21A483CF061FE80F0010484
:10ED1800E4B21DB1012000F037FA064604B3012021
:10ED280000F03AFA074613483BF071FE12483BF0F0
:10ED38006EFEFEF799FC11483BF069FE10483BF067
:10ED480066FE10483BF063FE15B1304600F01CFA31
:10ED580044B13846BDE8F84000F01EBA0125D2E7B4
:10ED68002746E0E7F8BD00BF894900208A4900200E
:10ED7800A0070020D32A0808D82A0808DD2A08088E
:10ED8800E12A0808D02A0808044B1B7823B9044B49
:10ED98001B780BB1FFF7A0BF704700BF894900205F
:10EDA8008A4900200122014B1A70704789490020C6
:10EDB8000022024B02481A7000F0CAB889490020A4
:10EDC800643C0020034B044A04481A6000225A603D
:10EDD8003CF0FFBD643C002091ED0108A007002035
:10EDE80001483BF051BE00BF783C002038B5094DC2
:10EDF80004462B6883420CD0074B19783BF0A3FCE0
:10EE08002C60011E18BF0121BDE83840034800F0FE
:10EE1800F7BD38BD743C0020580C0020783C002019
:10EE280070B50B4C257895B901260A490A48267011
:10EE380000F0CAFD2A46314607483BF04DFE4FF028
:10EE48008072064B18681A60FFF7D0FF257070BDF6
:10EE58008B490020ECB30708783C0020743C002064
:10EE6800014B1870704700BF580C0020014B1878F0
:10EE7800704700BF580C0020034B1868034B00284C
:10EE880008BF1846704700BF843C0020718521499F
:10EE98001FB50B4901A800F097FD012101A83BF01F
:10EEA80042FE01203CF0BAFE01A83BF0F8FD044602
:10EEB80001A83BF0E9FD84F00100C0B204B010BD28
:10EEC80024B207082DE9F843DFF8808000AF054633
:10EED8000E463BF051FCD8F8003043B31A483BF0DB
:10EEE800A3FDC0F500720446D8F8000043689919DC
:10EEF800914223D90734D21A294624F007043DF059
:10EF080010FFE946ADEB040D69460F48D8F80040FC
:10EF180000F0A0FA014620463DF0DAFF0A21D8F8B1
:10EF280000003DF086FF0023C8F80030CD4631468A
:10EF3800284600F001F9BD46BDE8F8833246294667
:10EF48003DF0EFFEF3E700BFDA8B0808DC3B00205A
:10EF580010B5044602F0C6F8E3681BB90C4A1168FC
:10EF6800A14203D1BDE8104002F0D6B8A360094B16
:10EF78001968E160196809B119688C60116801B9EC
:10EF880014601C6002F0C8F814F0FCFA10BD00BF51
:10EF9800903C00208C3C00202DE9F041144E44F0B8
:10EFA80031FB33680BB3134D02F09CF82C681CB18D
:10EFB800BDE8F04102F0B0B801230F4A2B60336876
:10EFC800346014601BB92B68013B2B60F0E79F6825
:10EFD800C3E90244D3E9006802F09EF80EB1404646
:10EFE800B04702F07FF83B46ECE7BDE8F08100BF90
:10EFF800903C0020883C00208C3C00202DE9F74301
:10F008000025A846144E019502F06CF8346801AF4B
:10F0180054B9019B3360114B1D60114B1C6003B048
:10F02800BDE8F04302F078B8D4F808902046C4F858
:10F03800088011F029FC18B10023E3604C46E7E78B
:10F04800606811F021FC0028F6D12B463C6025466B
:10F0580004F10807F1E700BF903C00208C3C002039
:10F06800883C002010B5044B1C6804B910BD6068CA
:10F0780040F0A0FCA468F8E7903C0020F8B50E46E4
:10F088001C4615466AB1094F3B781BB9FFF766FD68
:10F0980001233B7022463046691EBDE8F84014F053
:10F0A80085B9012B94BF00200120F8BD8C490020B0
:10F0B80010B5054C14F0D8F823780BB1FFF760FDB4
:10F0C8000023237010BD00BF8C49002010B50F4BE2
:10F0D80004460360838843F00503838041F081F888
:10F0E80001230E220A4984F88430231DC4E9082329
:10F0F800C4E90D2323616161064B0749A060C4F888
:10F108008040E260A162E36310BD00BFB49A0708C3
:10F118000BA8050869A9050885F0010810B5054C74
:10F1280023782BB93BF03CFC41F090F80123237085
:10F1380010BD00BF8D49002073B505460C46C1B10E
:10F148000E4B1B78C3B90A4601AB01460C4802F0C6
:10F158000DFB06460B4B1B7853B902F0BBFC40B1C4
:10F16800214628463BF024FC2146284614F0E0FBC3
:10F178003446204602B070BD0E46EBE78E490020AB
:10F188006C0800208F490020024B1A78187010462E
:10F19800704700BF8F490020024B1A78187010463C
:10F1A800704700BF8E490020014B1878704700BF98
:10F1B80090490020014B1870704700BF904900200B
:10F1C8002DE9F34114F0C2F93E4B074620F47F00C5
:10F1D80020F47F4098423C4D0BD117F47F4FC7F382
:10F1E800072406D014F0ACF92C70204602B0BDE814
:10F1F800F08100232B703BF0B7F8072803D8A2232F
:10F20800C340DB0735D4314814F09AF9FFF708FEFC
:10F218004FF07E532E4801A901933BF0BEF9DDED76
:10F22800017AF5EEC07AF1EE10FA24DB9FED297A27
:10F23800F4EEC77AF1EE10FA1DD89FED277A67EE43
:10F24800877AFCEEE77A17EE905A3BF022FA002410
:10F258000646884620462146A84271F100030DD390
:10F268000020FFF7C3FDFFF7BBFD4CBB384614F089
:10F2780067F90024B9E74FF47A75E6E7ACB9FA22E2
:10F288000023F1F7E9FD7D2A73F100030DD3204631
:10F29800FFF7ACFDFFF7FCFD044658B13BF0F9F968
:10F2A8004FF47A750646884604E00C48FFF79EFD41
:10F2B800002CEFD03BF0EDF9801B61EB0801CBE7A8
:10F2C800112492E7AF0000AD90490020AF1100ADC6
:10F2D800E82A08080000804F00007A440030300017
:10F2E800024B43EA002014F02BB900BFAF0000AD79
:10F2F8000D4D08B52B780446012B0FD901280DD9DF
:10F308000A4836F0BEF92146094836F0BAF9297894
:10F31800084836F0B6F936F0B8FFFCE72046FFF7A4
:10F32800DFFF40F06AFF00BF90490020022B080869
:10F33800182B0808242B080810B50446002838D0D4
:10F348001C4800F07DF8631E112B12D8DFE803F08B
:10F358002D1111111111112B1129111127212523FB
:10F36800091F154800F06CF8BDE81040134800F07C
:10F3780067B8023C1248E4B200F062F80A2C16D8CA
:10F38800104B53F8240000F05BF80F48EAE70F48E9
:10F39800E8E70F48E6E70F48E4E70F48E2E70F48D9
:10F3A800E0E70F48DEE70F48DCE70F48DAE70F48E9
:10F3B800E9E710BD5E8B0808E88B0808738B08081E
:10F3C800BE920808484A0708838B0808F89008087E
:10F3D80077930808F28C0808078D0808078E080834
:10F3E800D68D08081E930808DD8E0808A68C080824
:10F3F800A1F18003612B70B5064619D8194602237E
:10F408000D480E4C10F8012B914205DA03FB01441C
:10F41800E518A54206D870BD891A12FB03F201331C
:10F428001444EFE7304614F8011BFFF7E1FFF0E75B
:10F43800BDE870403DF004BDBB6A0808C56A08080D
:10F448000246024902483CF093BF00BF3B2B080824
:10F45800788E07082DE9FF41054680240A4615F8ED
:10F46800011B684601313DF0A0FC009E234FDFF8E8
:10F478009080013E019B9E4205D868463DF0CAFC3B
:10F4880004B0BDE8F08100239C4619461A46287846
:10F4980052002040003818BF0120640842EA0002E8
:10F4A80004BF8024013501316245C9B204D3785CB8
:10F4B80000EB4C0C0344EAE7A3EB0C034244D15C99
:10F4C800012916D10B2200202B7840002340003B55
:10F4D80018BF0123640804BF80240135013A40EABB
:10F4E8000300F1D13FF060FC014668463DF0F0FCB6
:10F4F800C0E76846FFF77CFFBCE700BF606D0808FF
:10F50800A86C080808B5024836F0BBF8002008BD0A
:10F518003E2B080838B5FFF7EDFA044620B90D4828
:10F5280036F0AFF8022038BD3BF05DF820B90A4844
:10F5380036F0A7F80420F6E7084D2B782BB92046BB
:10F548003BF089F808B90648F2E7012300202B7040
:10F55800E9E700BF512B0808632B080893490020EE
:10F56800762B0808F8B514460E461F46FFF7C2FA70
:10F5780005460420FFF73EFB3B4622463146284617
:10F5880042F064FFD5F8CC30A34207D134B14FF430
:10F598000072314605F5807053F092FED5F8BC3004
:10F5A8000020A3429EBF0122014B1A70F8BD00BF84
:10F5B8009249002038B50C461546FFF79BFA022CF5
:10F5C80003D0052C07D0012C15D12A46214615F069
:10F5D800DDFF002038BD2A4600210A4C15F0D6FF71
:10F5E8000420FFF70FFB2378002BF2D0FFF718FB5E
:10F5F80000232370EDE70448214636F042F86FF007
:10F608008500E7E792490020862B080870B5054673
:10F618000C4636F036FFD8B1237853B9144A284639
:10F628001370F5F78DF820B10121124A124836F00F
:10F6380077FC2678012E0BD100220D4B28461A7034
:10F64800F5F7E0F820B10D4A31460B4836F068FC72
:10F658002378052B06D16368054A003B18BF0123B0
:10F66800137070BD042B02BF0022014B1A70F8E71B
:10F6780091490020A32B0808B43D0708C32B0808AC
:10F6880013B5964835F0FDFF954835F0FAFF9549D2
:10F69800954836F057FF034638B1944A01219448FB
:10F6A80002B0BDE8104036F044BC92498E4836F0AE
:10F6B80049FF034608B1904AF0E790498A4836F076
:10F6C80041FF034608B18E4AE8E702F003FA98B909
:10F6D8000E2002F051FA02F003FAD8B90E2002F017
:10F6E80059FA8848F3F7E0FE014608B3864802B0A5
:10F6F800BDE8104035F0C5BF0121802014F046F860
:10F7080003460028E4D080228049814802F004FAA8
:10F718007F48DEE70121802014F038F803460028EE
:10F72800DCD080227B497C4802F0F6F97A48D6E79B
:10F738006D4836F066FE0128044650D1774835F00A
:10F74800A0FF2146764A6848F6F782F938B1754A2B
:10F758000121674802B0BDE8104036F0E1BB7248AD
:10F7680035F08FFF02F0B6F948B1704923462246BA
:10F778005D48F6F78DFA014608B16D48B7E702F023
:10F78800AFF940B101236B491A465748F6F780FA9A
:10F7980001460028F1D1012367491A465248F6F775
:10F7A80077FA014608B16548A1E7654835F069FF71
:10F7B80002F066FA60B1634835F063FF01236249DD
:10F7C8001A464948F6F764FA014608B15F488EE7D9
:10F7D80001210223EF224448009136F019FE5C48CB
:10F7E80035F04FFF00215B4A3F48F6F731F90446F0
:10F7F80008B1594AACE702F06DF978B1574835F0CD
:10F8080040FF0123224649493748F6F741FA28B113
:10F81800534802B0BDE8104035F033BF02F060F93C
:10F8280050B14E4835F02DFF0123002241492E48A2
:10F83800F6F72EFA0028EBD1012300223E492A4888
:10F84800F6F726FA044608B10146ACE702F018FAC2
:10F8580060B1444835F015FF3B4901232246224850
:10F86800F6F716FA014608B13F4840E7012402239B
:10F87800EF2200211C48009436F0CAFD3B4835F0C1
:10F8880000FF0021184836F0E7FD394835F0F9FE49
:10F898003849154837F022F908B1374A58E7374848
:10F8A80035F0EFFE02F018FB354835F0EAFE0E4859
:10F8B800F4F706FF034608B1324AEFE6324835F05E
:10F8C800E0FE094836F0DDFD30B90748F4F738FFA7
:10F8D800034608B12D4AE1E602B010BDE42B080842
:10F8E800F62B08088407002084120020122C080830
:10F8F800B43D07086C070020402C08085407002076
:10F90800722C0808E40600209F2C0808F43A07081F
:10F91800A8340020D83A070858340020C22C080818
:10F92800FC060020E32C08080A2D08086D1A0808B0
:10F93800302D08084D1A0808DC1A0808532D080845
:10F94800782D08089D2D08084E1C0808BF2D0808AA
:10F95800E52D080810070020062E08082D2E080897
:10F96800532E0808732E0808952E0808BB2E080881
:10F97800D12E080815F60108E72E08080B2F0808ED
:10F988001D2F0808282F0808512F0808622F08087B
:10F9980008B5064B1B7803F0FF002BB1044836F07E
:10F9A8006BFD80F00100C0B208BD00BF9149002086
:10F9B8008412002008B502F08DF80028014808BF1D
:10F9C800002008BDA834002038B50C460546084676
:10F9D8003AF0C7FC6C60606839F0A8FF20B90748A6
:10F9E80035F04FFE012038BD4FF48032217A60682F
:10F9F8003BF039F80028F5D12872F4E7AD2F080854
:10FA080038B5436804460D4658681A7A012303FA44
:10FA180002F1036982681B680B40003B18BF012391
:10FA2800AB4214BFD36813699847014610B1024826
:10FA380035F027FE657238BDC42F080838B543680D
:10FA48000129094A04460D4618BF4FF40032197AB5
:10FA580058683BF008F8014620B1044835F011FE1B
:10FA6800012038BDA572FCE706000200DC2F08085B
:10FA780008B5FEF781FC10B9FFF7F0F870B108BDC2
:10FA88000D4A934203D1BDE808403BF054BC0B4AF1
:10FA98009342F4D1BDE8084000F066BD0848036809
:10FAA800002BECD0074A9342E9D0074A9342E7D1AA
:10FAB800BDE8084044F067B8C44D07089C4B0708E8
:10FAC800F834002024600708B0C107084FF0FF335E
:10FAD80070B5204E204C336023682BB93368E3B9E6
:10FAE800BDE8704017F086BE1C4DAB42F6D01C4AEC
:10FAF800934204D1204644F05FF82560EEE7194AA6
:10FB0800934203D1204600F05FFDF6E7164A934280
:10FB1800F3D1204601F0C4F8EFE7144C2368002B1A
:10FB2800DED00E4DAB42DBD0114A934204D12046C1
:10FB38003BF0DDF82560D3E70E4A934203D1204617
:10FB480001F02CFAF6E70C4A9342F3D1204601F073
:10FB580035FDEFE79C070020F834002024600708F3
:10FB6800B0C107089C4B0708C44D0708943C002007
:10FB78003C4D0708404F070890510708F8B5334C2B
:10FB8800334E23680BB1B3420DD126603148036868
:10FB9800002B59D0B34257D02F4A934246D1BDE8E3
:10FBA800F84019F00DBA2D4A934216D16568A5425E
:10FBB80003D304F198039D42E8D9284610F064FE67
:10FBC8000028E3D0264B6C222946184653F078FBD0
:10FBD8006060284644F06EF8D8E7224A93421ED166
:10FBE8006568A54203D304F198039D42CED92846FF
:10FBF80010F04AFE0028C9D0194A2B46944605F150
:10FC0800200E174618685968083303C773453A46E3
:10FC1800F7D12846C4F804C044F0C0F9B6E7124A40
:10FC28009342B3D120463BF018FEAFE70F4A934208
:10FC380003D1BDE8F84000F0F3BC0D4A934203D16C
:10FC4800BDE8F84001F03EB8F8BD00BF943C002084
:10FC580024600708F8340020B0C107083C4D0708A5
:10FC68009C3C0020404F0708905107089C4B070810
:10FC7800C44D070808B5144803681BB9134803683E
:10FC88004BB908BD124A9342F8D0124A9342F5D1B3
:10FC98003BF074FEF2E70E4A9342F2D00E4A9342CA
:10FCA80003D1BDE8084043F096BF0C4A934203D104
:10FCB800BDE808403BF058BB094A9342E1D1BDE892
:10FCC80008403AF0AABF00BF943C0020F834002056
:10FCD8002460070890510708B0C10708C44D0708F9
:10FCE8009C4B070810B5084B084C1B68A34200D072
:10FCF80043B9B4220021064853F008FB044840F8F1
:10FD0800044D10BD0020FCE7F834002024600708EB
:10FD1800FC34002008B5FFF7E5FF10B9014803F0EF
:10FD280083FF08BD3D8D080810B5084B084C1B68BB
:10FD38000BB1A34208D194220021064853F0E6FAF9
:10FD4800044840F8044D10BD0020FCE7943C002016
:10FD580024600708983C002008B5FFF7E5FF10B9B4
:10FD6800014803F061FF08BD438D0808094B1B6873
:10FD78005A1C0DD0002B0BDCB8225343064A9818A6
:10FD8800D358064A934203D0002B08BF0E20704771
:10FD98000E2070479C070020F834002024600708D4
:10FDA8000E2807B506D14FF0FF330D4A136003B094
:10FDB8005DF804FB0B4B98421A6803D10A4B9A4230
:10FDC80000D05AB905F0A8FBC388E92200934FF484
:10FDD8008D7140F26113054803F062FF0023E4E7E8
:10FDE8009C070020F834002024600708479508087D
:10FDF800074A1368013304D1064B07491B688B4235
:10FE080000D17047002BFCD000231360704700BF5F
:10FE18009C070020F8340020246007082DE9F04FE3
:10FE280004464FF0000887B0CDE90312059300F1AE
:10FE38005009059B984502D307B0BDE8F08F049B95
:10FE480003EB080694F8B530757896F901B0002BE5
:10FE580035D0B57806F1030A48461AF043FB98B343
:10FE6800012300930021334694F8B620206D276EB5
:10FE7800B84700955346012194F8B620206D276EA7
:10FE8800B847484644F041FBBBF1000F23DB002094
:10FE98003BF0C4FE039B3BB1D4F88430164A93422E
:10FEA80002D020463AF048FEFEF766FA0028C3D191
:10FEB80094F8B5304544DBB905F10208B9E706F115
:10FEC800020A05F07F05C7E7FEF756FA0028C7D1F2
:10FED800FFF762F8C0E76B1C94F8B520DDB256FA5C
:10FEE80083F313445878FF2808BF4FF4FA70CFE71C
:10FEF80005F103089DE700BF24600708F0B54B6BC8
:10FF080005460C468BB0002B00F0D080012380F80A
:10FF18004030486B44F0E4FD85F83C00636B002BEF
:10FF280000F0C780A36B002B00F0C3804FF48073F0
:10FF3800A5F84030A06B44F0D3FD85F83D00B4F837
:10FF48005630002B14BF0123002385F8B43094F8F1
:10FF5800573018BF002685F8423094F8563018BF3D
:10FF6800042185F8433008BF0123626B0ABF194694
:10FF7800334694F855600AB9A26B32B1228EB2F5B5
:10FF8800807F02BF00260221334601220027CDE9E7
:10FF98000422CDE90222CDE9001305F10800638CA3
:10FFA800228BE18A45F006F894F8593008970993AE
:10FFB80094F8543005F15000CDE90673638D05932C
:10FFC800238D0493E38C0393A38C0293B4F920301C
:10FFD8000193B4F91E300093A38B628B21681AF049
:10FFE800F9F9A38D9FED357AA5F8AA3094F82E304B
:08FFF80085F8B030238EA5F856
:020000040802F0
:10000000AC3094F8323085F8B130D4ED117A67EE27
:10001000877AFCEEE77A17EE903AA5F8A83094F8C4
:100020004C3085F8B27085F8AF30D4ED147A67EEB5
:10003000877AFCEEE77AC5ED247A94F8543085F897
:10004000B36085F8B6306368C5F894302389A5F8A5
:10005000A030D4ED037A67EE877AFCEEE77A17EEEC
:10006000903AA5F8A6302369C5F89830A38AA5F878
:10007000A230E36BC5F89C30B4F84030A5F8A4304A
:10008000114BC5F8843094F8583085F8B530A36C1E
:100090004BB128460D4B40F8843FA16CFFF798FC0C
:1000A000A06C3AF060F9284609490BB0BDE8F04071
:1000B0003AF08BBD80F8403034E7002385F84130BA
:1000C00041E700BF00007A44246007084CC70708D6
:1000D000780A0020DFED077A20EE270ABCEEC00A7E
:1000E0000B68C0F894304B6880ED240AA0F8A0306B
:1000F000704700BF00007A4410B5038F04465A2BA6
:1001000028D0A3F5877CDCF1000343EB0C035A29CC
:100110001ED0A1F587704242424193421FBFA38E79
:10012000E28EE386A28604F1080044F006FF0C4B41
:100130009C4205D117F062FBE18EA08E17F000FA09
:10014000A06858B104F11801BDE8104044F09BB814
:100150000122E2E75A29E6D00123DAE710BD00BF09
:10016000F83400202DE9F04F97B090F8B2300446F3
:1001700002AFE3B1D0F88420B24B9A4217D1843059
:100180003AF091FC94F8AF30834204D10020543708
:10019000BD46BDE8F08FFEF7F7FC00212046B4F81D
:1001A000A230D4F8982084F8B210FFF73BFEA36881
:1001B000002B00F0C28120463AF010FD0028E5D166
:1001C00004F1500A504644F09DF90028DED094F81E
:1001D0004810002900F09C800023236304F12803C9
:1001E000FB6294F8B430002B40F0A380FEF7C8F80F
:1001F00038610028CAD120463AF0B4FC04F1080B5B
:100200005846F96A07F13802C7F808D044F074FF7D
:10021000002800F0878107F1380045F053F92025C8
:1002200094F83A30064607F13800B5FBF3F545F08F
:100230004EF9814607F1380045F049F9B0EBC51F8A
:100240004FEAC51800F2CC800123FB6180231FFA1E
:1002500089F09B00BB614009073323F0070301309D
:10026000ADEB030D78637B6B0DF108089B00073342
:1002700023F00703ADEB030D02ABBB62B4F8AC3067
:10028000B3F5807F14BF022301237B60BB69434425
:10029000FB6000237B6207F1380045F013F9B4F8E6
:1002A0007A303862B3F5807F05D05946504607F161
:1002B000380244F031F9B4F8AA3087F833307B6A59
:1002C0001BB1B4F8AC3087F8333050461AF00EF951
:1002D000002800F02781012394F8B6200093002124
:1002E00007F13303206D256EA847504644F011F9FD
:1002F000002399467B61BB8AFA699342C0F0A480CF
:1003000001227B6A7A627A6801339A42C3D809E192
:10031000A068002800F0118144F0AAF8F8620028D3
:1003200000F00B81B4F87A30B3F5807F7FF459AFD9
:1003300052E7204604F108063AF014FC3046C7F8AC
:1003400028D044F09EFE0546304644F09CFEC5F39E
:100350004F05EB1D23F00703ADEB030D0DF108096D
:100360002A4677218046484652F0D4FFB4F8AA3096
:10037000504687F844301AF0B9F8834688B12046D1
:10038000D7F828D03AF00DFC94F8B230002B3FF4A7
:100390002DAFFDF7F5FF00287FF428AFFEF700FE34
:1003A000F2E70123014694F8B6200093266E07F188
:1003B0004403206DB047504644F0ABF81FFA8BF36E
:1003C0009845DCD950461AF091F80BF1010B002842
:1003D000D5D094F8B62000954B460121266EE8E76B
:1003E00007F1380045F069F8B8FBF0F8464607F128
:1003F0003800012EB8BF012645F064F8B0FBF6F0D6
:1004000083B207F13800FB6145F05CF8B0FBF6F30E
:1004100003FB160080B218B1FB6901339BB2FB618C
:1004200007F1380045F049F816FB00F080B2B0FB48
:10043000F5F293B205FB1202002A3FF40AAF013332
:100440009BB206E74CC707083B69386A7A8FFB64A2
:100450003B8F8642A7F8443002EB090388BF3A6A13
:100460009BB298BF9219A7F8463095BF4A449B1893
:1004700093B29BB2A7F84A303B6AB7F93C109B1B7A
:100480009BB207F14400A7F848103B6245F01FF803
:10049000082294F83A300021B2FBF3F3B0FBF3F3F7
:1004A0007A6BB86A92001D4652F034FF0021404634
:1004B000BA6952F02FFF94F8B43013B940F2071321
:1004C000E3877B6AD3B194F8B33063B1062384F831
:1004D0003E3043465846BA6A07F1440144F0FFFDF6
:1004E00094F8B13013E094F8402012B184F83F3012
:1004F000EFE7B4F84230002BF2D0EAE74346584623
:10050000BA6A07F1440144F0EAFD94F8B030B3B997
:10051000504619F0EBFF7B69B14401337B611FFA50
:1005200089F9A8B9FB6AD7F808D09B68FB62002B51
:100530007FF464AE20463AF034FB012027E64346C0
:10054000FA689A42E4D01A68D24343F8042BF7E7DA
:10055000ABB294F8B620009301214346206D256E7E
:10056000A847504643F0D5FFFEF71AFDC3E600BF8B
:1005700010B590F8B23004463BB3D0F88420134B4A
:100580009A4214D184303AF08EFA94F8AF30834214
:100590001BD0FEF7F9FA002184F8B2102046B4F817
:1005A000A230D4F89820BDE81040FFF73BBC3AF0E9
:1005B00074F8D4E90432C01AB4F8A83061EB02012F
:1005C00083424FF000038B41E3D310BD4CC70708B3
:1005D00010B590F8B230044693B1D0F88420104B97
:1005E0009A4201D03AF0ACFAFEF7CEFA002120464A
:1005F000B4F8A230D4F8982084F8B210FFF712FCB7
:1006000004F1080044F05FFDD4F88420054B9A42C1
:1006100005D104F18400BDE810403AF039BA10BDAC
:10062000246007084CC7070810B504490446083081
:1006300044F0F9FC012384F8483010BD780A00200A
:1006400010B50B4C0B4B22689A420ED1A2680A4B94
:100650009A420AD120463AF0C1FA28B92046FFF75B
:1006600081FD80F00100C0B210BD0020FCE700BF9A
:10067000F83400209C4B0708780A002008B5014890
:1006800003F0CEFA0F94080810B504493DF04FF876
:1006900004460BF061FA204610BD00BF9C4B0708D2
:1006A000F0B50C4689B0064654F8040B1746FFF720
:1006B000EBFF054603AB01930B4B3A4621460093F3
:1006C000701E022306F04AFA052205A9039805F0D8
:1006D000C9FA049805F0D4F8284605A9FFF7FAFCF2
:1006E0000E2009B0F0BD00BF8C4B070808B5FFF71E
:1006F000CBFFFFF737FD10B9024803F099FA0E203F
:1007000008BD00BF7A8E080808B5FFF7BDFF3AF0B4
:1007100065FAD0B16430EFF7B9FE0D4B0022F0F767
:1007200059F8F0F7EFF907EE900AF4EE677AF1EE78
:1007300010FA7DBF17EE903A23F0030040F002005C
:10074000044878BFA0F1FF4008BD0348FCE700BFA4
:1007500000408F4002004000020080802DE9F04FF1
:100760002DED048BC9B0084611461A4628AB0193FB
:100770006E4B08AF009320233CF0E4FB289B05223E
:1007800039462998029305F06DFA05220BA92A989B
:1007900005F068FA40F246313E983AF02CFF5A22B2
:1007A000319E824696FBF2F302FB136313B160485D
:1007B00003F020FAFFF7B2FA04463D9805F060F81E
:1007C0004098F0EE408A05F05BF84698B0EE408A1B
:1007D00005F056F83A9B389803933B9B0E28B0EEF1
:1007E000409A049300F091803BF08CFF0546DDF8C1
:1007F000F0B00DF11C09494658469DF8148104F0EB
:10080000BDFF002800F0848003203EF0D5FF079A4A
:1008100003460270002208F1020942708270454AC4
:10082000002122600DF14E005222059352F072FD1C
:100830003A68029B12927A681193ADF84C200B9A99
:100840008DED149A15920C9AADF86660ADF85820AB
:100850002B9A2046ADF85A202C9A11A9ADF85C20AD
:100860002D9AADF85E202E9AADF860202F9AADF843
:100870006220309AADF86420329AADF86820339A3D
:10088000ADF86A20349AADF86C20359AADF86E2038
:10089000369A039BADF870201E93049B9DF8DC20D4
:1008A0001F93059B8DF8722020939DF8FC309DF8D6
:1008B000E4208DF890309DF80431CDED228A8DF83A
:1008C00098309DF808318DED258A8DF899309DF886
:1008D0000C31ADF874508DF89A309DF810318DF8C8
:1008E00076208DF89B309DF81C31ADF88490CDF8C2
:1008F0008CA08DF89C808DF89D30FFF703FB20467F
:1009000049B0BDEC048BBDE8F08F4FF480756EE705
:10091000012258460EA905F0A5F910B1DDE90E39FE
:100920007DE740F20251044803F0AAF98C4A070817
:10093000539208089C4B0708DC90080870B58AB0F1
:1009400004AB01931B4B0C46009304310323013885
:1009500006F004F9FF22002140F26733049806F004
:1009600099F905228DF80F0007A90598246805F06C
:1009700079F920463AF07AFAC0B101259DF818605D
:10098000204632460DF10F03002100953AF08EFA11
:10099000089B3246294620460093079B3AF086FA88
:1009A00020463AF002FB0E200AB070BDFEF7F8FABE
:1009B000DFE700BF244D070870B58CB0084611462C
:1009C0001A4605AB0193184B009307233CF0BAFA83
:1009D00040F277521549059806F0DAF90646FFF716
:1009E000BFF9134B04460360012240F2DC430021AF
:1009F0000A9806F04FF940F2D14305460122002142
:100A00000B9806F047F9099BC0B20193089BEDB221
:100A1000039000932046DDE90623314602953AF023
:100A2000B3F920460CB070BDEC4C0708F4C30708BE
:100A30003C4D070808B53AF08BF920B940F2145143
:100A4000024803F0FDF80E2008BD00BFE98F08083A
:100A500010B5038F04465A2B28D0A3F5877CDCF110
:100A6000000343EB0C035A291ED0A1F587704242C4
:100A7000424193421FBFA38EE28EE386A28604F119
:100A8000080044F05AFA0C4B9C4205D116F0B6FE11
:100A9000E18EA08E16F054FDA06858B104F1180143
:100AA000BDE8104043F0EFBB0122E2E75A29E6D04F
:100AB0000123DAE710BD00BFF8340020F8B590F844
:100AC000783004460D46174643B10023204684F88B
:100AD00079303AF07AFA01263046F8BD90F879601C
:100AE000002EF2D14B1CF0D039F0D7FD2369C31A88
:100AF000BB4202D90D4803F09BF8A26EC4E91A016B
:100B0000821A9542E8D3B3FBF5F205FB1233ED1AD6
:100B100039F0C3FDD4E91A32C01A61EB0201A842D0
:100B200071F10001D1D2FEF73BFAF1E79993080881
:100B30002DE9F04F1F4600238BB0044680F8783033
:100B4000016540F2E74090460EF084FD6065C369A0
:100B5000002B00F09080206D984786B2636D206D69
:100B60001B69984783B20793636D206D5B69984753
:100B700083B20893636D04F1080B5B6A002B7CD091
:100B8000206D98478146636DDD6A15B1206DA847D9
:100B90000546636D9B69002B76D0206D98475FFA00
:100BA00080FA636D1B6B13B1206D98470346626D2D
:100BB000526B22B1206D099390470246099BCDE903
:100BC0000432DDE9071200235846CDE9025ACDE987
:100BD000006944F0F3F9636D1B6A13B1206D984707
:100BE00083B2A4F87430636D9B6B002B4FD1A38E3E
:100BF00094F83A205343DB10A4F87630636D206DEF
:100C00005B6804F158019847E28EB4F87610B4F8A6
:100C10007430013A01FB023394F83A20A18EE06D62
:100C200051434FF47E7203EBD10106F07DF887F05B
:100C3000010384F87930636D9B6A83B3206D984714
:100C400080B24FF47A73B3FBF0F3A4F87000A4F809
:100C50007230B8F1000F03D041462046FFF7F8FE8E
:100C60005846104944F0DFF9394620460BB0BDE83C
:100C7000F04F3AF050BB102670E7072E8CBF4FF0B4
:100C800000094FF001097EE74FF0020A89E7206D65
:100C9000984780B2A4F876000028AFD1A7E73C209F
:100CA000CFE700BF780A002010B5044600213AF0D3
:100CB00032FB04F1080044F006FA636D206DDB6836
:100CC0009847014B236010BD2460070810B5044607
:100CD000006D04F025FC78B10A4B98420CD001213C
:100CE00020463AF018FB084904F1080044F09BF94B
:100CF000012384F8483010BD2046BDE81040FFF7BE
:100D0000D3BF00BF24600708780A002008B5083068
:100D100044F089F910B9024802F06CFF0E2008BDBA
:100D20007391080808B5014802F07AFF0F9408088B
:100D300010B504493CF0FBFC04460AF00DFF2046C8
:100D400010BD00BFC44D070830B50C4685B002ABDE
:100D50000193154B043100930138022305F0FEFE88
:100D60002068FFF7E5FF039B0546002BC8BF4FF443
:100D70007A740298CCBF94FBF3F44FF0FF340E2842
:100D80000FD03BF0BFFC4FF47A7191FBF0F122469B
:100D90002846FFF793FE00280CBF1E203E2005B01A
:100DA00030BD4FF0FF31F2E7B44D070808B5FFF74B
:100DB000BFFF3AF097FAB5EEC00AF1EE10FA02D58D
:100DC000094802F035FFB4EE400AF1EE10FA7DBF9B
:100DD00010EE103A23F0030040F00200034878BF01
:100DE000A0F1FF4008BD00BF6A9308080200400060
:100DF00038B50C46FFF79CFF0E2C05460AD020465E
:100E00001AF050FA01462846FFF780FF20B9034840
:100E100002F0F0FE0021F6E70E2038BD73910808BD
:100E200070B586B0084611461A4603AB01930F4BC6
:100E3000009303233CF086F8DDE903655A2295FB15
:100E4000F2F302FB135313B1094802F0D3FEFEF78D
:100E500065FF0446074B314603609DF81430AAB283
:100E6000FFF766FE204606B070BD00BF8C4D070838
:100E700053920808C44D070838B50D46FFF758FFD0
:100E80000446284604F0FCFCB5EEC00AF1EE10FA68
:100E900006D4B7EE007AB4EEC70AF1EE10FA06DD1A
:100EA0000123002240F23E31054802F0E9FE2046CF
:100EB0003AF020FA10B9034802F0BAFE0E2038BD0D
:100EC000769508086A9308082DE9F0430C468DB022
:100ED00002AF07F1080301932E4B04310093013850
:100EE000022305F03BFE2068FFF722FFD7E90286C8
:100EF00005460622304607F1100104F0B3FEBB6937
:100F0000012B02D0244802F075FE95F83A30102BE0
:100F100001D02248F7E70024B5F83490FC6107F1CE
:100F20001C00A7F81E8008F101087C62A7F8209039
:100F3000A7F8228044F0CBFA00F0010281B2786970
:100F400002EB5902B0EB820F3B6920D34A09A44659
:100F5000214601327A607A689200073222F0070255
:100F6000ADEB020D02AA7C6888B2844201F1010156
:100F70000AD807F11C0105F1080044F0B0F830462A
:100F80002C37BD46BDE8F08342F820C0EBE70448AB
:100F9000B9E700BFA44D07085F93080866920808E8
:100FA0004993080810B50446406804F108039842C4
:100FB00001D142F0F6FF0023A26A6360044B9A421B
:100FC00005D104F12800BDE8104039F061BD10BD25
:100FD0004CC7070810B50A4B826A9A420ED000F13E
:100FE000280400212046FEF70FFD04203AF0AFFA56
:100FF00020460121FEF708FD012010BD0020FCE77E
:10100000246007082DE9F04104460E4615461F46A8
:101010007BB9154B83623046E9B242F0C4FFE0B9B8
:10102000114B20462360FFF7BDFF29460F4802F011
:1010300027FE80460E4B394648F8283F4046FEF7CB
:10104000C7FC00220121404639F04AFD384639F0FC
:101050008AF92046FFF7BEFFDDE73046666043F0C1
:1010600038F8A586BDE8F08124600708CB8C080815
:101070004CC7070870B586B0084611461A4603AB40
:101080000193104B009303233BF05CFF40F214519B
:1010900005983AF0B0FA40F22E4206460A49039803
:1010A00005F076FE0546FEF75BFE0446074B294633
:1010B0000360BDF810203346FFF7A4FF204606B0BA
:1010C00070BD00BF284F07089CC50708404F0708A0
:1010D00008B5FFF77FFF20B940F21451024802F033
:1010E000AFFD0E2008BD00BFE98F080810B50A4CFF
:1010F00023686BB938F0CFFE08B9FBF7B1FBEFF30B
:101100001182102383F31288BFF36F8F034B1A6091
:1011100023680133236010BD2C3D0020303D0020AA
:1011200008B50C4B1A6812B90520FEF7E5F81A68E5
:10113000013A1A601B6863B9074B1B6883F3118877
:10114000BFF36F8F38F0A7FE18B9BDE80840FBF772
:101150009BBB08BD2C3D0020303D002008B539F078
:1011600007F9BDE80840014601483BF035BF00BF24
:1011700058500708F7B5184CA568E6680195002592
:10118000019FECB2A74215D8144CA568E6680195FA
:101190000025019FECB2BC421CD206EBC40CDCF86B
:1011A00004700135B842F4D140F28A40086040F240
:1011B000D3410AE006EBC40CDCF804700135874229
:1011C000DED1002008604FF44E71116056F83420D3
:1011D00012091A6003B0F0BD9C9D07080C9F070818
:1011E00040F2922310B586B00393059304AA05AB91
:1011F0000446084603A9FFF7BDFFDDE90312059B7E
:1012000041B10093204613460A4606493BF0B4F824
:1012100006B010BD2046044906B0BDE810403BF0C2
:10122000ABB800BFF92F0808FC2F08080A4601498F
:1012300005F0AEBD045107081FB5044688B10E285D
:101240000FD039F093F860B940F29223204603930F
:1012500001A903AB02AAFFF78DFF0399024802F030
:101260000FFD04B010BD00BFB89508080E2373B57C
:101270000B600D4601A901F09DF8012804460FD925
:10128000019E3046EFF758FE0246012A03D9531E4D
:10129000F15C2F2907D03146044807F08BFD286008
:1012A000204602B070BD1A46EFE700BF3C60070859
:1012B0000E2373B50B600D4601A901F07BF80128E0
:1012C000044609D9019E3046EFF736FE3146024604
:1012D000034807F06FFD2860204602B070BD00BFD4
:1012E0003C600708F8B5037806462F2B00AF6BD09B
:1012F000514CD4F8B45045B902203EF05DFA054691
:101300004E49EFF711FEC4F8B4502846EFF714FE2B
:1013100004463046EFF710FE204402303EF04CFA0F
:1013200004462846EFF708FE29460246204651F0BB
:10133000CBFF2846EFF700FE054638B1231813F817
:10134000013C2F2B1EBF2F23013523543046EFF7CE
:10135000F3FD3146421C601951F0B6FF2046EFF70D
:10136000EBFD002221461346154690422ED145B38F
:101370009B00073323F00703ADEB030D2046EFF787
:10138000DBFD00236E4619461A46651E204415F8FB
:1013900001EF01F1010CBEF12F0F04F801E002D0C2
:1013A000BEF1000F45D1012B2FD115F8013C2E2B9A
:1013B0003AD1531E56F823100023A842E7D1002348
:1013C00063542046BD46F8BD1D4D9EE711F8016BE4
:1013D00002F1020E2F2E08BF0133704502F1010CFD
:1013E0000FD92F2E0DD10E782E2E0AD14E782E2EFB
:1013F00007D10332904206D08A782F2A08BF45F0E1
:1014000001056246B1E70125FBE7022B0CD115F877
:10141000013C2E2B08D115F8023C2E2B04D1012AB9
:1014200088BF02F1FF32C4E746F822C061460132AC
:10143000C2E761460133C0E728400020240C0808B9
:10144000A729080837B5FFF74DFF124C6946C4F8C5
:10145000B400FFF70BFFC4F8EC00B0B9D4F8F040CB
:101460000CB903B030BD6568012D0CD129460A487E
:1014700007F07AFC2A46019040F25231204601AB37
:101480003AF0CCF8EDE7E468EAE76B46012240F277
:101490005231F5E728400020240C080810B5084B0D
:1014A000D3F8B4404CB12046EFF746FD2146BDE8E5
:1014B00010400246034807F07DBC662010BD00BF07
:1014C000284000203C60070837B5FFF70BFF01A953
:1014D000FFF7CCFE28B9144BD3F8F000A0B966236F
:1014E0000193012240F2324101AB3AF097F800211A
:1014F000054608463BF0C4FA0446284602F094FF2D
:1015000038B9204603B030BD4368012BE7D0C0682E
:10151000E4E70422012104F069FB014620463BF088
:101520009BF9FDF73DFDE8E72840002013B5FFF7E4
:10153000D9FE01A9FFF79AFE044610B9112003F065
:10154000F7FA012807D0019808F04CF90649EFF79F
:10155000E1FC0028F2D0012240F29141204601AB8B
:101560003AF05CF802B010BD240C080807B5FFF78C
:10157000B9FE01A9FFF79CFED8B9114BD3F8F000D2
:1015800080B901460A200CF019FF0121031D00F16A
:10159000280243F8041F9342FBD1C123C36203B066
:1015A0005DF804FB4368012B01D0C068E8E76623BF
:1015B0000193012240F2825101AB3AF02FF8EEE79D
:1015C0002840002010B50D4B026804469A4214D101
:1015D000406804F10803984201D142F06EFBA06F0D
:1015E00038F0C2FED4F8800012F0F4F82046BDE8CE
:1015F00010409822002151F08DBE10BD9051070877
:1016000070B58AB0084611461A4604AB0193124BD6
:10161000009306233BF096FC40F25331059839F0D5
:10162000E2FF40F277510646049818F0F1F80546BB
:10163000FEF796FB0446094B324603609DF82430C2
:1016400029460293079B0193069B0093089B3AF05F
:101650006FF920460AB070BD605107089051070825
:1016600038B5437904468B420D4609D0837913B1CE
:1016700004483AF0A7FA6571BDE83840FDF730BB81
:1016800038BD00BF6C08002038B50C460F4D114620
:101690001A460F4B9D4201D134F02AFE0D4B9D425C
:1016A000FAD00D4B9D42F7D00C4B9D42F4D0A307CE
:1016B0000AD12368AB4207D143F0F9F8014620462E
:1016C000BDE8384044F0D3BD38BD00BFB0D50708F1
:1016D00000600708A85E07083C6007082460070848
:1016E000F7B514460AB1002313701C4BDFF87CE0F9
:1016F000734501D134F0FCFD194FBB42FAD0194EAD
:10170000B342F7D0DFF868C06345F3D010F00302AE
:101710000FD105689D420CD18DF807200DF107020D
:1017200044F08FFB14B19DF80730237080B203B0F2
:10173000F0BD0D4B7345DDD0BB42DBD0B342D9D0F9
:101740006345D7D012B14FF6FF70F0E702689A42B6
:10175000F9D144F0CCF9FF28E9D1F4E7B0D5070876
:10176000A85E07083C6007089CD0070800600708CF
:10177000246007082DE9F04F0446E36888461046C8
:1017800085B043B10F468B1865890193019B9F4239
:1017900004D3A7EB080005B0BDE8F08F38463AF057
:1017A000C7FE814638463AF0DEFE94F82010074620
:1017B00019B3B9F11B0F08D103785C2B05D10023B5
:1017C000013784F820306361E0E7E38B002BDDD143
:1017D0002369002BDAD0E28A5B8B9A42D6D2636906
:1017E00023B90122204611463AF0CAF901234A469C
:1017F000194620463AF03DF9C8E7B9F11F0F00F24B
:101800003581B9F10D0F0CD8B9F1070F0CD9A9F139
:101810000809B9F1050F07D8DFE809F060505C0648
:10182000064DB9F11B0F5ED0E0682389028B294673
:101830009A4208D8628901326281028BB3FBF2F5C9
:1018400002FB153323816589428B954221BFB5FB8D
:10185000F2F302FB13539DB26581A94296D0468BE9
:10186000B4F81CC0AA19531E93FBF6F106FB113104
:10187000438C6344B3FBF6FE06FB1E33994285D1CD
:10188000618B51B9731E9C4507D10132B2FBF6F34F
:1018900006FB132292B243F0C8F800266589268120
:1018A000E26833B2128B01369342C0F2E580002326
:1018B000658123816AE700232381B5E7042601239C
:1018C000202200212046013E3AF0D3F816F0FF0610
:1018D000F5D1A9E7638901336381A5E72389002B4B
:1018E000A2D0013BE8E70126ADF80A10BB5DA3F1E9
:1018F0003002092A36D801EB810103EB410301369E
:10190000303B062E19B2F1D13B785B2B40F09F8023
:101910004FF0020C02A8B9F13B0F26D0A9F13F0904
:10192000E068B9F10C0F4BD801A353F829F000BFC0
:1019300029180208C1190208C1190208C1190208B0
:10194000C1190208DD190208C1190208C1190208EB
:10195000C1190208071A0208C1190208EB19020886
:10196000AD1902089946F6B2CEE70023721CD6B232
:1019700057FA82F20B2E438010D812F801EBAEF129
:10198000300ABAF1090F08D803EB83030EEB4303C7
:10199000303B01361BB2F6B2ECE7F146BCF1010F69
:1019A00000F10200BAD04FF0010CB4E7B4F808908F
:1019B000D4F808A0B0F918B0D94504DBC4F808A0E1
:1019C0000136374430E7012320220021204609F167
:1019D00001093AF04EF81FFA89F9EDE72389994297
:1019E000CCBF00235B1A2381EAE70229E8D1002259
:1019F0000025114643F019F8012229462046A5602A
:101A00003AF0BEF8DCE7BDF90A300029C8BF01F1A1
:101A1000FF31428BC8BF09B2002BC8BF03F1FF33AF
:101A2000058BC8BF1BB29142A4BF02F1FF3109B2BE
:101A3000AB42A4BF05F1FF352BB2458C23810D4489
:101A400095FBF2F102FB1155ADB26581B8E75D2B54
:101A50007FF4EAAEB9F13B0F7FF4E6AE01231E44FA
:101A600084F82030E18357FA86F7DDE601234A4601
:101A7000204639F0FEFFD7E6012320220021204630
:101A800039F0F7FF0CE700BF002373B50DF1070035
:101A90008DF807303EF0BBFB094B9DF80760A0FBBB
:101AA000035403FB0144430843EAC173E81847F2B7
:101AB000367344EB5101C6FB830102B070BD00BF19
:101AC000B2E60E000122034B1A700022024B1A707C
:101AD000704700BF9549002094490020014B1878B9
:101AE000704700BF95490020014B1878704700BF30
:101AF000944900200023034A01201370024A137006
:101B0000704700BF9549002094490020024B18708F
:101B1000024B01201970704795490020944900201C
:101B200010B5044617F060FC014B2046236010BD41
:101B3000E852070808B5FFF7DDFF10B9024802F0C8
:101B400077F80E2008BD00BFF49208081FB502AB5D
:101B50000193094B0093022305F000F89DF80C1047
:101B60009DF80800FFF7D2FF10B9044802F060F8B2
:101B70000E2005B05DF804FBBC520708F49208087B
:101B800010B50022044643F2F661034810F076FFD8
:101B900000B1446010BD00BFAC07002010B50022AA
:101BA000044643F61601034810F068FF00B1446094
:101BB00010BD00BFAC07002008B53AF04EF8B5EEF6
:101BC000C00AF1EE10FA0FD4B4EE400AF1EE10FAAA
:101BD0007DBF10EE103A23F0030040F002000348EE
:101BE00078BFA0F1FF4008BD0E20FCE702004000D6
:101BF00008B53AF02EF8B5EEC00AF1EE10FA0FD49F
